:10F0000038B504460D460DF0B7FC0848216801608C
:10F0100061684160A16881600DF020FB0CF097F8F9
:10F020002846BDE8324003F08CBA00BF30480020CB
:10F03000DFF8481C0870704738B5DFF8444CDFF83B
:10F04000445C20762878C00000F0C4FFE061C8B1BD
:10F05000002108E04FF6FF7220F8312000EBC103D9
:10F0600000225A60491C2A789142F3DB052000F007
:10F07000AEF8207E01F06DF8BDE83240DFF8080CF4
:10F0800001F0DABC31BD38B50C46200418D5DFF8E4
:10F09000F00B007E01F0D9FE05000ED02878B028D4
:10F0A00008D1284600F0FAF820B1297905F10800C6
:10F0B00002F0B4FA284601F05BFE84F4004032BD51
:10F0C000002032BD7CB504001D460CD0ADF8001008
:10F0D0008DF80220019400A800F0CFFF060019D19E
:10F0E000C5B164890CB9022614E00C2000F072FF4F
:10F0F00008B913260EE00021016084808560DFF8E6
:10F100008C1B0A6812B9086004E00A4611680029DD
:10F11000FBD11060304676BD30B50D46DFF86C1B74
:10F120000446086883B0002201E00246006890B1FE
:10F130008388A342F9D10368002A0CBF0B601360D7
:10F1400000F055FF00A9204600F0E3FF10B90DB113
:10F15000019929603EBD01203EBD70B558BB012913
:10F1600027D1DFF81C0BC16900230C2601E05B1CD2
:10F17000DBB2DFF8104B2478A34216DA31F83340C3
:10F180004FF6FF75AC42F2D0002400E0641C457ECF
:10F19000E4B2AC42EBD201EBC3056D6806FB04554B
:10F1A0002D88002DF2D0012070BDBDE87040107890
:10F1B0000DE0182070BD022070BD0022002803BFA2
:10F1C000DFF8BC0A407E08700222104670472DE925
:10F1D000F843DFF8AC7A0446002078760C25F8690D
:10F1E000DFF8A06A406805FB04F868B100F0FFFE94
:10F1F0000020002204E0F96901EBC001401C4A60D4
:10F20000C0B231788842F6D3307808FB00F080B283
:10F2100000F0E0FE5FEA000927D0307808FB00F23A
:10F220000021484601F075FD00200FE0516805FB04
:10F230000CF34FF0000E23F801E059180CF1010C0B
:10F24000C1F808E0A445F1DBC144401C3178C0B2EC
:10F25000884207D2F96901EBC0024FF0000CC2F8F6
:10F260000490EFE77C76002000E01320BDE8F283F5
:10F2700001460020C90705D5002310220121DFF82F
:10F280000C0D1FE77047DFF8041A096821B18A885E
:10F290008242FAD188687047002070472DE9F04318
:10F2A00087B004460020ADF8100001208DF8120050
:10F2B000DFF8CC59286A38B902F050FA00F08AFE1B
:10F2C0000028286200F0E48018220021284601F07E
:10F2D00020FD2079022800F1010804F108074FF60B
:10F2E000FF7917D006282CD008282FD00A2832D032
:10F2F0000C2855D00E2800F08880102800F08A8055
:10F30000122800F08C80162800F09080182800F059
:10F310009480BAE002F022FA28802946608802F040
:10F320003BFA00283988288804D0814228BF01464A
:10F3300029809DE0814228BF0146608802F0DBF809
:10F34000A3E004A9204600F0ADF87AE004A9204625
:10F3500000F02FF975E000F0A0F8060050D06088AA
:10F3600005AB4A460B2102F01DF903006B6023D068
:10F370002079BDF81620039000953146BDF81400A1
:10F3800000F0A1F900F026FA060004D160882946B1
:10F3900002F04CFA29E0162E686808BF00262BE020
:10F3A00000F07BF806002BD0608805AB4A460D21A3
:10F3B00002F0F8F8686020B93888ADF8100011261E
:10F3C00043E02179BDF8162003910346BDF81410DF
:10F3D0000291798801910095314600F0FBF9060011
:10F3E00006D16088294602F02FFA002840D129E092
:10F3F000162E686808BF002602F0CFFA0EB921E089
:10F4000001263888ADF810001CE004A9204600F061
:10F410005EF916E004A9204600F0E3F911E00DF1D1
:10F42000120204A9204600F07EFA0AE00DF1120251
:10F4300004A9204600F0BFFA03E004A9204600F02A
:10F4400028FB064696B1162E12D0607814280DD0EF
:10F45000207928702946BDF8100068802E716088D8
:10F4600002F091F910B14FF0010801E0162E0CD115
:10F4700060882B465FFA88F2162102F032F820B13C
:10F480005FFA88F1284602F0C9F8204601F060FFD3
:10F490009DF8120007B0BDE8F08338880DF1160121
:10F4A00000F0CDBE2DE9FA4786B0044604F1080508
:10F4B00000F034FA05906A1D0DF1120000902B79CE
:10F4C0006988288800F08DFE002780464FF0FF0AEB
:10F4D000B8F1000F5BD009E0BDF810300B54BDF857
:10F4E0001000716892B2000A5054571C0598BFB2C0
:10F4F000401F87424BDA2079BDF8122003904FF06D
:10F5000000090598CDF80490C01F80B202904146D2
:10F5100000F05CF9002802BF728B2889904214D158
:10F52000316AE86801F0E7FB78B1706858B900F01B
:10F5300048F9072102F036F8706020B9069928884A
:10F540000880112032E0B8F80A90BDF812206988CE
:10F5500004AB404600F097FEB9F1000F8046B7D0EB
:10F56000706807F80090781C726880B24FEA292111
:10F570008154411C4A1C7068B8F1000F89B2ABD1AC
:10F5800001F800A092B2706802F800A0571CBFB248
:10F5900047B1B80830803146608802F021F928B1BF
:10F5A000162003E00699288808800A2008B0BDE8E4
:10F5B000F0872DE9F04F89B0044604F1080005906A
:10F5C0008A4606886088DFF8B85602F0EFFB07909D
:10F5D0000027001FB84606904FF6FF7900E0761C22
:10F5E0000698B84257DB04A8009005980379418833
:10F5F000421DB0B200F0F5FD5FEA000B4BD0BBF846
:10F600000A60BDF810209BF80810608800F0A5FD86
:10F610005FEA00083FD100F0DFF859460798001F65
:10F6200000F050F805F11A0000902B6A00F0D2F8B3
:10F630005FEA00082FD17FB9608800234A4609217C
:10F6400001F0B0FF686018B9AAF80060112036E038
:10F65000688B801C688004E0698B6888891C8842FC
:10F660001AD1698B0698C919884214DB6968BBF8FE
:10F670000A007854BBF80A106A6800F049F9686813
:10F680006A8B296ABFB2381801F011FB688BC71961
:10F690004E45BFB2A3D157B1688897FBF0F02880E0
:10F6A0002946608802F0ACF848B1162007E0B8F1AE
:10F6B000000F08BF4FF00A08AAF80060404609B0E2
:10F6C000BDE8F08F80B202900020019070472DE9D4
:10F6D000F04F85B00D46044604F108066088DFF857
:10F6E000A07502F063FB4FF0000BA0F10108A0F140
:10F6F000010A16E039887A8B084612189245BCBF79
:10F70000A8EB010179837B687A8B396AC01801F014
:10F71000CEFA3888798B081838800BF101001FFA6F
:10F7200080FBB0888345BCBF3888504537DA3068E5
:10F7300010F81B2000EB4B0004A9407802EB0020DE
:10F7400080B200F07CFD01000BD14FF0010900F008
:10F750002EF8786808B102F020F9484605B0BDE8F7
:10F76000F08F00F039F81FFA88F0FFF7ACFF07F1CF
:10F770001A0000903B6A00F02DF85FEA0009E6D11C
:10F7800078680028B6D100F01CF80F2101F00AFFBC
:10F7900000287860AED100F00AF81120DEE760881A
:10F7A000394602F05FF80028D8D01620D6E7306836
:10F7B00010F81B1000EB4B00407801EB0020288074
:10F7C0007047608800234FF6FF72704706F11A00F9
:10F7D0000090336A608861E22079BDF810200390C0
:10F7E00070472DE9F04786B08846044604F10809C1
:10F7F00000F094F8059009F1050204A8009099F82A
:10F800000430B9F80210B9F8000000F0EAFC002753
:10F81000BA4605460FE07268FF21B95480B272689B
:10F820008154471C7068728B316ABFB2381801F07E
:10F830003EFA708BC719BFB2BDB1BDF81020297A4E
:10F84000608800F08AFC5FEA000A0BD1FFF7C4FF72
:10F8500029460598801FFFF735FFFFF7B7FF5FEADE
:10F86000000A10D06889A8F80000002F43D07088E3
:10F8700097FBF0F030803146608802F002F80028F3
:10F8800043D0162041E07FB9FFF79BFF112101F023
:10F8900089FE706020B96889A8F80000112034E062
:10F8A000708B001D708009E0708B7188021D914281
:10F8B000DDD10599891FC0198142D8DB716868893B
:10F8C00078546989726800F023F8BDF81020B9F8FF
:10F8D00002100DF11203284600F0D5FC0546781CF5
:10F8E000002DBFB297D07268BDF81210B954BDF8A0
:10F8F0001210090A92E7B9F80000A8F80000BAF15E
:10F90000000F08BF4FF00A0A504606B0BDE8F08766
:10F91000781C80B2090A8154471C70476088DFF860
:10F92000606302F043BA2DE9F041044604F1080790
:10F9300084B00D463888904602A900F080FC06008D
:10F940002FD0307A80060BD5BDF8080000F0A0F962
:10F9500003000BD06088122231469847060021D15F
:10F96000787A002814BF5220207901E00E2619E091
:10F970000190002000907B887A683988608800F0C8
:10F9800087FA060007D1787A70B9608801F08AFF9B
:10F9900050B116200CE0162E04D1002688F8006025
:10F9A00002E0012638882880787A00B100263046A7
:10F9B00004B0BDE8F0812DE9F84389469046012165
:10F9C000044604F10806608801F0BAF8002718B967
:10F9D000142060700E205AE0308800A900F02FFC3F
:10F9E00005004FD0287A80060BD5BDF8000000F046
:10F9F0004FF9030015D06088122229469847070066
:10FA000041D16588284600F006F9010006D14FF67D
:10FA1000FF7000F000F9010030D00D800022984DF9
:10FA200002E00E272FE0521C687ED2B2824225D21D
:10FA300048680C2303FB02000388002BF3D10C223F
:10FA4000314601F034F9002088F800000C223146DC
:10FA5000284601F02CF9B28860880023172101F0B4
:10FA6000A1FDA86060B1B288B16801F020F960889A
:10FA7000294601F01DFF48B1162008E0092702E0E1
:10FA8000112700E001273088A9F800003846BDE8BA
:10FA9000F2832DE9F04383B089460027044604F140
:10FAA0000805608800F0B7F85FEA00084AD02878B7
:10FAB000012843D14146284600F050F8A0B1D8F8BB
:10FAC00004501820019068880090AB88AA682988A3
:10FAD000608800F0DDF90746162F02D10020A860EB
:10FAE0002CE05FB3288827E000250EE001907088A5
:10FAF0000090B388B268608800F0CAF90746162FF4
:10FB000017D10020B0606D1CEDB25D48407E85428B
:10FB100014DAD8F804100C2202FB051216463188BC
:10FB200061B16B1C83421DBF9089002816201820EC
:10FB3000DCE7002FE7D03088A9F80000404600F04D
:10FB40007DF82FB9608801F0C0FE20B1162003E0D7
:10FB5000162F08BF00273846BDE8FE832DE9F84F71
:10FB60000C46002100250E464FF00C0B44480EE0D9
:10FB7000994202BFBCF8027093B2BB4224D1BCF8D8
:10FB800004305D19ADB29A18761C92B2F6B2437E7B
:10FB90009E420EDA63680BFB063CBCF8003043B1B2
:10FBA0000029E5D1BCF80450BCF802201946AA1877
:10FBB000EAE7022E2CDB28004FF0000904D001F008
:10FBC000D5FE5FEA000801D1002022E0CA4619E014
:10FBD0000BFB0A07B96859B1BA8809EB080001F0B4
:10FBE00066F8B88848441FFA80F9B86801F0D5FE75
:10FBF000BAF1000F04D00C220021384601F089F838
:10FC00000AF1010AB2456068E2DBC0F8088085802D
:10FC10000120BDE8F28F1A4AD269002100E0491C98
:10FC2000184B1B78C9B2994206D232F83130834260
:10FC3000F5D102EBC10070470020704770B5044653
:10FC400000250BE0B06808B101F0A7FE0C220021EE
:10FC5000304601F05EF8002030806D1C0848407E80
:10FC6000EDB2854206D260680C2101FB05063088A2
:10FC70000028E7D14FF6FF70208070BDA24600201B
:10FC8000D44700206C47002037FF00009C4800202C
:10FC900080B5FFF7F8FA00B1806802BD2DE9FE4F8C
:10FCA0000D468046287AC00693461E464FF0000A4D
:10FCB0000CD55846FFF7ECFF030000F0E4800A2261
:10FCC0002946404698475FEA000A49D128780C9FA8
:10FCD0000D9CDDF83890022816D100F016F94FF48B
:10FCE0002051401A012810D9801E3AD0401E14D04D
:10FCF000FD3876D0401E00F07D80401E6AD0401E48
:10FD00006FD0401E00F09180A7E0002C2AD1E86857
:10FD1000017839800278416883E0002C22D10120EB
:10FD200038800021E868007830706889401C80B213
:10FD300000F085FA398860B10278921C5118398038
:10FD4000418971704189090AB17002784168F01CDB
:10FD500068E0081D388004220021701C00F0D9FFE3
:10FD600093E0002C62D1E868048804203880347065
:10FD7000200A70700DF10201204600F060FA0500C3
:10FD80001ED0EC68BDF802204FF6FF7800AB41466C
:10FD900000F079FA40B92B786A688B48022101F0AB
:10FDA000B4FF08B9ADF80080207802280AD1616854
:10FDB0000222301D00F07BFF3888801C388001E073
:10FDC000ADF80040BDF80000B070BDF80000000ABA
:10FDD000F0705AE054BBE8680168404602F018F839
:10FDE00002E01CBBE8680088022139803070000AFC
:10FDF00070704AE0E86800F058FF82B2A242B8BFD3
:10FE00004FF0070A41DB944208BF002206D009EBFD
:10FE100004019142B2BF4A46121B92B23A80E9688D
:10FE20006118304600F043FF2FE014B14FF00B0A89
:10FE30002BE0E868072139800178317041787170D2
:10FE40004188B1704188090AF17001793171C18826
:10FE50007171C088000AB07117E05846FFF713FAB5
:10FE600000281CBFD0F800C0BCF1000F0BD00F98C9
:10FE70000290CDF8049000943B4632462946404615
:10FE8000E047824601E04FF00E0A5046BDE8FE8F83
:10FE90002DE9FE438046894617461E4602A948467C
:10FEA00000F0CDF905002CD0BDF80800FFF7EBF904
:10FEB00000281CBFD0F804C0BCF1000F1FD00A9866
:10FEC0000B9C0090019433463A4629464046E04751
:10FED000060017D1FE2C15D02878022812D100F088
:10FEE00014F842F6021188420CD13878797800EB88
:10FEF000012292B24946404600F04AF802E00E263E
:10FF000000E001263046BDE8FE836868017840784D
:10FF100001EB002080B27047E0B58DF80820022385
:10FF2000120A8DF80920FE2201920022009202AAF4
:10FF3000FFF7AEFF0EBD7CB50129044605D00229AE
:10FF400022D1012100F0FCFDF0B92046FFF763FE4D
:10FF500008B1FFF773FE01A800904FF6FF7502236A
:10FF60001A4A2946012000F03CF90BE0F0680168CC
:10FF7000204601F033FFBDF8042000232946304617
:10FF800000F081F90600F1D173BD0000904500201A
:10FF9000F8B50F4F04463878FF280D46164611D0A5
:10FFA0000A2000F0D3FE68B1B12101704480002125
:10FFB00041700171C580068101463878BDE8F44082
:10FFC00000F0E5BEF1BD0000ACC90100B4C90100FC
:10FFD000A2460020E0B50821ADF8001001900421F0
:10FFE00000F00FF8002814BF002002980EBD00B5E5
:10FFF00083B00821ADF800100190052100F001F850
:020000040001F9
:1000000007BDADF8021068460149096808470000BD
:100010003048002070B5DFF858592878062460432E
:10002000FFF7D8FFDFF84C19086008B9132070BD3E
:100030000020FF2206E03380401C0023F270B270E3
:100040003371C0B22B78984209DA0B6804FB003692
:1000500000280CBF4FF6FE734FF6FF73EBE70FF26D
:10006000314001F069F90FF6390001F089FB0FF614
:10007000790000F0E1FC002070BD70B504462088D6
:1000800068B160680378426800F03AF948B960687E
:1000900003784268DFF8E00800F034F908B902207C
:1000A00070BDA078C01F0A2801D3182070BDDFF8EA
:1000B000CC58288820B12188C0F58030884201DAE8
:1000C000012070BD0C20FFF785FF060001D1132031
:1000D00070BD002007E06268298802EB0012401C16
:1000E0005181491C298080B221888842F3D30020A5
:1000F000306008222146301D00F0D9FD686810B933
:100100006E6004E0084601680029FBD1066000200B
:1001100070BD38B502460846DFF860184C68002309
:1001200001E02346246894B1A5686D899542F8D111
:100130002268002B0CBF4A601A6018B10822211DEA
:1001400000F0B5FD2046FFF752FF002032BD012030
:1001500032BDDFF82C180870704710B50446104601
:100160001422114203D000F0D6F8012204E04A061E
:1001700008D500F0D0F8002201462046BDE8104026
:1001800000F01FBDC80701D4022010BD002010BD23
:1001900070B504460D46A8061E4609D5104600F067
:1001A000BAF801462046BDE87040012200F009BDC2
:1001B000882005420FD0104600F0ADF8014605F04A
:1001C0000802204600F0FDFC48B1717A41B1317A55
:1001D000012904D070BDA80701D4032070BD002000
:1001E00070BD2DE9F0478146DFF8900744688A46E4
:1001F00090461E4600E02468F4B1002700E07F1C12
:10020000A088BFB28742F6D2A06800EB07156889C4
:10021000484528BF8245F2D33EB129786868334605
:10022000424601F072FD0028E9D0089810B1A1689B
:1002300049890180284600E00020BDE8F087F0B53C
:10024000DFF83827536800E01B68D3B19D686E89DA
:10025000B042F9DB9F88BA199042F5DA4FF0000CF2
:1002600001E004F1010C1FFA8CF4BC42ECD205EB66
:100270000412B2F80AE08645F3D101B10E801046AF
:10028000F0BD0020F0BD2DE9FC4104460027ADF88B
:1002900004704FF6FF786089404515461E4608D029
:1002A00001AA0092401C2378626880B2FFF799FF90
:1002B00007462378626800F023F830B92378626833
:1002C000DFF8B40600F01EF808B160890CE023786E
:1002D0006268DFF8B00600F015F858B11FB1BDF83C
:1002E0000400A84203D0284600F0C7F803E078894C
:1002F000404400E0608906B130803846BDE8F681B0
:10030000DFF88406022101F000BD80B500F08BFA11
:1003100000B1008802BD80B500F085FA08B1807890
:1003200002BD102002BD70B5012982B004461546F9
:1003300016D0032918D0052925D0072927D0092947
:1003400029D00B292BD00D292DD00F292FD01129E1
:1003500031D0132933D0172934D0192936D039E0B8
:10036000294601F010FA33E001F0F8F9ADF8000089
:1003700000A9204601F010FA06002CD12988204659
:1003800001F0B9F827E0294601F012FA20E02946E9
:1003900001F026FA1CE0294601F032FA18E029465D
:1003A00001F044FA14E0294601F04EFA10E0294623
:1003B00001F058FA0CE0294601F063FA08E001F078
:1003C00071FA05E0294601F073FA01E001F07DFAC7
:1003D000064600E00226304676BD2DE9FC410D467A
:1003E000044616461F4601A900F02AFA5FEA0008F3
:1003F0001DD156B100F037F8BDF80000FFF78BFFB4
:1004000000F036F85FEA000811D12946204601F0D5
:100410006DFA5FEA00080AD1019CFF2F07D0A31CE8
:100420001E2221460FF2954001F047F8E770404642
:10043000BDE8F6817CB50D460446164601A900F0DC
:10044000FFF917280ED04EB1002000F00CF8BDF8CF
:100450000000FFF760FF00F00BF818B929462046AE
:1004600001F039FA76BDADF8000000A92888E6E66B
:1004700001460122204600F0A4BB10B50446FFF758
:1004800044FF08B1611E0C18A0B210BD00000000AE
:100490002DE9F0470D468046A87800241E2888B034
:1004A000914614D1404600F0DFF904001EBFA07849
:1004B000FE28FF2822D0002000900022AB78E078B0
:1004C000414600F0CFFF204600F0E2F916E0122886
:1004D00004BF6878012813D0404600F0C5F9040035
:1004E0001CBF2279002A0BD0100607D4A9784046F9
:1004F00001F014F8207940F08000207100206BE0BA
:10050000DFF87C743878FF2817D0A978881E172860
:1005100013D20FF2784A48080AEBC000A0F108068F
:10052000306800281CBF7068002806D0287810B9F1
:100530006A78012A03D1122901D006204CE002A9D1
:100540000091AB88AA6869783668B047060042D146
:10055000AA7852080AEBC20202A952F8042C4046BB
:10056000904706001CD1AB78042B34D002A8009031
:1005700000223878414600F075FF06002BD1A9789B
:1005800002A800F0E5FF10B1002089F80000A8786B
:10059000122804BF697801291DD0E4B120711AE046
:1005A0006878C0B9A8788DF800008DF8046000A9BB
:1005B000A878042818BF0628BDF80800ADF8020086
:1005C000404601F0E0F828B100AB01221621404678
:1005D00000F087FF0026304608B0BDE8F087002015
:1005E00070472DE9FE430D46804628886988814280
:1005F00000D308B901206AE00021ADF8041002918F
:100600004FF6FF7900E0401C002100910A466988FE
:10061000002380B2FFF7E5FD070034D0BDF80400E9
:10062000002835D100AB4A460521404600F0BAFF0C
:10063000040001D111204AE002943878022806D142
:1006400001208DF80600BDF80000860824E0022095
:100650008DF806001221BDF8000090FBF1F67889B4
:1006600004F8010B102200F034F81034BDF8040037
:10067000401CADF80400B6B2BDF80400B04202D28E
:1006800078894845BFD1BDF8040080B90A201EE032
:100690009DF806000128E2D138780228F3D1788944
:1006A00004F8010B022200F014F8A41CDEE701A9F3
:1006B000404601F07DF848B101AB052216214046C5
:1006C00000F00FFF10B1029801F067F90020BDE8BB
:1006D000FE837889000A04F8010B2046796800F04F
:1006E000E6BA10B582B04C880888844200D308B9B5
:1006F000012016BD00F015F808B90A2016BD00202B
:1007000016BD10B582B04C880888844200D308B961
:10071000012016BD00F005F808B90A2016BD00201A
:1007200016BD002200924A1D0B79214659E510B5ED
:10073000044682B0084600A90088FFF780FD08B98A
:10074000012016BD017ABDF800202046FFF705FD07
:1007500016BD70B582B006460D46002401E0641C4B
:10076000A4B2A888844229DA286810F8142000EB83
:10077000440000A9407802EB002080B2FFF75FFD43
:1007800050B9286810F814100170286800EB440173
:1007900049784170012076BD017ABDF800203046CD
:1007A000FFF7DBFC0028DAD0296811F814200A7062
:1007B000296801EB440252784A7076BD002076BD6C
:1007C00010B50C4682B020886188814200D308B9F8
:1007D000012016BD23796C48621DFFF793FD08B90F
:1007E000102016BD00200090237961882088621DAA
:1007F000FFF7F7FC08B90A2016BD002016BD38B572
:1008000004460D4600A92888FFF719FD08B9012004
:1008100032BD017ABDF800202B462046FFF7B8FC18
:1008200032BD002070475549496800E0096829B188
:100830008A6852898242F9D1081D704700207047AA
:1008400010B50C4600F010F860B104B1206080785B
:10085000FE2801D1172010BDFF2801D1002010BDB6
:10086000162010BD022010BD10B5424A12680021AA
:1008700000E0491C3E4B1B78C9B2994206D20623C0
:100880004B439C5A8442F4D1981810BD002010BDEF
:1008900010B50446A01C00F018FEFF20E07010BD4B
:1008A00010B50C46FFF7E0FF30B101794A1C9442C5
:1008B00004BF01F08001017110BD000010B582B0CD
:1008C00004001EBFA078FF28FE280BD00020009057
:1008D0001E232188E078172200F0C4FDFE20A070BE
:1008E000FF20E07013BD000070B504464FF6FE70A7
:1008F000844282B036D04FF6FF7651B92046FFF7DA
:10090000B3FF78BB3046FFF7AFFF05002AD0048065
:1009100073BD012906D12046FFF7A6FF050021D0AF
:100920002E800BE002291DD10121204600F008F99C
:10093000C0B92046FFF798FF050013D0A878FF281C
:100940000ED0FE2807D0002000901E23E878142245
:10095000214600F087FD2846FFF79AFFFF20A87088
:100960000020287173BD0548008870470000000012
:10097000AE480020A0480020ACC90100A0450020DE
:10098000A4460020B0C90100A8C90100A51A0100B1
:10099000DF050100BF1A0100E3050100E11A0100B3
:1009A000E30601002B1B010003070100691B010086
:1009B0002F070100B71B01002F070100DF1B0100FB
:1009C000530701002B1B0100C1070100871B010019
:1009D000FF07010000000000000000000D1C0100E6
:1009E000FF070100531C01002308010038B5904C9B
:1009F00000220021204601F070FA20782C2568435F
:100A0000FFF7E8FA6060B0B1002109E005FB0102E0
:100A10004FF6FF735380491C002313719362C9B2D0
:100A200022789142F2DB0020002104EB8002401C7E
:100A30000C289160F9DB31BD00217D4A02EB810277
:100A4000936813B9906000207047491CC9B20C2903
:100A5000F3DB132070472DE9F04106460C4617469C
:100A60009846204600F03EF808B111201EE04FF6EF
:100A7000FF7000F037F8050017D085F805800622D2
:100A80000699A81D00F013F96C802F712E700020BC
:100A9000A8620021079828730898E881099828829D
:100AA000204600F0B4F8002000E01520BDE8F081F9
:100AB00010B500F017F8040012D06088012100F092
:100AC000A6F8A06A08B1FFF792FA2C22002120466E
:100AD00000F01FF94FF6FF7060800020207110BDFC
:100AE000022010BD10B50022514B00E0521C1978B5
:100AF000D2B28A4208D259682C2404FB02114C88D5
:100B00008442F3D1084610BD002010BDF0B5484B1B
:100B10005C6800224FF6FF7701E0521CD2B21978D0
:100B20008A420BDA2C2101FB02F529194E88BE42BC
:100B3000F3D02D5D8542F0D10846F0BD0020F0BD18
:100B400010B50C464FF6FE71884206D0FFF7CAFF7B
:100B500000281CBF0079204201D0012010BD0020D8
:100B600010BD80B5FFF7BEFF00B1007B02BD10B520
:100B7000002000212E4A2C2406E0536804FB013398
:100B80001B7903B1401C491C1378C9B29942F4D3B4
:100B9000C0B210BD26480078704710B50C46FFF76C
:100BA000A1FF00281CBF018AA14202D004820020BC
:100BB00010BD012010BD80B5FFF794FF00B1008A81
:100BC00002BD70B505460C461646FFF78BFF28B9E7
:100BD0004FF6FE70854218D0142070BD0179806AEE
:100BE00028B9CA0609D5C90609D40F2070BD01F07D
:100BF0001202102AF7D1002EF5D0052070BD20B1C9
:100C0000807EA04201D20C2070BD002070BD70B566
:100C100004460D460026064800EB86008268100058
:100C200002D0294620469047761C0C2EF3DB70BD7F
:100C30006C47002000B583B00821ADF8001001908A
:100C40000B21ADF802106846DFF8C816096888471E
:100C50000EBD1FB5ADF806100824ADF80040ADF884
:100C600004000624DFF8AC168DF808200393ADF8D5
:100C7000024068460968884704B010BD80B500F09E
:100C8000C6F90C2000F001F802BDDFF888160968EB
:100C9000ADF802006846084700B583B000F0B7F928
:100CA0001220FFF7F2FF01980EBD01F045BA03E0F4
:100CB00011F8013B00F8013B13465A1E002BF7D1F7
:100CC00070471144491E03E011F8013900F8013B57
:100CD00013465A1E002BF7D1704770B504460D46D7
:100CE000A8B2FFF777F9060003D02A462146FFF79E
:100CF000DEFF304670BD10B513465A1E3BB110F8EA
:100D0000013B11F8014BA342F6D0002010BD012099
:100D100010BD10B5044610460A460146204601F0B3
:100D200027FA204610BD01F05BBADFF8EC25DFF8AA
:100D3000EC35526A11541B7805E0DFF8E035DFF836
:100D4000D8251B78526AC0181154704710B504009A
:100D500001D1002010BD04F10C0080B2FFF73AF978
:100D600028B1002101600481FF2181720C3010BD87
:100D700080B508B9052002BD10F8021CFF2901D07A
:100D8000042002BD0C38FFF732F9002002BD38B54F
:100D90000C46010622D5DFF880150A78FF2A08BF25
:100DA0004D7805D0DFF874351B78496A9A188D5C48
:100DB000FF2D02D1FFF762FF0EE000F0A0F901461F
:100DC000FF2004F8020C234600222846FFF741FFCB
:100DD00048B12046FFF7CCFF012032BD2146BDE8D7
:100DE0003840002200E032BD70B50D0004461646C2
:100DF00018D0200648BFFFF741FFDFF8201509781B
:100E00008C4204D32846FFF7B3FF032070BDA5F141
:100E10000C000168002904BF817AFF2904D028460C
:100E2000FFF7A6FF052070BD8472012EDFF8E804ED
:100E3000294603D1001D00F055F802E0001D00F026
:100E400039F800F033F8002070BD2DE9F041044678
:100E5000DFF8CC04DFF8C07400688047804678680B
:100E60000026002503E005B9064650F80C0C50B1E9
:100E700010F8021CA142F6D1002D08BF0546F4D09F
:100E800000F014F805E04FF40041204600F0A4F80B
:100E900025B132462946381D00F031F8DFF88414B8
:100EA0000968404688472846BDE8F0814FF4004174
:100EB000204642E038B500F00FF8002145F80C1C40
:100EC000216811B9256006E0114651F80C2C002A62
:100ED000FAD141F80C5C2DE10446DFF844040068C7
:100EE0000D46004738B5FFF7F7FF216845F80C1CA1
:100EF0002560DFF830140968BDE83440084770B554
:100F0000044600F014F8A5F10C0123680A689D421C
:100F10000CBF226046F80C2C00220A60FF228A7265
:100F2000BDE8704008E1DFF8FC1309680847DFF806
:100F3000F00300680D46164600472DE9F0410446CF
:100F4000DFF8D803DFF8D05390F8008020060E4673
:100F50002CD50420FFF7FAFE070008BF042039D083
:100F60004FF6FF7038807E80A7F10C062878FF28A6
:100F70000FBF6D78696A40440D5CFF2D05D138467E
:100F8000FFF7F6FEFFF77AFE0EE0204600F0B7F816
:100F9000FF21B1723B46014600222846FFF759FE69
:100FA000C0B13846FFF7E4FE012013E0444510D2FB
:100FB00000F02AF8DFF87013096831F81420324382
:100FC00021F81420FFF7AFFFE868FFF733FE002099
:100FD00000E00320BDE8F08138B50C46DFF83C1393
:100FE0000978884205460DD200F00EF8DFF8381374
:100FF000096831F81520A24321F81520FFF793FF67
:10100000002032BD032032BDC548006800470820DB
:10101000ADF80000704730B5BF4C0020606083B071
:1010200001F0E8F801F0FDF9BC4805786800FEF72A
:10103000D1FF60626A00FF21FFF76BFE0222FF21F1
:10104000A01CFFF766FE01F03FFAFFF725FE2061C6
:10105000FFF7DDFF1420AF4D2968ADF802006846A8
:10106000884701986061FFF7D2FF1520ADF80200B4
:101070006846296888470198801EA06100203EBD0F
:1010800030B587B00820ADF808001B20ADF80A0085
:1010900001200390A04D0FF281009E4C2168059025
:1010A000286A0690E869049002A888470499E961D3
:1010B00008B1FFF7E3FD00F053F8FFF7A8FF0A209F
:1010C000ADF802004FF0FF30019068462168884774
:1010D000F1E780B50021904A0A449378FF2B01D1B3
:1010E000907001E0834203D141F08000C0B202BDA4
:1010F000491C0229EFD3FFF7C1FDFF2002BD10B547
:1011000080F08004022CA8BFFFF7B8FD824820447D
:10111000807810BD0000000038B50446FFF774FF6A
:1011200005467D48016A8C4204BFC068FFF782FD16
:101130004FEA0500BDE834407A490968084710B510
:101140000446608848B9E088FFF7C3FF2072FF2893
:101150000CBF6FF00300002010BD6FF0010010BD48
:101160002DE9F0478AB001F037F9FFF795FD6A4E97
:101170007769D6F810A00025B7F57A7FA0EB0A04AE
:1011800014D0A7FB04014FF47A72002301F00CFA8B
:101190004FF47A78A8FB0023044608FB013310467D
:1011A00019463A46002301F0FFF9504430612046C9
:1011B00001F072FAB068010003D0804701E0FFF748
:1011C0005DFD0820ADF808000720524C2168ADF8FD
:1011D0000A0002A888475149BDF80E20049F0978EB
:1011E000F8B9002400E0641C8C42E8D2706A005D0B
:1011F0009042F8D1E4B2FF2CE1D0A7F1080898F8AA
:101200000000FFF766FF98F80210012908BF387048
:1012100002D0022908BFB87039462046FFF7B7FD53
:10122000CFE7414F3868EDB230F8150018B96D1CA2
:10123000E8B28842F5D3E8B28842DFF8E880DFF808
:10124000E0901DD2D9F8000080473968EDB231F83E
:1012500015A0002200F048F8344A3570514652F883
:101260002520284690478246FF203070D9F800009C
:101270008047396831F815204AEA020200F034F854
:1012800001F0AAF8054615F1010F2AD005B9284D3D
:10129000B069A84238BF0546D9F800008047074624
:1012A000FFF7B5FE1C20ADF80200F069216801903F
:1012B000684688470821306AADF81410401C132195
:1012C0003062ADF81610099006951A49F069089138
:1012D000079005A8216888470798F061384600F014
:1012E00005F80AB0BDE8F08721F81520D8F80010FD
:1012F000084710B548B1002300E05B1CDCB2944203
:1013000005D2DBB2C45C8C42F7D0002010BD0120B6
:1013100010BD0000304800202844002074C901009E
:101320003448002038480020884800204CC901007B
:101330008EC2F52819110100814908607047814962
:1013400008707047032290FBF2F080B200F0D8B929
:101350000178B02904BF417800290CD10179122904
:1013600003D1417C012906D101E01B2903D140882A
:10137000012100F0E2B9704780B5734A5070042132
:1013800072480078401C1070507800F05DF9BDE89C
:101390000140FEF73FBE38B50C46200411D56A481F
:1013A0004078FFF752FD050008D02878A02804BF38
:1013B000284600F008F82846FFF7DAFC84F40040DD
:1013C00032BD002032BD30B587B0044601208DF813
:1013D000000001A9204600F02FFB05002AD19DF84E
:1013E00006105748C9070AD54368180005D0608819
:1013F00000AA01A9984705461CE006251AE00368E3
:10140000180006D0608800AA01A99847050001D1FC
:1014100010E006259DF8050060B99DF806008DF8DE
:1014200010008DF814500020ADF8120004A9608857
:1014300000F0A9F99DF8000000281EBFA068002850
:1014400000F0ABFA45B99DF80600122806BF9DF8DA
:10145000051001291B2803D06088012100F06DF9D7
:1014600007B030BD2DE9F0410446FF2C0D4616466D
:1014700098461FD02020FFF769FC070018D0B02045
:1014800038707E707D8087F80480069929B1182213
:1014900007F10800FFF70BFC04E0182207F1080031
:1014A000FFF737FC39462046FFF771FC002002E0C9
:1014B000132000E00220BDE8F08110B54FF47A74EB
:1014C0006243BDE8104001F05EB910B504001EBFD4
:1014D0002078FF28FE2803D001F05DF9FF2020705E
:1014E00010BD80B5009313460A46014615480078A2
:1014F000FFF7B8FF02BD30B583B004460D4600F0DB
:1015000040FC50B901A80090ADF804507F230D486D
:10151000007800222146FFF7A5FF37BD00B583B054
:101520007E238DF804108DF8052001A9009100227A
:10153000014604480078FFF795FF07BD0000000052
:1015400068480020A3460020AE4800206C470020D9
:10155000052923D006291BD0072918BF09291DD02A
:101560000B2918BF0D2919D00E2913D00F291CBF24
:101570001129122912D0162918BF17290CD01B299E
:1015800018BF1D290AD0522918BFD22906D007E05A
:10159000C06870470068704780687047406870474F
:1015A0000020704770B5052914461D4616D006293F
:1015B00012D0092918BF112910D0122912D01629CA
:1015C00018BF17290CD01B2918BF1D290AD0522972
:1015D00018BFD22906D007E0072606E0022604E05D
:1015E000052602E0032600E001264FF6FF72944232
:1015F00003D100F0DBFB841B02E0D22908BF0C34CE
:10160000301980B201F01CFC38B105B12C80714258
:10161000BDE8704009B200F0E5B970BD80B5FFF7D4
:1016200097FF00281CBFBDE8024000F0B6B901BD1D
:10163000DFF800F0F5950010DFF800F031960010AB
:10164000DFF800F05D9600100A4610B5052A18BFB5
:10165000042A03D0062A18BF072A08D1414B0C24BC
:1016600004FB023222F8301D9070002010BD0220D1
:1016700010BD38B50D4604462888052818BF042833
:1016800003D0062818BF072801D1686808B90220CE
:1016900032BD01212046FFF753FA08B9142032BDAC
:1016A0004FF6FE70844207D02046FFF784FA29895E
:1016B000884201D21B2032BD2B48007800282946E1
:1016C00020461CBFBDE8344001F0A7B9BDE8344056
:1016D00001F059B980B5254B009313460A46012104
:1016E0000BE0E0B5019200230422009202930A4627
:1016F0001F4B122101F0DCF80EBD01F00DF902BD07
:1017000038B504461B480129017011D11A480088D8
:10171000051D0120FFF78CFF01B0ADB2284694FBF8
:10172000F5F2BDE83040002392B20021FFF784BFFC
:10173000BDE832400020FFF77BBF03B50D480078BD
:10174000012881B003D102AA01A9FFF779FF07BDE3
:10175000094A001F1080044801707047064800883D
:1017600070470000A447002072480020172B01009A
:10177000952B0100B3480020A046002070470000D0
:101780006E490860704780B5002200920B46012226
:101790006B4900F0BAF802BD80B50A88172A05DB4C
:1017A000002200920B4603226649F2E7022002BDA6
:1017B00038B50D460446A878012818BF02280DD177
:1017C000288800281CBF6868002807D0022100F084
:1017D00009F900902B4605225B4931E0022032BD19
:1017E00038B500F01EF81CBF6868002806D000F06D
:1017F00036F800902B460722544921E0022032BDE2
:1018000038B500F00EF81CBF6868002807D0022128
:1018100000F0E8F800902B4609224D4910E0022024
:1018200032BD0D46044628880028704738B500F0C0
:1018300024F808B100F013F800902B460B2245491C
:10184000204600F062F832BD38B500F016F808B155
:1018500000F005F800902B460D223F49F0E70121EA
:1018600000F0C0B838B500F008F808B1FFF7F7FF8E
:1018700000902B460F223949E2E70D46044668687E
:10188000704738B5FFF7CDFF1CBF6868002807D048
:10189000022100F0A7F800902B4611223049CFE733
:1018A000022032BD80B5002100910023132270E791
:1018B00038B50D460446A86810B1052100F092F82D
:1018C00000902B4617222749BAE780B500210091E6
:1018D000002319225DE738B5FFF7CFFF10B10321D0
:1018E00000F080F800902B461B2209E038B5FFF786
:1018F000C4FF10B1032100F075F800902B461D22A3
:101900001949204600F0BFF932BDF8B504460698E3
:10191000009015461E46204600F0B5F907000AD192
:1019200006480268100006D0012D04BF3078451C1F
:10193000E9B2204690473846F2BD00008C480020AE
:10194000931A0100AF1A0100C91A0100231B0100FC
:10195000671B0100831B0100DB1B0100F71B01005B
:10196000FB1B0100351C0100651C010070B500F077
:1019700035F8054604F1080080B2FEF72BFB06009F
:1019800005D02A48B48001683160066008362849CD
:10199000096828468847304670BD38B500F01EF803
:1019A000224A05461068002101E00146006878B12E
:1019B00000F108039C4221BF8388C3180833A34267
:1019C000F3D3036800290CBF13600B60FEF70FFB15
:1019D0002846BDE8344016490968084704461548BA
:1019E0000068004738B504460D4600F00FF80100C6
:1019F0000AD06842204401F10803984221BF8B8835
:101A0000C9180831814200D2204632BD0749096811
:101A100041B101F10802904221BF8A888A18083238
:101A20008242F4D30846704700000000844800203A
:101A30003848002034480020F8B505460C46AF89E8
:101A40002FB3AA68167830060FD50D2F1FDB0C3F79
:101A5000BFB2B81800903B466888012101F0CAFB6C
:101A6000002814BF0220012000E000202070B009EF
:101A700000F00100607006F03F00A070781EA080AA
:101A800080B208B1A868401CA0600020F2BD01200F
:101A9000F2BD0A7802704A8842704A88120A82703F
:101AA000097985E0022B00D163E00420704700BF74
:101AB0000A8802700988090A417002207047042BC5
:101AC00000D17DE0042070478A7802708878098808
:101AD00001280CBF042012204843401C80B27047EC
:101AE00070B51E46062E144619DB049D20786178D9
:101AF00000EB012028800222A078E17800EB012091
:101B00006880211D02202871681DFFF7D0F8B01FE2
:101B1000288180B200B1A01DE860002070BD0420C3
:101B200070BD08888004000C704710B5029C062B1D
:101B3000104612D1022121714278017801EB022175
:101B40002180C278817801EB02216180011D227918
:101B5000601DFFF7ACF8002010BD142B08BF10214A
:101B6000E9D0042010BD49E0022B00D101E004209F
:101B700070471078517800EB012000990880002010
:101B800070470888704710B5022B0FDB029C20724B
:101B900061721078517800EB01202080981E6080DF
:101BA00080B200B1901C6060002010BD042010BD08
:101BB000C17004207047042B00D101E0042070475D
:101BC00000981178537801EB032101809178D27845
:101BD00001EB022141800020704708887047D80738
:101BE00007D45908022904DB009881800260002094
:101BF0007047042070470888704700BF4A880988EA
:101C00000270514389B2481C80B2704710B5042B52
:101C10000EDB00F031F8D478917801EB042141809B
:101C2000191F818089B201B1111D8160002010BD92
:101C3000042010BD00BF0A8802700A88120A427090
:101C40004A8882704A88120AC2708888001D80B251
:101C50007047012B04D1009910780870002070475C
:101C60000420704700BF0A8802700A88120A427076
:101C70004888801C80B2704702981178547801EB34
:101C80000421018070472DE9F04784B080460C9D07
:101C90000C4691469A4655B9172001F0D1F8012615
:101CA000050005D11324204604B0BDE8F0870026C6
:101CB0002846012700F8019B14B15146A047471C54
:101CC0005FEA09600DD510214046FEF739FFD0B913
:101CD000BFB27A193946284601F03FFA04000CD108
:101CE0000C370420ADF800000195ADF8087000A98C
:101CF0004046FFF7BEFC0400D5D0002ED3D02846C6
:101D0000FFF74BFECFE71924F7E730B5022918BFDC
:101D1000102985B00446154603D1022B18BF102B9D
:101D200001D0002017E0994204D10A462946FEF767
:101D3000E2FF10E0102900A906D1284600F00DF8B6
:101D4000102200A9204604E000F007F8102200A9A4
:101D50002846FEF7D0FF05B030BD38B504000D466B
:101D600018BF002D0BD010220FF260012846FEF79D
:101D70009EFF2078287360786873012032BD0020B0
:101D800032BD38B504464FF6FE7084420D460BD086
:101D9000172D09DBFFF7E2FCA84205D329462046B0
:101DA000BDE83440FEF7F9BE012032BD80B54FF6E4
:101DB000FE71884204D0FEF7FEFE28B9172002BD4E
:101DC000BDE80140FFF7CABC02BD0000FB349B5FC9
:101DD00080000080001000000000000038B54FF6C1
:101DE000FF74A0420DD10020164A137898420EDAF3
:101DF00021F8204001EB80050023401CAB70C0B2ED
:101E0000F3E700F00BF810B104800021817031BDC0
:101E100080B500F003F800B1807802BD10B5002253
:101E200000E0521C074C2478D3B2A34207D2D2B2AE
:101E300031F822308342F4D101EB820010BD002042
:101E400010BD00006C470020DFF800F0DD8A0010B4
:101E5000DFF800F0A18B0010DFF800F0D570001063
:101E6000DFF800F09D58001030B540F67B44851F28
:101E7000A5423CBF8D1FA54212D2814210D3B2F5BC
:101E8000FA7F0DDAA3F10A0040F67744A04207D2A8
:101E9000501C49004843B0EBC30F8041C00F30BD18
:101EA000002030BD80B501F04BFD8DF8000002F040
:101EB0003DFA74490020087000AA73490880012186
:101EC00040F603405DE080B50FF22822412141F247
:101ED0000200FFF7B9FF002002BD7CB5002808BF53
:101EE000002938D1BABB01A802F0A0F99DF804007E
:101EF00000EBC000451DEDB22846FEF76BF806006A
:101F00004FF6204418D0202030700420707000203C
:101F1000B0709DF8040000280CBF0022721D311D16
:101F2000F01C01F099FD32462946204602F00FFBD5
:101F30003046FEF75CF80CE020208DF8000004210C
:101F400000A800AA4170072181702046032102F0F9
:101F5000FEFA002076BD01F07FFD76BD80B5002041
:101F60008DF8000000AA494800788DF8010004218E
:101F700000208DF80200464800788DF8030042F2F8
:101F80000200FFF761FF002002BD38B5044642F2AF
:101F9000160529460020FFF75BFF204601F0F2FD01
:101FA0008DF8000020B100AA01212846FFF74CFF60
:101FB000002032BD80B5012301F00FFF00F01BF8B7
:101FC00042F21E00DDE780B5012101F07FFF00F045
:101FD00012F842F21D00D4E780B530B10146082264
:101FE0002C48FEF764FE002000E0122000F003F809
:101FF00040F66340C5E78DF8000000AA0121704754
:1020000080B542F213010C20FFF722FF002002BD31
:1020100010B582B01D218DF8001000AC04218DF8A0
:10202000011010B9FFF718FF00E01120A07000AAFE
:1020300003214FF61D4002F08AFA002016BD80B53C
:102040001C208DF8000000AA04208DF80100032157
:102050000C208DF802004FF61C4002F078FA0020A8
:1020600002BD02F0EDB880B530B10B4902780A70BC
:1020700040784870002000E01220FFF7BCFF42F2D9
:1020800001007EE7244F0020264F0020104800204A
:102090008B4C0020284800202048002000B585B047
:1020A00000AA0DF1020101A8FFF7DAFE8DF8080081
:1020B000102107208DF8090002AA02A881700221D0
:1020C0008DF80B109DF804108DF80C10BDF802105F
:1020D0008DF80D10090A8DF80E10BDF80010C171B1
:1020E000090A017241F201000921FFF7ADFE00204B
:1020F00005B000BD000000800000C000000000E44A
:102100000000002822000000000000040000F7C3C7
:10211000B37E00000000000000000000000000008E
:1021200000000000000000000000000000000000AF
:10213000000000000000000000F10103810704D04E
:1021400010F8011B89B18107FAD10268B2F101319F
:10215000914311F0803F04BF50F8042FF6E710F8C8
:10216000011B11B110F8011BFBE7C01A70470000FA
:1021700062F30F2262F31F42401810F0030308D0ED
:10218000C91A1FD3DB0748BF00F8012D28BF20F86C
:10219000022D130030B414461546103928BF20E92B
:1021A0003C00FAD8490728BF20E90C0048BF40F896
:1021B000042D890028BF20F8022D48BF00F8012D0A
:1021C00030BC7047C91818BF00F8012DCB0728BFD5
:1021D00000F8012D70470000DFF800F001580010F2
:1021E00080B502216846FFF7F7FFBDF8000002BD89
:1021F000704770477F4900204860704770B50446BB
:102200000D46164600F018F808B1466070BD102063
:10221000FDF7E0FE78B1847205814660002101601F
:10222000C16074490A6812B9086070BD0A46116835
:102230000029FBD1106070BD6E4A12682AB1138963
:102240008B4204BF937A8342F7D11046704708B19E
:10225000002101817047F8B500F022F800F01BF86A
:1022600000F04AF8044638468847002C14BF002086
:102270000820F2BDF8B500F013F800F00CF80400E7
:102280005D4918BFE660096838468847002C14BFCE
:1022900000200820F2BD0746324629462046ADE719
:1022A0000446564800680D461646004770B500F0D3
:1022B00026F8064629462046FFF7BEFF040018BF51
:1022C000FFF7C5FF00F018F830468847002C14BF10
:1022D0000020062070BDF8B500F011F80746294629
:1022E0002046FFF7A9FF002600B1466800F004F879
:1022F000384688473046F2BD3F4909687047044672
:102300003E4800680D4600472DE9F047DFF8EC90A5
:10231000384D82B00746D9F8000000978047014643
:102320006868381868600846334F396888472E68EF
:10233000002E4FD04FF00008D9F8000080478246A9
:10234000BDF802000024002804BF9DF80100002809
:1023500007D130799DF80020904202D3801A307165
:1023600006E07068009981423ABF401A706074605C
:10237000B08858B9F08858B9F06868B13189080058
:102380000AD0B07AFEF7D9FDF0687060B08808B95D
:10239000F08808B1308940B93068B8F1000F0CBF3F
:1023A0002860C8F80000344600E0B0463668396856
:1023B0005046884764B1A088002804BFE088002800
:1023C00003D12189A07AFEF7B8FD2046FDF70FFE64
:1023D000002EB1D1BDE8F3870648016841B1084835
:1023E0004A680968824298BF10460029F8D17047B0
:1023F0000020704760480020384800203448002002
:102400008EC2F52800B583B00821ADF800108DF814
:1024100004001721ADF8021068461A490968884778
:102420000EBD194800218180012101707047F8B567
:102430000C46164909788842054601D30320F2BDAF
:10244000114E3078E8B112480068804707460120F5
:1024500000FA05F5B08844B920EA0501B18058B109
:1024600051B90020FFF7CEFF06E010B90120FFF7B9
:10247000C9FFB0882843B0803846064909688847B4
:102480000020F2BD304800205048002074C90100EF
:10249000344800203848002030B585B01446082262
:1024A0000291ADF80020002238490968ADF8040017
:1024B000ADF802201D4668468847BDF80C10218003
:1024C0000499296005B030BD1CB51420FDF782FDCC
:1024D0002F49086014220021FEF71BFC002001F0A8
:1024E00053F8012002F072F8022000F005F90320F1
:1024F00002F0A2F8042002F0E4F9052002F01EFB2D
:102500000620FEF739FF0720FCF796FD082003F0B0
:102510008EF8092003F062FA01AB6A460021102010
:10252000FFF7BAFFBDF800100920FEF7FEFB0024FC
:10253000BDF800102046FEF700FC641C092CF7DBF8
:1025400013BD10B582B003F0C9FE124B124A1349F5
:102550005020FFF7A1FF48B10820ADF800000C2083
:102560000A490968ADF80200684688470C480068C7
:102570008047044604F063F8FEF74DFD09490968F9
:1025800020468847FEF77CFD002016BD304800201D
:1025900088480020344400207E4800203F1101007C
:1025A00034480020384800201B4213D1094236D15C
:1025B0002AB18446B0FBF2F002FB10C2704704F06F
:1025C000FBB8FCD30022002370470B00020000215F
:1025D00000207047904271EB030CF6D370B5B1FA4E
:1025E00081F4B3FA83F52C1BA340C4F1200532FA21
:1025F00005F63343A2405FF00046E64002E05B0888
:102600005FEA3202841A71EB030524BF2046294693
:102610007641F4D302000B003000002170BD012A86
:10262000CFD970B5140C20D0B1FA81F4B2FA82F58A
:10263000C4F120046419B4F12006D6D3B2405FF08F
:102640000044F440002502E052085FEA3303C61A52
:1026500071EB020E24BF3046714664416D41F3D3E5
:1026600002000B002000290070BD0C46B1FBF2F106
:1026700002FB11452D0445EA1045B5FBF2F402FBBF
:10268000145580B240EA0545B5FBF2F002FB10524A
:1026900040EA044070BD000070B5134D0446286840
:1026A0006FF0020108402860104800688047104918
:1026B0000A68A218B2F57A7F0AD34FF47A734E688B
:1026C000B2FBF3F39E194E604FF47A7606FB1322A9
:1026D0000A600849096888472046FFF715FE286800
:1026E00040F00200286070BD10E000E03448002097
:1026F00048480020384800205F4B1988FF2905D141
:10270000188078220021181DFEF703BB70472DE9C1
:10271000F04104460D46280448BF85F4004030D4FB
:1027200028002DD055480068804780462F4600205D
:1027300025FA00F1C9071AD54F490A88121BC2EBC6
:102740000212821801EBC2010F1D012101FA00F6ED
:10275000396808001CBF78688847B1B22046FFF787
:10276000BAFD08B93860786086EA050702E0401CC7
:102770000F28DDDB4249096840468847B8B200E0CF
:102780000020BDE8F08110B582B00024FFE700947E
:1027900000F02AF816BDF8B504463848384E0068EF
:1027A00080470F2C05461ADA334800EBC4077968D6
:1027B000A9B10F2194FBF1F2C2EB021300880121B1
:1027C000E31A9940801889B2C0B2FFF76FFD00206C
:1027D0007860B8602846316888470020F2BD3168CB
:1027E000284688470220F2BD2DE9F44F8046234851
:1027F000234C006889461E46804783465FEA0800EE
:1028000004D1216858468847022031E00025DFF8CE
:1028100068A00AEBC507786818BB9DF82800009AE5
:1028200001280CBF174B184B0F2095FBF0F0C0EBA5
:10283000001E4FF0010CA5EB0E010CFA01F1BAF8E5
:1028400000C0604489B2C0B2984750B9C7F804804C
:10285000C7F8089006B135702168584688470020AF
:1028600006E06D1C0F2DD4DB2168584688470820F0
:10287000BDE8F28F000000005044002034480020E2
:10288000384800207522010057220100DFF800F0CF
:10289000E9940010DFF800F0A19400100A780270AB
:1028A0004A7842708A78C97802EB012141807047EA
:1028B0002DE9FC410D4616461F460A9A0999044621
:1028C00001AB00F0EFF95FEA000822D10199089806
:1028D00008703346DFF84C050178491CC9B200295D
:1028E00006BF012101220A460170294601980271A2
:1028F000009701980279204600F00EF85FEA000880
:1029000004D101981E2100F013FA02E0019800F0B2
:10291000F2F94046BDE8F6812DE9F041044684B065
:102920000E4617469846172000F08AFA050025D073
:102930000A9A100003D04146281D904700E000206D
:10294000010A2E70E9706F70A8700521001DADF8A6
:102950000800ADF80010019500A9DFF8CC0400785C
:102960000028204602D000F058F801E000F00BF8F3
:10297000040004D02846FFF710F800E01324204696
:1029800004B0BDE8F08110B50B88DFF8A0240C245A
:1029900004FB0322303A536833B94B68536009890A
:1029A00050811181002010BD162010BD80B505207A
:1029B00000F00FF858B9062000F00BF838B90420E1
:1029C00000F007F818B9072000F003F800B1012063
:1029D00002BDDFF858140C2202FB001110B5A1F162
:1029E000300484B06168A9B1DFF83C2412787AB170
:1029F000ADF80000019100A92089ADF808006089B8
:102A000000F00BF810B16068FEF7C7FF00206060AF
:102A1000012000E0002004B010BD70B50D46044652
:102A2000288920B1DFF808140988814201D21B20CF
:102A300070BD68680421FEF7D5FF0646288930700E
:102A40002889000A70702888B0702888000AF07001
:102A50002889051D4FF6FE70844213D10C20FEF725
:102A600075F901000CD0902008704C80022008718C
:102A7000CD808E60DFF8BC030078FEF788F917E0A0
:102A8000132070BD3346AAB200212046FFF7FEFE98
:102A9000010007D002280DD007280FD012280BD034
:102AA0001F280CD1DFF88003017809B1491E01709D
:102AB000002070BD142070BD022070BD042070BDC8
:102AC00038B50446002060600879022821D1CA8800
:102AD000042A1EDB886801784378C57801EB03215E
:102AE000837889B203EB05230D1D95429BB210D16B
:102AF000052B18BF042B03D0062B18BF072B08D1BA
:102B0000218123806FF00301FEF76CFF60600020DD
:102B100032BD012032BD0B88037002220B881B0AD4
:102B200043700B88012B06D14A88827004224988A1
:102B3000090AC1700CE0022B0AD14A8882704A88C7
:102B4000120AC2708A88027106228988090A4171B4
:102B500010467047022A1BDB0A784B7802EB0322EF
:102B600002800288012A05D18A78C97802EB012106
:102B700041800BE0022A09D18A78CB7802EB03224C
:102B800042800A79497902EB012181800020704757
:102B9000012070470A8802700A88120A42704A8827
:102BA00082704A88120AC2708A8802718A88120A60
:102BB0004271CA888271C988090AC17108207047A8
:102BC000082A18D10A784B7802EB0322028011F808
:102BD000022F4B7802EB0322428011F8022F4B7830
:102BE00002EB0322828011F8022F497802EB0121C7
:102BF000C1800020704701207047022A00D101E007
:102C0000012070470A78497802EB012101800020F9
:102C10007047F8B504460D4616461020FEF796F8A4
:102C2000070016D0A02038707D80002078702EB16B
:102C30000C223146381DFEF73AF804E00C22002140
:102C4000381DFEF766F839462046FEF7A0F800204A
:102C5000F2BD0120F2BD2DE9F04180460D46164639
:102C60001F462020FEF772F8040019D0A220207021
:102C700066706580069820716771079929B11822DE
:102C800004F10800FEF713F804E0182204F108002C
:102C9000FEF73FF821464046BDE8F041FEF777B821
:102CA000BDE8F08170B51E0004460D4621D001211B
:102CB000FDF746FFD8B160480078002100E0491CCC
:102CC000C9B2814211DA5D4B1B6803EB01125388D4
:102CD000002BF4D10020107001F14000508022B18F
:102CE000D48015723260002070BD152070BD142094
:102CF00070BD012070BD10B5044610220021FEF702
:102D000008F824E0002201E0521CD2B24A490978B6
:102D10008A420BDA4949096801EB02114B88002B02
:102D2000F2D00B798342EFD10846704700207047FC
:102D30004FF47A724A4300F1090301460FF215007D
:102D4000FFF721BD10B50446607AFFF724FDFF2090
:102D5000607210BD10B504001CBF6088002807D049
:102D60001721204600F005F82046BDE81040C2E7D4
:102D700010BD1CB50446207804280FD10020019016
:102D800000900A46E188207A1323FFF764FFE18868
:102D900002B0BDE81040122205202DE013BD07212E
:102DA00070B50446002531BB17E02448006800EBED
:102DB0000516307800281CBF707AFF280CD0F088E8
:102DC000A04209D13046FFF7BDFF14213046FFF77E
:102DD000D0FF3046FFF78FFF6D1C17480078EDB22B
:102DE0008542E2D30425FF222146284600F004F85C
:102DF0006D1C082DF7DB70BD10B50C4B0C2404FBCB
:102E00000030A0F13004608988420AD1606840B186
:102E1000FF2A1CBF0178914203D1FEF7BEFD0020BE
:102E2000606010BDB448002072480020A447002014
:102E3000A0460020704800207148002074480020FF
:102E400080B5001D80B2FFF725FD28B1BDE8044024
:102E50006FF00301FEF7C6BD02BD0000DFF800F011
:102E6000519B0010DFF800F0D557001038B5040072
:102E70000D4618BF002D01D1022032BD032100A84C
:102E800000F029F900A82A4600F027F8040004D130
:102E9000032200A9E81CFDF70AFF204632BD30B529
:102EA00004000D4618BF002D83B001D102203EBDA5
:102EB0000322E91C00A8FDF7FAFE00A801AA00F011
:102EC0000CF848B90322294601A8FDF714FF012890
:102ED00001D100203EBD01203EBD817801F03F01BF
:102EE00041F040018170204600A950E070B5234CAC
:102EF0000546206870B3A5B9027862B90822801C23
:102F0000FDF7D5FEFFF7AAFF18B921680120087068
:102F10001FE0012503E008220A30FDF7C8FE206803
:102F2000B8B11220FDF712FF06000DD0C12030709D
:102F3000757010222068811CB01CFDF7B8FE206857
:102F400040783146FDF723FF2068FDF750F8002058
:102F50002060012070BD80B5202003F041FC38B115
:102F6000024607480078BDE808400121FFF773B921
:102F700001BD034800780121FFF798B9A848002057
:102F8000B54800201022214600A8FDF79ABE70B572
:102F90008CB000F00FF8FFF7F5FF032229460DF182
:102FA0001D00FDF78EFE00F00DF8044603220DF122
:102FB0002D0185E004460D4616463022002100A86A
:102FC000FDF7A7BE00A8C2E0F0B595B005460C46D7
:102FD00016461F463022002108A8FDF79AFE10224F
:102FE000294608A8FDF76DFE1022002100A8FDF774
:102FF00090FE07223146FFF7C7FF072239460DF141
:103000000700FDF75EFE1C9901B101218DF80E103D
:103010001A9901B101218DF80F101022002104A886
:10302000FDF777FE1B99062205A8FDF74AFE1D99BC
:1030300006220DF11A00FDF744FE102221460CA8CD
:10304000FDF73FFE00A90CA800F01AF808A800F050
:103050007EF80446102210A90CA8FDF728FE04A94A
:103060000CA800F00DF808A800F071F805461E98AD
:10307000102210A9FDF725FE45EA040015B0F0BDA9
:1030800010B51022037811F8014B6340521E00F86E
:10309000013BF7D110BD70B50C468CB0154601460A
:1030A0001E461022FFF770FF0822214604A8FDF7F4
:1030B00008FE00F00BF8FFF785FF0446102208A970
:1030C0003046FDF7FEFD20460CB070BD08222946B3
:1030D00006A8FDF7F6BD70B504460D46002609E0CA
:1030E000FDF721FE010A3155761CF6B2AE423CBF17
:1030F0003055761CF6B2AE42F2D370BD006800F0D7
:103100000301C0F3800241EA8201C0F3C00241EA38
:10311000C201000941EA0010C0B27047026861F3C1
:10312000010202604A0703684CBF0422002223F018
:1031300004031A4302600B074CBF0823002322F04C
:10314000F8021A43090942EA01110160704700F1CF
:10315000200200F11001FFF785BE2DE9F0470700BE
:10316000144614BF002C022088B089463FD009F1D4
:103170000405A8B2FCF72EFF060036D003F084FC4D
:1031800080464A463946301DFDF79BFD86F8038090
:103190004FEA1827B7704FEA184986F801904FEAAE
:1031A000186A86F800A003F06CFC0146102203A800
:1031B000FDF787FD0820009001ABAAB2314603A8B5
:1031C00000F085F805000DD184F80080677084F860
:1031D000029084F803A0082201A9201DFDF771FDCB
:1031E00003F056FC00F070F800E01325284608B004
:1031F000BDE8F0872DE9F04F89B015001CBF129F84
:10320000002F80460E469A4615D0FDF76BFC040051
:1032100008BF142055D03878797800EB0120B978B0
:1032200000EB0140F97800EB0169606A484504D37E
:1032300010F1010F01D0022043E026B12079800770
:1032400058BF01203DD50822002101A8FDF761FDEE
:103250000AF1040B1FFA8BF0FCF7BCFE060008BF56
:1032600013202ED052462946301DFDF72AFD042298
:1032700039463046FDF725FD102204F1140105A85A
:10328000FDF71FFD0820009001AB1FFA8BF23146BD
:1032900005A800F01CF8050010D1082201A903A818
:1032A000FDF70FFD0822391D03A8FDF724FD0128B5
:1032B00011BF01254946404603F0A5FD00F004F882
:1032C000284609B0BDE8F08F3046FCF790BE2DE9E6
:1032D000FA4F834685B0154600F0CFF8814600F0DE
:1032E000CCF8B9F1000F804608BF132400F0B68077
:1032F000B8F1000F08BF132400F0AD8000F0BDF856
:1033000000F0BAF8BAF1000F064608BF132436D011
:103310000EB9132430E010220021FDF7FAFC5246CA
:1033200031465846FFF717FF040025D19AF80000F0
:103330000FF27C17000604D44946504600F0AAF864
:1033400008E03146504600F0A5F84A463946304676
:1033500000F096F899F80000000604D4414648466B
:1033600000F098F808E03146484600F093F84246ED
:103370003946304600F084F85046FCF738FE0EB16E
:10338000FFF7A2FF002C66D100F077F800F074F888
:10339000BAF1000F064608BF132459D00EB9132402
:1033A00053E005F10F00C11000EB117007033F144B
:1033B00005F00F0102D10127002202E04A1E9241CE
:1033C000D20F781E059B000503EB104012B222B10C
:1033D0003246494600F054F810E000AB8A42B8BFCC
:1033E000155C02DB0CBF80250025D554521C102A29
:1033F000F4DB3246414600A800F042F810220021DA
:103400005046FDF786FC00250BE00598290189B29E
:10341000091800AA504600F033F800F029F80446D5
:103420006D1C2DB2781E854201DA002CEDD064B9F6
:1034300000AA3146504600F023F800F019F804467F
:10344000109A06985146FDF732FC5046FCF7CFFD26
:103450000EB1FFF739FF4846FCF7C9FDB8F1000F80
:103460001CBF4046FCF7C3FD204607B0BDE8F08F07
:10347000524600A958466EE682461020FCF7AABDC7
:1034800030B500231C5C5D5C6C409C545B1C102BB5
:10349000F8DB30BD10B500220F231C5C42EA440269
:1034A0005A541A5CD2095B1EF7D510BD000000000B
:1034B0000000000000000000000000000000008785
:1034C000DFF800F001720010DFF800F021AD00100D
:1034D000DFF800F06DAD0010DFF800F0C1D800108B
:1034E000DFF800F0B5D80010DFF800F01DB50010CF
:1034F000DFF800F03DAC0010DFF800F0AD8E0010FA
:10350000DFF800F0F58B0010DFF800F00D7200100E
:10351000DFF800F089D10010DFF800F0C9B4001026
:10352000DFF800F019570010DFF800F06184001098
:10353000DFF800F08D670010DFF800F0BD800010AC
:10354000DFF800F02D8A0010DFF800F0C9870010C6
:10355000DFF800F069720010DFF800F071940010DD
:10356000DFF800F0A9AC0010DFF800F0E573001000
:10357000DFF800F035A30010DFF800F0E1AC001038
:10358000DFF800F0EDAB00102DE9F84FDFF8104B3D
:10359000DFF8105B207007210020A860DFF8080B1F
:1035A00001700D2141804FF404718180DFF8FC0A25
:1035B000DFF8FC1AE9608A7E0270FF2ACB7E437036
:1035C00008BFFF2B0E7F86704F7FC77091F81EC01B
:1035D00080F804C0C97F417116D1FF2E08BFFF2FAC
:1035E00012D1BCF1FF0F08BFFF290DD1DFF8C41ABB
:1035F0000A7802704A7842708A788270CA78C270FB
:103600000A79027149794171DFF8AC1A0278DFF862
:10361000AC8ADFF8AC7ADFF8ACEA0A7042784A701C
:1036200082788A70C278CA7002790A714079DFF8AC
:10363000D82B4871FF21DFF8900A0170417081702A
:10364000C17001714171101D017141718171C171B0
:1036500001724172002101708172A02181810321D8
:1036600081730721C1730021017428214182012146
:1036700001750021817502F15A0100224A70012270
:103680000A7042750020DFF8441A0880D8F82C3000
:10369000DFF83C1A58780870197839709A782A70CF
:1036A0009E683679761E8EF80060DB78DFF85C6BFA
:1036B0006B704FF4967333801B261B2392FBF3F33E
:1036C00006FB132202B10122D21850436880881CE5
:1036D0001821484380B2FCF77DFCDFF85C6BB060DA
:1036E000002855D03878002855D04FF490714843C1
:1036F00080B2FCF76FFCDFF8449BC9F8040008B9FE
:10370000B06843E0387838214843FCF763FC6860D0
:1037100020B900F08AF8D9F8040037E03878DFF8EB
:1037200064AB0001FCF756FCCAF8000028B900F0B1
:103730007CF800F07DF8686828E03878DFF848BB4E
:103740000001FCF747FCCBF8000048B900F06DF829
:1037500000F06EF86868FCF74AFCDAF8000015E043
:10376000387830214843FCF735FCDFF8201B08602F
:1037700088B900F05AF800F05BF86868FCF737FC8D
:10378000DAF80000FCF733FCDBF80000FCF72FFC54
:103790004FF4804144E0DFF8F80A006880470746AC
:1037A00004F00FF8FFF78CFEDFF8E80A0069006804
:1037B0008047FFF789FEFFF78BFEDFF8DC0A002168
:1037C00001600160C160C16003F048FE04F060F96F
:1037D000DFF8C81A40F2FF700860FFF77DFE06466A
:1037E000FFF77AFE864208BFFFF77AFED8F80C0092
:1037F000697800880843DFF8A81A08803846DFF89F
:10380000A41A096888470C21DFF89C0AFFF76CFEB0
:1038100020780021FEF70BFE00F092F84FF40051E3
:103820002078BDE8F44FFDF788BBB068FCF7DFBB3C
:10383000D9F80400FCF7DBBB30B50C46E00785B0D7
:1038400013D5FFF755FE38B100218160DFF85C0A1F
:103850000068010018BF8047DFF8440800780021A5
:10386000FEF7E5FD84F001005EE0A00707D500F05B
:103870005DF83C20FFF740FE84F0020054E0610751
:10388000DFF8200824D5DFF8B41940688A78496841
:103890004FF4907303FB0211382303FB02008D1DCC
:1038A00011F82C2F04924A8912090392AA8B0292D2
:1038B0000122C9884908019100F12C01009190F87A
:1038C000283029780020FFF717FE84F004002BE051
:1038D000210607D500F02AF83B20FFF70DFE84F003
:1038E000800021E0A10508D5DFF8C409016841F096
:1038F0000041016084F4007016E0610504D5FEF714
:1039000077FC84F480600FE0610405D58120FFF727
:10391000F7FD84F4804007E0A10443BF4FF0FF317E
:10392000816084F40050002005B030BD0020049078
:1039300003900290019000900146002301227047FD
:10394000F8B503F065FEDFF84809DFF8F0680068B5
:10395000DFF86C7780470446002003F0DBFF40F27D
:103960000140FFF7D1FDDFF82C090069C0688047EE
:10397000FFF7AAFDDFF84407DFF83819C06A80684E
:1039800040790870002504F024FCDFF82C09FFF7CB
:10399000BFFDFFF7C1FDFFF7C3FDDFF820090021E0
:1039A0000170017141718171C17101724172002216
:1039B000DFF8540800F10E010A70A0224A800722A5
:1039C0004A7103220A7100220A738A7200F8592F81
:1039D0000122CA720021427081700BE070684FF4BE
:1039E000907101FB05004179012908BF04F0E0F95D
:1039F0006D1CEDB238788542F0DBFFF795FD04F0E1
:103A00003BFD04F061F9DFF8B81800200870DFF81A
:103A1000B41808700120DFF8B01808700020DFF833
:103A2000AC1808700120DFF8A81808700020DFF833
:103A3000A4180870DFF8A0180870DFF8A018088034
:103A4000DFF89C18087003F01EFEDFF858180968AC
:103A5000204688470020F2BD2DE9F0411446DFF8EA
:103A6000605608B12A780270DFF8D08711B198F853
:103A700001000870002C3ED0002600271CE0C9B2CF
:103A8000DBB2085502F1280001791955591C427919
:103A900000F034F8827900F031F8C27900F02EF8A5
:103AA000027A00F02BF8427A00F028F80078C9B2C8
:103AB0004E1C08557F1CFFB2287887421BDA384617
:103AC000FFF736FD0028F5D1D8F804004FF49071C7
:103AD000F6B201FB0700DFF8CC15496837553822EC
:103AE0000068007802FB0712711C4B1C80280CBF79
:103AF00000200120C3E70020BDE8F081C9B20A55CB
:103B0000491C704738B50C00054601D1122032BD62
:103B1000FFF70EFDC0B900F019F901FB05000168BF
:103B20000978402901D00C2032BD00210A5D431ADA
:103B3000491C102983F8E220F8DB012180F8E41009
:103B4000052104F0C5F9002032BD10B50446FFF789
:103B5000EFFCB0B900F035F801680978402901D0D0
:103B60000C2010BD00F1F0010A78012A03D10622D1
:103B70000A77022102E006224A700D2104F0A8F91A
:103B8000002010BD10B50446FFF7D2FC60B900F06C
:103B900018F890F8F810022907D1817900F1F9029C
:103BA000002000F029FC002010BD01680978802960
:103BB00003D10821FFF7C0FCF5E74029F3D111201C
:103BC00010BDDFF8780640684FF4907101FB0400E7
:103BD000704710B5040001D1122010BDDFF85C065B
:103BE000407808B10C2010BD04F06EF82078DFF8A2
:103BF000F41600F01F0020704A7810404870002032
:103C000010BD38B50D00044606D0DFF8B004C06A18
:103C100080680079844201D3122032BD03F008FE8F
:103C2000032803D0204604F019FB02E0DFF88406E5
:103C3000047001202870002032BDDFF88014C96AAA
:103C400089680979884201D312207047DFF874141B
:103C500008700020704710B5140019D011B1012967
:103C600008D015E004F013FB10F1800F20700DD187
:103C7000302010BDDFF84404C06A80680168007914
:103C800000EB4000401810F8030C2070002010BD1D
:103C9000122010BD2DE9F0410C0082B0074690467D
:103CA0001D4628D0DFF8FC633078404528D33846DD
:103CB000FFF73EFC002847D100F048F801FB07075A
:103CC00004F0CEFD1B2298FBF2F21B2303FB1283B0
:103CD00003B10123718810181818814204DA0120F9
:103CE000FFF72EFC07202FE030781C2814DA002D77
:103CF00018BF012D01D0122026E0B8F11C0F04DB03
:103D00008A20FFF7FDFB30201EE02B46424621466D
:103D10003846FFF719FC13E042462146384604F0C6
:103D200041F988B92046FDF738FEB879ADF80000B2
:103D30000DF102020120ADF8020000A900F098FB8D
:103D4000384604F0EEF90020BDE8F681DFF8EC0417
:103D500040684FF49071704770B50646282E01DB1D
:103D6000122070BDDFF87845207808B1212070BDA1
:103D700003F04EFCDFF81C5528698068804770000E
:103D800000F6621189B20020FFF7E2FBDFF8580568
:103D900040F6070101804060002141808160017B85
:103DA00001F060010173417B01F0F00141F002017B
:103DB000417302218173DFF83415016100214161F3
:103DC000C17B01F0F00141F00101C1730C212170B0
:103DD000296989698847002070BD2DE9F0410446B2
:103DE0000D46282CB8BF262D16460FDA002E18BF18
:103DF000012E0DD0022E18BF032E09D0042E18BF9D
:103E0000052E05D0062E18BF072E01D012205BE02C
:103E1000DFF8CC8498F8000008B1212054E003F0CA
:103E2000F7FBDFF8CC74DFF8CC1441F60A003880D9
:103E30000022002078807F60B860387B00F060004E
:103E40003873787B00F0F00040F002007873600077
:103E50006630B8738020F873DFF89C0438617961AC
:103E60000280857040F6C4124260C670027A02F089
:103E7000FE02027200224272C260C27A02F0F002B6
:103E800042F00102C272002008800021DFF86C04B9
:103E90008180C180047080214570867001728948DC
:103EA000DFF8F043007804F0D9F9092088F8000021
:103EB00000222369DFF848045B68002198472169E4
:103EC0008969384688470020BDE8F08170B504460E
:103ED000282C01DB122070BDDFF80454287808B1CB
:103EE000212070BD03F094FBDFF80464DFF81414A4
:103EF000766041F609003080716100207080B0600A
:103F00000022307B00F060003073707B00F0F00026
:103F100040F00200707360006630B0738020F07370
:103F2000DFF8E403306102600F2202710122427166
:103F3000DFF8B82382605522027342738273002235
:103F40000261C27B02F0F00242F00102C273002063
:103F50000880488088800022802088710020886046
:103F60000021DFF898034170FF2181700470002167
:103F70008180C1808021C74C01720A2028700021F5
:103F80002369DFF87C035B689847216989693046BB
:103F90008847002070BD70B5D14C2078092818BF23
:103FA0000A2801D0212070BD40F20240FFF7ACFA90
:103FB0002078D249092809D1CE4800888880BD4898
:103FC000007804F04BF90021002015E00A2815D1F3
:103FD000CC4A538810889688CB801D1875198D801F
:103FE0009279802A18BF812A0FBF7F22C74B93F98D
:103FF0000030D21A0A720121FFF7AEFAFFF764FA15
:104000000020207003F03FFB002070BD38B5B44C99
:10401000207808B1212032BD03F0FAFAB44DB54A38
:10402000297B6D6001F0E00141F08501297341F6C3
:104030000A00697B288001F0F00141F002016973F8
:1040400000206621A97368808021E97340F6C410BE
:10405000A949A86029616A6148600123087A0B8038
:1040600000F0FE0008722523C87A8B7000F0F00083
:10407000002340F00100CB704B72CB60C8721380FC
:104080000D2020700022834CA14823695B681146F3
:1040900098472169896928468847002032BD000079
:1040A000844C0020104800208C4C00206C4C0020D8
:1040B000B63F0050E81200507C4C0020A4C801001C
:1040C000BC4C0020854C0020744C0020984C0020F3
:1040D0008B4C0020F8B5824C2178092918BF0A2999
:1040E00063D00B291CBF0C290D295ED0464DA97C3D
:1040F000002918BF012904D003291CBF0229042963
:1041000003D12A79002A18BF012A7BD1032918BFBD
:10411000022902D12B8AA02B74DB002843D001286E
:1041200070D1A87B012840D000291CBF0129042997
:104130000ED1FFF715FAFD21084236D175480078F7
:1041400000285FD03D494978814201D10920F2BD64
:10415000012004F0AAF9286000260120A87303F0CA
:1041600057FAFFF701FA6C48182101FB0607387B64
:1041700040F080003873A87C012807D026B9FFF7EB
:10418000ABF900F5C87000E00020B860761C032E83
:10419000E9DB207828B9A97C6048085C2070FFF72B
:1041A000E7F90020F2BDA87B08B92120F2BD38480C
:1041B000006880470646FFF7DFF9012804D0FFF7C3
:1041C00097F92968884207D103F022FA40F20240A9
:1041D000FFF79AF9012700E000270020A87328685C
:1041E00003F098FB2846FFF7CBF9207810B903F0CD
:1041F0004AFA02E00FB1FFF7BBF92A4909683046D5
:104200008847CEE71220F2BDEC490020964C0020F2
:10421000017841F08F010170C17841F02001C17037
:10422000817841F0300181700020704710B103495E
:104230004978017000207047F44E0020B04C0020F7
:1042400070B504460D461646FFF772F930B9FFF710
:10425000B8FC00F58E7005704680002070BD304BB4
:1042600010B1012802D00AE0198070471888107038
:104270001888000A507000209070D070704712208B
:10428000704700000C4F00201C4F0020104F0020F2
:10429000344800202C4F002010100440000004601F
:1042A000944C002038480020E84E0020C44C0020E8
:1042B00004000940B94C00208C4A00209C4C00208E
:1042C000864C0020BA4C0020874C0020884C0020EF
:1042D000BB4C0020894C00208A4C0020BE4C0020A2
:1042E000B84C0020D04E0020404E0020294176716D
:1042F000284E0020204F0020A84E0020DC4E002039
:1043000002000080C44E0020844E0020C04C0020DB
:1043100001000080BC4C0020244C0020C0D90010BB
:10432000984C0020DFF800F0818C00109E4890210E
:10433000017088214170012181700221C17000212A
:10434000017180214171002181712021C171002101
:1043500096488160C1601F21017000214170418039
:1043600041601F209249087070472DE9F04100F02C
:1043700078F81F463ED58D48007840073AD5DFF8DB
:10438000348298F8000098B10C20FCF7DFFC88B369
:104390009121017084803E214170C580032181708C
:1043A00006810021C1704781014698F8000020E095
:1043B0001520FCF7CBFCE8B101210170042200F0CC
:1043C000C0F80A704C713E224A70CD710A228A7080
:1043D0004E720322CA70CF7200220A71220A8A71B9
:1043E0002A0A0A72320A8A723A0A0A730146724823
:1043F0000078E7E0BDE8F081F8B500F032F82FD59D
:104400006A48007800072BD51720FCF79FFC0700AF
:1044100026D0012038700822FF20787007F10800AC
:1044200078600420796808703E20796848700C2014
:104430007968887004207968C87078680471786831
:104440004571280A7968887131467868C01DFCF783
:104450002EFC3946BDE8F44057480078FCF797BC7D
:10446000F1BD04465048C07980060D461646704797
:10447000F8B5524E074630780C46154620B3B800C2
:104480000C3080B2FCF762FC00284DD09021017006
:1044900087701321417000F10C01416000EB47016E
:1044A0000C31816000210AE0436834F8112023F8C0
:1044B0001120836835F8112023F81120491CB942D6
:1044C000F2DB014630782BE0B800461C06F10B0009
:1044D000C0B2FCF73BFC38B30121017000F031F8A9
:1044E00004214268117013214268517041688E7036
:1044F0004168CF7000210EE000F01DF8137100F04C
:104500001AF81B0A537100F010F8937100F00DF8BF
:104510001B0AD371491CB942EEDB014626480078DC
:10452000BDE8F440FCF733BCF1BD426835F811300A
:1045300002EB81027047426834F8113002EB8102CD
:104540007047FF21417000F10801416070472DE97B
:10455000F041184F044638780D469046C8B11848C7
:104560000078B0B905F10C0080B2FCF7EFFB060053
:1045700017D0912030702A46FF207070B570B4803B
:1045800006F10C00B0604146FCF791FB38783146EB
:1045900018E043462A462146BDE8F041FF20FFF7D8
:1045A000C1BEBDE8F0810000004F0020204800207F
:1045B000084F00207A480020784800207B480020DF
:1045C000284F0020BDE8F041FCF7E1BB80B5184959
:1045D0000870002048708870C87008714871FFF733
:1045E000A5FE14490020087001BD38B50C46200412
:1045F00012D50F480078FCF728FC050009D0287870
:10460000032812BF0128E868FDF7C7F92846FCF720
:10461000AFFB84F4004032BD002032BD04498870F5
:1046200070470349C870704701490871704700001E
:1046300078480020284F002010B5924C2070FCF7DD
:10464000D5F9302200219048FCF763FB8F49607850
:104650000978081860700006000DFBF7BBFC60606D
:1046600088B161780A010021FCF753FB0020FF228A
:104670006178C0B288423FBF616801EB00114A72A5
:10468000401CF5D300E060702078FFF7CAFFBDE85A
:1046900010400FF2FD10FCF7CFB938B50C462004DE
:1046A000784D0CD52878FCF7D0FB050004D000F03D
:1046B00018F82846FCF75CFB84F4004032BDE007A4
:1046C0000DD5FEF773F900281CBFA878002803D089
:1046D00028780121FCF731FC84F0010032BD002074
:1046E00032BD3EB504462078902848D16078132822
:1046F00014D10020634A05E0A36833F8103059183C
:104700009170401CA3789178C0B29842F4D30029EC
:1047100035D010780121FCF710FC37BD65882146A3
:1047200000A8FEF7CDF90199F9B1BDF80000052800
:1047300004D100A9284600F023F818E004281CBF83
:104740000628072813D150490C2202FB001030F82C
:10475000301D61B1807800AA2946FEF75AFA30B9B7
:10476000BDF8000004280AD005E0012803D1A068A4
:1047700008B1FDF712F901212846FCF7DEFF37BD2D
:10478000F0B50E46044630890025042889B044DB84
:10479000716802A8FEF782F8BDF80A20182A63DAC9
:1047A0003189101D814235D19DF80800C00736D5EA
:1047B0007068071D9DF80900FEF7A4FA06002CD0CA
:1047C00035719DF8080001280BD0132821D13078CD
:1047D000042822D1BDF80A20394603A8FEF70DFAB5
:1047E00005E0BDF80A20394603A8FEF7B3F90546EF
:1047F0003046FEF7A7FA03A80190002000902A4651
:104800009DF80830307A2146FEF725FA3046FEF74B
:1048100072FA15B12046FEF7C2FA09B0F0BD9DF854
:104820000800122817D17068011D03A8FEF7C8F907
:104830000500EED1144881890029EAD003A901912D
:1048400000229DF809109DF80830807B00912146D8
:10485000FEF701FADDE79DF80910ADF8005000AA57
:104860002046FCF737FFD4E70120ADF80000172001
:10487000ADF8020000AA9DF809102046FCF72AFFB7
:10488000CBE7000070480020A44700206C470020C0
:1048900010B504464FF6FE7084420ED0012906D0B2
:1048A00002290AD101212046FCF74AF928B92046FD
:1048B000BDE810400021FEF773BA10BD984948705A
:1048C000704710B5964C2070FFF7A8FE2078BDE821
:1048D00010400521FCF7B8BE7CB5914D28780C46F8
:1048E000210419D5FCF7B1FA060084F4004411D074
:1048F00000F057F858B93078A22806BF89480078E8
:104900006878FF2803D03146FCF741FA02E03046D0
:10491000FCF72EFA204676BDE10709D5A86820B13C
:10492000416808001CBF0020884784F0010076BD64
:10493000A10709D5686820B1416808001CBF0120A3
:10494000884784F0020076BD610726D5764E31880F
:10495000E9B1481E308080B2E0B904F001F848B1F6
:10496000724901200870686820B1416808001CBFC6
:104970000120884702F0A6F800A9FEF777FA00A800
:1049800002F011F81D2001F02BFF308002E004211D
:10499000FDF78CFC84F0040076BD002076BDFCF7AA
:1049A000E6B838B502780124912A4FF6FF7103D09A
:1049B000A22A00F08E8092E04278594B052A4DD011
:1049C0000E2A04D00F2A4CD03E2A6DD087E0828870
:1049D00041F20905511B32D040F6F975491B34D01C
:1049E000C91E36D0491E09D0891E022906D9C91E02
:1049F0001BD0491E15D0891E08D070E059680029C7
:104A00006ED009680A006BD0884766E0484909689B
:104A1000002965D04B68190062D0014642F20E00B1
:104A200040E08168097800295AD09968002957D058
:104A30000B68190054D00146104698474DE0806835
:104A4000411C007801F073FF47E0806801F08BFFA4
:104A500043E08068007801F0E4FF41E002F057FA9B
:104A60003EE0828842F20D05531B13D09B1F02D0FB
:104A70009B1F0FD033E02F4B1B888B420AD02E494F
:104A8000096869B30A6811002AD0014642F213008E
:104A9000904722E02649096811B34B6819001FD0DE
:104AA00001461046984718E08178012907D016D3AF
:104AB000032901D006D312E0024680880BE002F001
:104AC000CEF90DE0996859B149680A0008D08847C5
:104AD00006E00246408800F005F8044600E00024A5
:104AE000204632BD70B50C461546FCF73AF8012653
:104AF000042804D11048006858B1026803E00C484B
:104B0000006830B14268100003D029462046904723
:104B10000646304670BD02494860704700000000FC
:104B2000804500200445002008450020074500205E
:104B3000E4440020D84400209048002010B53C4CAC
:104B40002070FFF771FD20780621FCF77DFDBDE8A0
:104B500010403848FBF770BF38B50C46200416D516
:104B600033480078FCF771F905000DD000F01FF80C
:104B700038B931480078FF2803D02946FCF707F9F7
:104B800002E02846FCF7F4F884F4004032BDE00768
:104B900004D503F0B5FF84F0010032BDA00704D5B1
:104BA00004F079F884F0020032BD002032BD38B53F
:104BB000044601252078922802D0A0282CD033E08A
:104BC00060780E2802D03E280BD02DE0A08842F25B
:104BD0001801884228D1A068411C0078FEF786F9A8
:104BE00018E0A078052806D008281DD1A179A08852
:104BF00003F0FCFF0EE0A088FBF7B3FF042814D1FC
:104C00000E48006888B1836818000ED0E289A08839
:104C1000A11D9847054608E0204603F073FFA068F1
:104C200018B1FCF7BAFE00E00025284632BD0000AE
:104C3000B5480020E98A0100814500204048002055
:104C4000DFF800F0F9990010DFF800F0159A001075
:104C50007CB5164600244FF48063C21ADFF85C5C12
:104C60001DD0521E22D0521E25D0521E2AD0521EB6
:104C70002FD0521E34D0521E3BD0521E40D0521E56
:104C800043D0521E4AD0521E70D0521E75D0521EB2
:104C90007AD0521E00F08080D21E4AD08AE00129CC
:104CA0000AD1307803280ADA68708DE0022903D12E
:104CB0003088A88388E001297AD13078022877DA11
:104CC000A87081E0012973D13078052870DAE87086
:104CD0007AE001296CD13078022869DA287173E012
:104CE000102965D11022314605F13000FBF7DFFFB6
:104CF0006AE001295CD13078022859DA687163E0F2
:104D0000012955D1307828725EE0042950D13068ED
:104D1000DFF8AC1B88424BD2286255E0002947D10E
:104D2000FFF73DFE10B900F003FC17E00120E87228
:104D30004AE007293CD10622711C6846FBF7C1FFF7
:104D400030780022694600F049F906460A2E3ADA20
:104D5000FFF725FE30B9304600F0F6FB502001F099
:104D600003FD22E0A919012008742DE001291FD1BB
:104D7000307802281CDAA87126E0012918D1307891
:104D80000A2815DAE8711FE0012911D13078C11F16
:104D90000A290DD2687217E0012909D1A97A307861
:104DA000A872002908BF01280ED100F089FB0BE092
:104DB000182409E0272806DA022904D1318801F0F5
:104DC00001FD044600E00224204676BD38B50024EB
:104DD0004FF480630D46C21ADFF8E01A1AD0521E53
:104DE0001AD0521E1AD0521E1AD0521E1AD0521E5B
:104DF0001AD0521E1ED0521E1ED0521E1ED0921EFF
:104E00001FD0521E1FD0521E1FD0521E1FD0521E26
:104E10001FD022E048781EE0888B22E088781AE0D4
:104E2000C87818E0087916E0102230312846FBF7E0
:104E30003EFF19E048790EE0087A0CE0086A286025
:104E400012E0887907E0C87905E0487A03E0887ABB
:104E500001E000F05AFB287006E0272803DA01F091
:104E6000BFFC288000E00224204632BD2DE9F04F2F
:104E700093B092461C4609AA0023C2E90033DFF82A
:104E80003C7A00F0ABF806460A2E6BDA4FF0060BC0
:104E90000BFB06F808F1200000F045FA00287878AE
:104EA0000CBFBDF80C904FF0000902280CBF012583
:104EB00000250BFB06F0082C0CBF00F1220B00F1C3
:104EC000210B1C2200210BA8FBF723FF0BAA1C219E
:104ED0005FFA8BF001F034FC09F0010950B99DF83C
:104EE0004600C01F0A2805D22B460BAA4946504649
:104EF00001F04CFF1422002104A8FBF70AFF08F17F
:104F0000240004AA102100F010FA80B91022FF2119
:104F100004A8FCF7EEF950B908F1250008AA04210D
:104F200000F003FA04AA4946504601F070FE06F16B
:104F300070006A46102100F0F8F998B9684600F050
:104F400005FA002630463DF8201041B1694601EBD4
:104F500080018A783DF820105046FAF7DDFF761C74
:104F6000042EEFDB042C04BF787802280AD179796B
:104F7000002001B10120B97801B10421014350465C
:104F800004F0D8F8002013B0BDE8F08F70B5FFF73B
:104F900006FD10BBDFF82449E07A01280AD100F0B1
:104FA000C7FA0020E0720A22002104F11000FBF78A
:104FB000B0FE0CE000256619307C012804D128469B
:104FC00000F0C2FA002030746D1C0A2DF3DB502073
:104FD00001F0CAFBBDE8704072E270BD2DE9FF41EF
:104FE0000A2403280D46164643D8DFE800F00202E3
:104FF0001021284600F04FFA04460A2C39DA002E18
:1050000037D0062229463046FBF751FE31E0002713
:10501000DFF8B0880E207843404406222946801DE0
:10502000FBF769FEE8B97F1CFFB20A2FF2DB20E034
:1050300000270620784323306A46102100F075F9D6
:1050400050B91022FF216846FCF753F920B92946D0
:10505000684603F083FC20B17F1CFFB20A2FE8DB17
:1050600007E00A2F3C4604DA1EB13146204600F024
:10507000FBF9204604B0BDE8F081F8B50C461526D2
:105080004FF6FF71884215460BD100272A4621466C
:10509000384600F0FFF800B100267F1C0A2FF5DB30
:1050A00010E0FBF71FFD60B1811D40790022FFF782
:1050B00095FF0A2806DA2A46214600F0EBF800267A
:1050C00000E014263046F2BD10B5DFF8F047217835
:1050D0006062262001F076FB2078BDE81040F9F7E9
:1050E000A7BF38B50446002508000DD1DFF8D0076A
:1050F000DFF8CC37B2FBF0F0214603FB102001F0C3
:105100001FFE050003D00121204601F0F1FD2846D5
:1051100032BD70B5044686B0A078DFF8A0570628E7
:1051200000F0AA80092867D00A281AD00B2804D0DA
:105130000E2858D00F286ED0A1E0686A40B10668EA
:10514000300005D0637B227B6189E01CB04796E08C
:105150006189286A01F0F4FD0028F8D060890121F6
:1051600077E06078002660BBA079C00729D5A86ADF
:1051700038BB0E2200F08AF8606918B1062200F1EF
:10518000100106E0A088FBF7ADFC002877D00622CE
:10519000811D6846FBF78BFDA179BDF80C008908DD
:1051A00001F001010843ADF80C002146684600F00B
:1051B000DCF828B928780221FBF7BFFE00205FE069
:1051C0001526686A00285AD04368180057D06278BC
:1051D000A08801219847300051D06B6AA0885B6895
:1051E0003246032146E0686A002848D04368180028
:1051F00045D0627802213CE0E0780022211DFFF7D3
:10520000EDFE0A283BDA06235843253004F10C0250
:1052100000F038F833E0A088A97909B1E97918E0FD
:10522000697809B9052114E0FBF75CFC060026D07B
:10523000A07AC00710D5707901000DD0E168C1F3E4
:10524000402149B904AAB11DFFF7C8FE20B9A088C2
:10525000032101F04DFD12E07179A08804F10802EC
:1052600000F0A6FA686A50B14368180007D000221F
:105270000021A088984702E0A088FFF787FE012060
:1052800006B070BD0421C0B201F0E8B90021684643
:10529000FBF73FBD70B506460620704388B00C464C
:1052A0001546203004AA00F03FF8002838D1062225
:1052B000FF2104A8FCF71DF890BB70366A46102148
:1052C000F0B201F03DFA48BB684600F03FF820001C
:1052D00009D1102200216846FCF70BF8F0B9102222
:1052E000FFF7D4FF12E0694600F022F838B9280031
:1052F00016D06946002000F01BF888B10480817840
:10530000A9420BD085700DB900210180684600F0DC
:105310001DF86A461021F0B201F0A0F9012000E06A
:10532000002008B070BD6A460E21C0B201F008BA74
:10533000002231F82230834202D101EB8200704713
:10534000521CD2B2042AF4DB00207047002130F84E
:105350002120D24320F8212000EB8102491C9378C0
:10536000DB4304299370F2DB70472DE9F043DFF84B
:105370004C45DFF850958046A06A85B00F460E2652
:10538000C8B9B8F1000F18BF002F69D0404600F02F
:1053900082F80A2820730EDB002506FB05F00622A2
:1053A000FF214844FBF7A5FF20B96D1CEDB20A2D83
:1053B000F3DB0A252573207B0A2851DA0625A16A2A
:1053C0006843B1B9203042460E21FFF75CFF10223E
:1053D000FF21FFF75CFF207B703000F023F9207B7A
:1053E00070430E2241464844FBF761FCA76200204F
:1053F00037E08A683AB121301C21FFF744FFA16AE7
:1054000000208860F3E70A693AB122301C21FFF7D7
:105410003AFFA16A00200861E9E74A693AB12330FE
:105420001021FFF730FFA16A00204861DFE7CA685A
:1054300082B124301021FFF726FFA06AC06800F176
:105440001002207B68432530FFF71CFFA16A002073
:10545000C860CCE7A07A08B100F00CFA00F099F926
:10546000012005B0BDE8F08330B50A2885B00C46B0
:1054700000DA0CB902200CE0062358432030FFF775
:1054800052FF050004D1062269462046FBF70FFCB7
:10549000284605B030BD70B504460025DFF8246409
:1054A0000E206843062221463044FBF724FC08B155
:1054B000284670BD6D1CEDB20A2DF1DB0A2070BDCF
:1054C00038B5002400F0E9F90620604320302A4670
:1054D0000E21C0B201F034F958B10622FF2128464E
:1054E000FBF717FC0622FF21A81DFBF712FC00208A
:1054F000A881641C0A2CE5DBDFF8C003807A08B1C0
:1055000000F0B8F9BDE8314043E170B50024002552
:10551000DFF8B0630E2068430622FF213044FBF71A
:10552000E8FE00B9641C6D1C0A2DF3DBE0B270BD0F
:1055300010B50024204600F007F8641CE4B20A2CE1
:1055400001DA0100F6D010BD2DE9F047DFF86C5309
:10555000297B884290B0814609D128780121FBF748
:105560003BFD28780221FBF737FD00F09BF9062070
:1055700000FB09F505F1200607AA0E21F0B201F0A3
:10558000DFF8002845D10622FF2107A8FBF7B1FE6E
:1055900000283ED10E22FF2107A8FBF7BAFB1C22F0
:1055A000FF21FFF774FE1022FF210BA8FBF7B1FBD0
:1055B00007AA0E21F0B201F051F8064605F12100CC
:1055C00000F02BF8824605F1220000F026F8804614
:1055D00005F1230000F026F8044605F1240000F050
:1055E00021F8074605F125006A460421C0B201F002
:1055F00035F848EA0A012143394340EA010509F137
:1056000070000BAA1021C0B201F028F828433043E3
:1056100000E0002010B0BDE8F0876A461C21C0B24F
:1056200001F01CB86A461021C0B201F017B8A349B6
:10563000087045E7F0B50D46280485B09F4C25D588
:105640002078FBF702FC04001DD021780120B0294E
:105650000FD0B12905D0D02904BF2046FFF759FD4E
:105660000DE0207960B92289E1886088FFF705FDA7
:1056700006E0217904F10800FBF7D0FF00E010B14B
:105680002046FBF775FB85F4004065E0A80709D5C7
:1056900000210020FFF769FE002885F0020550D1A7
:1056A00002214FE0E80752D5A06A8688E06A4FF6EB
:1056B000FF7748B904F11E0000900223824A394660
:1056C0000120FAF78EFDE06285F00105E16A21B361
:1056D000FF20039002200290002001900DF11200A3
:1056E000009004ABE28B3046FAF7D8FA68B99DF81F
:1056F00010009DF8111000EB012290B228B1E06A71
:10570000418992B23046FFF7B8FCE28BE06A002391
:105710003946FAF7B8FDE06298B9606A70B143683B
:1057200018000BD0A06A8088002201219847A06A47
:10573000636A80885B6800220321984700F0B2F812
:1057400003E001212078FBF7F8FB284604E0680716
:105750004CBF85F00400002005B0F0BD10B5203826
:10576000062390FBF3F30624012204FB1300052813
:105770000DD8DFE800F00305050707090E2904E04E
:105780001C2902E0102900E0042908BF002210466D
:1057900010BD80B5FFF7B9FE0228ACBF02200A2079
:1057A0008DF800006A460121052003F049FD01BD86
:1057B00070B588B006460C4615462022FFF766FDF8
:1057C000ADF800603D4EF078327A31798DF8040002
:1057D00002F00103707A8DF81C008DF80510069810
:1057E000400843EA40006FF002030340500800F015
:1057F000010043EA400020F48073100900F001002A
:1058000043EA002020F40073500900F0010043EA4D
:10581000402020F48063900900F0010043EA8020DA
:105820006FF004039208184002F0010240EA82007F
:10583000069031B1102206F130010DF10600FBF7A0
:1058400036FA707928B11CB1069840F00200069033
:1058500001209DF816100843B1788DF8160001B1AB
:10586000042108438DF816002946684601F0F3F933
:1058700008B070BD38B5FFF7E3F9002400F00DF86B
:105880000622FF212846FBF734FD10B92946FFF711
:10589000DBF9641C0A2CF1DB31BD0E2109486143A0
:1058A0004518704710B5054CA06A18B1FBF760FAAF
:1058B0000020A0620A20207310BD0000E8430020F1
:1058C00040420F00A8460020B4C90100DFF800F0F4
:1058D00041950010DFF800F071950010DFF800F03E
:1058E000D1950010DFF800F03D970010DFF800F0D0
:1058F00065970010DFF800F08D970010DFF800F0DA
:1059000029980010DFF800F0F5980010DFF800F09B
:10591000C9990010DFF800F0319A0010DFF800F0AC
:10592000A19A0010DFF800F0F59A0010DFF800F0FF
:10593000159C0010DFF800F08D9C0010DFF800F0DF
:10594000099D0010DFF800F0459D0010DFF800F021
:10595000D19D0010DFF800F02D9E0010DFF800F060
:105960004D9E0010DFF800F06D9E0010DFF800F093
:105970008D9E0010DFF800F0AD9E0010DFF800F003
:10598000CD9E0010DFF800F0ED9E0010DFF800F073
:105990000D9F0010DFF800F0499F0010DFF800F0C5
:1059A000699F0010DFF800F0D19F0010DFF800F0D1
:1059B00011A00010DFF800F031A00010DFF800F0B7
:1059C00075A00010DFF800F0F1A00010DFF800F083
:1059D00009A10010DFF800F0B5A10010DFF8E01811
:1059E000087070472DE9FE430C46200454D5DFF8BB
:1059F000D0080078FBF729FA05004AD0DFF8C47810
:105A000039680126002918BF11F1010F07D0DFF80E
:105A1000B8080078FBF7BBF94FF0FF303860287802
:105A2000812802D082282CD02FE000208DF8086039
:105A30008DF80900AE88AF7995F80280B00A3F284A
:105A400007D1C6F3C21020B100F029F800F02EF8FB
:105A500003E000F024F800F080F881462846FBF7C8
:105A600087F99DF80800A0B1DFF8600801904B4667
:105A70009DF8090000903A463146404600F0B2F9E0
:105A800007E0284600F046FB064616B12846FBF71D
:105A90006FF984F4004000E00020BDE8FE8302AB13
:105AA0000DF10902294630467047000038B500F074
:105AB0007F04C00900F00700401E04280D464AD8A4
:105AC000DFE800F0030C2C3F4400122C43D12A7C69
:105AD000E9682889BDE83840FBF703BE2889E968F2
:105AE000012C17D00B2C11D00D2C0BD0132C05D062
:105AF000192C30D1BDE83240FBF7E7BEBDE832409B
:105B0000FBF7D0BEBDE83440FBF79EBEBDE8344095
:105B1000FBF78CBEBDE83440FBF735BE28891B2C53
:105B200009D01D2C17D16B7C2A7CE96801B0BDE837
:105B30003040FAF752BC2A7CE968BDE83840FAF7F1
:105B400079BC204601B0BDE830400CE2204601B0EF
:105B5000BDE830408AE1012032BD0B4640F21D41D4
:105B6000401A00F0978040F2E471401A00F09580EE
:105B7000801E00F098802A3800F09780363800F0B8
:105B80008F8040F29E31401A00F09480401E00F059
:105B90009380401E00F09280801F00F091804FF4AF
:105BA0007F71401A00F08E8040F6FC31401A00F000
:105BB0008C80801E00F08C80001F00F08B800838E5
:105BC00000F08A80401E00F08980401E00F088802E
:105BD000401E00F08A80C01E00F08C80401E00F045
:105BE0008C80401E00F08C80401F00F08D80401E95
:105BF00000F09180401E00F08980401E00F08F80F0
:105C00004DF6E231401A00F08C80401E00F08D808D
:105C1000C01E00F08E80401E00F08F80401E00F0FD
:105C20008F80401E00F09480401E00F09780401E40
:105C300000F09680401E00F09780401E00F0968095
:105C4000401E00F09680401E00F09680C01E00F0BE
:105C50009580801E00F09680401E00F09680401EC9
:105C600000F09880801E00F09980401E00F09B801C
:105C7000801E69D0401E00F09C80401E00F09E8077
:105C8000401E00F09E80801E00F09F80401E00F0AD
:105C9000A280A5E01889FFF719BE9868FFF71ABE21
:105CA0009868FCF799B9FCF7FDB859891889C9B209
:105CB000FFF714BEFCF7F2B9FCF705B9FFF712BE07
:105CC000FFF714BE1889FFF715BE9868FCF7CBB92B
:105CD000FFF714BEFFF716BEFFF718BEFEF7B0BF02
:105CE0001889D968C0B2FEF7AFBF1889D968C0B2A9
:105CF000FFF710BE1889FFF711BE1889FCF745B9E8
:105D0000D9689868FFF70EBEFFF710BE9A7A597AE5
:105D1000187AFCF74FB91889C0B2FCF754B9FFF7ED
:105D200009BE1889C0B2FFF709BE1889C0B2FFF7D3
:105D300009BED9689868FFF709BE9868FFF70ABEE0
:105D40001889C0B2FFF70ABE1889C0B2FFF70ABEB1
:105D500059891889C9B2C0B2FFF708BEFFF70ABE59
:105D60001889C0B2FFF70ABEFFF70CBE9868FFF7AC
:105D70000DBE1889FFF70EBEFFF710BE1889C0B21E
:105D8000FFF710BE1889FFF711BE59891889C9B2EB
:105D9000FFF710BED9681889FFF710BE1889598916
:105DA000C0B2FFF70FBE59899A891889C9B2FCF7AA
:105DB00058B918895989C0B2FFF708BE1889FCF78D
:105DC0003EB91889C0B2FCF723B959891889C9B2FC
:105DD000C0B2FFF7FFBD1A69D9689868FCF77DB8B3
:105DE000012070472DE9F843089C804604F10C001F
:105DF0000F461546994680B2FAF7A8FF060016D05E
:105E00008020307086F8019040F27F607080B7800B
:105E1000B57106F10C00F471B06022460999FAF7E9
:105E200046FF31464046BDE8F443FAF7B0BFBDE84F
:105E3000F18310B502460020941E012C02D9A41E45
:105E400002D004E0102900E004290ED00CE0A2F1F9
:105E50002004402C04D2BDE810401046FFF77EBC61
:105E6000A2F18001102900D3022010BD70B5401EA0
:105E7000052882B00C461546DFF8546448D8DFE8A0
:105E800000F0030C15182A3600F044F808BBE2684D
:105E90003146284600F054FC76BD00F03BF8C0B90E
:105EA000E2683146284600F0D9FB76BDFCF7A1F93F
:105EB0000FE0A06868B1DFF81C140160DFF8181467
:105EC00009888180912181710321018114214181FF
:105ED0001CE0022076BD01F0EBFDB071010AF1710A
:105EE000010C000E70723172042028700EE04FF623
:105EF000FF70ADF80000FAF736FDADF800000222A1
:105F0000022028706946B01DFAF7D1FE002076BD48
:105F1000012076BD257A667A3146284689E738B56C
:105F2000012815461C4602D0022809D00DE0049B2A
:105F30000A462146284601B0BDE83040FBF732BB97
:105F40000846BDE83240FCF77BBF0846BDE832405A
:105F5000FBF70CBD0B4601281146184608BFFBF79E
:105F60005DBBFBF71ABDF0B583B00F461446DFF8F2
:105F7000605360B3032845D0062833D0072836D0B5
:105F800008283BD00A2842D00B284AD00C285FD0E2
:105F90000D2800F083800E2854D00F284BD01028F5
:105FA00044D0112839D030285CD0312863D0322831
:105FB00053D0332877D0342879D0352800F0878023
:105FC000362800F08780372800F08B80A0E07869C1
:105FD000019038690090FB68BA7A797A387A03F0D0
:105FE000A3FAFEBDF968387A03F0C6FAFEBDFB6875
:105FF000BA7A797A387A03F00EFBFEBD387A03F06C
:1060000041FBFEBDF968387A00F026FCFEBD3A7B04
:106010007989387A00F086FDFEBDB86800F0BFFDD2
:10602000FEBDF968B86800F016FEFEBDB97A388981
:1060300000F05EFEFEBD3B7CFA68B97A388900F05C
:10604000A5FEFEBDFA68B97A388900F0E0FDFEBD14
:106050003989F86800F05BFEFEBDF968B86802F0A7
:106060007DFCFEBD3889798926282ED027282CDA98
:1060700000F0A8FBFEBD4FF6FF76ADF80060388952
:10608000FF2822DA262820D027281EDA00F0A8FBD5
:10609000B042ADF8000018D002200EE0B97A38897D
:1060A00003F048F8FEBDB86803F012FBFEBD387A75
:1060B00003F040FB009040B1042020700246694686
:1060C000A81DFAF7F4FD0020FEBD0220FEBD03F07E
:1060D0003BFBFEBD7989FA683889C9B2FEF7B8FD85
:1060E000FEBD3E89A91D3046FEF770FE40F201411B
:1060F000761A04D0361F04D0F61E04D005E0022123
:1061000004E0102102E0042100E001212170FEBD25
:106110000120FEBD2DE9F04184B0044600208DF839
:10612000090001208DF80800A588A079A778042D22
:10613000804662D8DFE805F061030A283D0002AA24
:106140000DF10901204600F074F854E000261028F3
:1061500014D013280DD0142807D015284DD1E2688B
:10616000A17A2089FAF7DFF845E0A068FBF7F0F89C
:1061700007E0A17A2089FBF7E5F802E0207AFBF737
:10618000DEF88DF8086039E078B1052802D00628DD
:1061900006D032E02089E168C0B203F091F82AE02D
:1061A00000F041F803F04CF825E0A06803F0A3F8F4
:1061B00021E0062821D8DFE800F01B20140F20047E
:1061C0000A002089E168C0B2F8F7F7FF13E000F099
:1061D0002AF8F8F7C2FF0EE0E1682089F8F79CFF83
:1061E00009E02369A27BA189A068F8F76BFF02E0B0
:1061F000A068F9F73DF8064600E001262046FAF7C8
:10620000B7FD9DF8080050B13048019033469DF825
:1062100009000090424629463846FFF7E3FD00207A
:1062200004B0BDE8F08161892089E268C9B2C0B2DA
:106230007047F8B50D468179254F0024042916468C
:106240001AD010290CD011290ED0122911D01329DF
:1062500016D014291AD0152920D0172923D02BE0C5
:10626000007AFEF72BFB1CE0817A0089FAF768FCC4
:106270001EE0FAF78FFC1BE08068FEF725FF10E0B8
:10628000C268817A0089FEF72CFF05E0837C028AD0
:10629000C168007AFEF7EAFD04460EE00089FEF7C9
:1062A00075FE347009E00269C168007AFEF796FE57
:1062B000B8710120287000E001242046F2BD0000E2
:1062C000B248002018480020784800203A470020B3
:1062D00034470020000102007E17010010B50400C1
:1062E00082B01FD0207B8DF80000607B8DF801000C
:1062F0006846FBF743FA206908B10B490160606901
:1063000008B10A4901600A4821780170617841703A
:10631000A1788170E178C17061684160A168816095
:10632000A169C16013BD00BF1F5F0100555F01007F
:106330003C46002038B1DFF86824DFF868041268B2
:10634000526801211047704738B5DFF8584420469D
:1063500003F04CFC0546C0B258B1DFF84424126883
:106360005268002120469047204603F03FFC002859
:10637000FAD1E8B232BD70B5DFF82C542E78002483
:1063800082B02C71EC70AC7003E0F0B200F05DF8FC
:10639000761C6878F1B288421ED304236A46002135
:1063A000F0B203F02BFC0098B0F5801F0CD1A87858
:1063B000010007D000F049F8F0B200F046F80020E4
:1063C000A870E5E7AE70E3E70028DED1E0B208B1DF
:1063D00000F03BF83446DBE7A8780028E0B20DD1A6
:1063E00028B9287800F014F80420E8800BE0AC709D
:1063F00000F049F8E0B200F07FF804E008B100F0E6
:1064000024F800F040F82979481E8041C00F76BD7D
:1064100010B582B004464FF48010009001236A4604
:106420000021204600F0D2F8DFF87C03C17801B9E2
:10643000847013BD80B5002000900123DA48807875
:106440006A46002100F0C2F801BD70B50446D74885
:10645000006880470546FFF777FF06460021204683
:1064600003F0EDFB03F0F6FB04463046FFF762FF56
:106470001CB1CD4801210171C1702846BDE87040B2
:10648000CB490968084738B540F6FC74C64DA87872
:1064900004236A46214603F0B1FB009810F1010F76
:1064A00003D1241FA4B2042CF1DA201DE88031BDF1
:1064B00070B582B0044615460E1F00E0361FB6B216
:1064C000042E17DB04236A463146204603F096FB70
:1064D000BDF80010BDF80200A94203D1C0B2301AC5
:1064E00080B276BD0104E9D4011D8E42A4BF301AEA
:1064F000061FE4DA002076BD2DE9FE4FAA4E96F87D
:1065000000A08046504508BF96F801A0F0884FF0E3
:10651000FF0B04271AE0BDF808002918B0780423FF
:1065200001AA89B203F06AFBE919012301AA89B221
:10653000504600F04BF82D1DADB2A945EBD2BDF889
:106540000200001DC719BDF80200201A041FA4B2E2
:10655000042C30DB3079B8BB04236A462146404620
:1065600003F04CFBBDF800004FF6FF71884209D1E3
:10657000BDF80200010448BF241FE8D4001D844276
:10658000E1DA21E00004DED4BDF800005FFA8BF10F
:106590008842D8D083465FFA8BF2B9B25046FFF7F3
:1065A00087FF0028CFD1BDF80290A4EB0900ADF819
:1065B00008000025C1E75046FFF72AFF307918B9D7
:1065C000F7804046FFF741FFBDE8F78F2DE9F04720
:1065D000754C82B08046E0780D4616461F4660BB7B
:1065E0007248006880478146FFF7AEFE8246294622
:1065F000404603F024FBBA00314603F01BFB504633
:10660000FFF798FE01E02D1D361D3846471EC0B22B
:1066100078B104236A46A9B2404603F0EFFA042297
:1066200031466846FAF767FB0028ECD1012020715B
:10663000E07048465E4909688847BDE8F3875A48D4
:106640005C49090B10B5017000240178491C4170A8
:10665000FFF791FE00B90124204610BD2DE9FC474B
:106660008146514E002030710F469246F188B07835
:106670004A46FFF71DFF8046B0B1002410E0B07815
:10668000012301AA1FFA88F103F0B8FAE4B29DF8D9
:1066900004001AF80410884206D108F10108641CAD
:1066A000E0B2B842EBD341D0F81C411000EB91703E
:1066B00080108700F088BFB23818001DB0F5805FE9
:1066C00004DDFFF7B7FEB078FFF716FFB478B6F831
:1066D00006804FF6FF70ADF8000007EB080547F4A1
:1066E000004000F026F8BDF80200C0F30E0000F0F4
:1066F00020F8BB051B0E524641462046FFF766FFB9
:1067000049F40040ADF8000000F015F8BDF80000B5
:10671000C0F30E00ADF8000000F00DF8307908B1BC
:106720000A2004E0F088391D0818F0800020BDE838
:10673000F687ADF8020001236A46A9B2204645E774
:1067400070B51546184E0C460246F188B078FFF732
:10675000AFFE010006D0B07823462A4603F04EFA79
:10676000002070BD0A2070BD10B5A0F146011A29A5
:1067700001D3022010BD0C4CE17871B9E18864228C
:106780005143B1EB003F08D300202071FFF752FEC8
:10679000A078FFF7B1FE002010BD0A2010BD000058
:1067A000D801001000400340584800203448002021
:1067B0003848002000D0010070470000DFF800F0EA
:1067C00049980010272809DA4FF6FF72914205D048
:1067D000DFF8382322F8101000207047022070479D
:1067E000272803DAC94931F8100070474FF6FF70C7
:1067F000704770B504460D46C54E1C220021304638
:10680000FAF787FA34777577FFF770F800280EBF2C
:10681000012100211220317070BD38B5BC4D0446F5
:106820000846EA60A8606C6010220021FAF761FD5A
:10683000012803D1A8681021FCF74DFC102200218B
:106840002046FAF756FD012805D16868BDE83440B6
:106850001021FCF740BC31BD2DE9FC41AC4D044694
:10686000002695F81E80042C0F4624DA2878032889
:1068700018BF102054D1FEF792F828B902F070F832
:1068800010B902F071F808B1122049E0012C18BFCC
:10689000022C1DD1BFB10622002100A8FAF739FA57
:1068A00000F040F838B90622FF2100A8FAF731FAC3
:1068B00000F038F808B1022032E00622394600A87C
:1068C000FAF7F5F90BE0062100A8FCF704FC06E056
:1068D000032C04D1686800A9FCF7C8FA06468D4F5E
:1068E000AC7704213878FBF7E1FC002028849EB9BE
:1068F000ACB100A800F057F806000DD1032C0ED162
:106900001D20FFF76DFF288448B138784EF66022CD
:106910000421FBF7AFFC02E00EB185F81E80304683
:10692000BDE8F681062200A93846FAF7E4B970B549
:1069300004460025764E2CB921B1062206F110003E
:10694000FAF7B5F9307801280BD1012524B90220D6
:106950003070FBF703FB04E000203070204600F0AD
:10696000B4F8284670BD38B50025D0B10478684A1F
:1069700034B94178837801EB0321D182C078107655
:10698000107802280DD1012534B903201070117E32
:10699000D08AFAF7DDFE01E000201070204600F0FA
:1069A00094F8284632BD10B5594CA17F81B10146FB
:1069B000062204F12400FAF77AF9A07F04F12401F9
:1069C00000F008F804F12400BDE81040FFF7F6BE1F
:1069D000002010BD0022002918BF00280ED04A79DF
:1069E000012808BF42F0C00006D002F03F02032891
:1069F0004A7102D142F040004871012210467047AE
:106A0000002918BF00280BD0487900F0C000C0282A
:106A100001D101207047402801D103207047022096
:106A2000704770B53A4D0446287FFF2815D00A20DC
:106A3000FAF78CF9060010D0D0203070747008205E
:106A4000B0700622A87FF07005F12401301DFAF71E
:106A50002EF9287F3146FAF79AF9E87F01280FD1FD
:106A60002D48006818B18068010018BF8047BDE854
:106A70007040284800784EF660220421FBF7FABBEC
:106A800070BD2348806870472148C068006870471F
:106A90001F48C1680A68521C0A60007FFF281CBF9B
:106AA0004FF48041FAF749BA70471948807F704720
:106AB000174A02F1100118B9907F08B102F12401C0
:106AC0000846704712484068704770B5104D04463C
:106AD000287FFF2819D00E20FAF738F9060014D0C5
:106AE000D020307074700020B070062205F11001C3
:106AF000F01CFAF7DCF8E88A70813146287E3073A2
:106B0000287FBDE87040FAF742B970BD14450020F7
:106B1000E84400208045002084450020DFF800F094
:106B2000259500102DE9F04104468846122740467D
:106B30004FF6FE7188421646DFF8545808D1A8690E
:106B400050B30268100027D041462046904720E00D
:106B50004FF6FF71884212D1A86938B1026810005F
:106B600004D0414620469047070005D031462046D4
:106B700000F05FFA07000FD12C706E700CE0F9F78F
:106B8000B1FF48B10078A04205D131464046FFF739
:106B9000C5FF074600E003273846BDE8F08110B581
:106BA00004462389E288A188608884B0FBF75CF9F9
:106BB00008B9022029E020880121F9F7C1FF08B9AE
:106BC000142022E02088F9F7CCFF042812D1DFF846
:106BD000C00781894FF6FF72914218BF112014D16E
:106BE0002188818161888180A188C180E1880181BB
:106BF0002189418100200290019020890090E38842
:106C0000A28861882088FBF7FBF904B010BD70B53D
:106C10000C46DFF880170978022918BF01291546AC
:106C200001D1122070BD0DB9022070BDF9F75AFFD5
:106C3000060001D1142070BD1CB1307940F0020073
:106C400030711022294606F11400FAF730F828694D
:106C50007062002070BDF8B506000C4601D102201C
:106C6000F2BD3088F9F73EFF050001D11420F2BDD6
:106C7000DFF820070078022818BF012803D0287BFE
:106C8000082802D10CB11220F2BDDFF80477786930
:106C900008B11120F2BD2C20F9F79CF9786108B9F0
:106CA0001320F2BD2C2200F079FA786931884180F6
:106CB0001C22311D001DF9F7FAFF796902200870C6
:106CC000287B7969328808280CBF012000200B1D21
:106CD000DFF8C416097801F083FE06461CB1214690
:106CE000284602F03BF80EB100F018FA3046F2BD2B
:106CF00038B504460D46F9F7F5FE08B9142032BD43
:106D00008DF8005000A9204601F062FF32BD38B571
:106D1000002298B101230624251815F8015C303DA6
:106D20000A2D0BD203FB05220A25641E6B43E4B235
:106D3000002CF1D11046BDE8344001E0022032BD04
:106D400030B505460C4685B02046F9F7CBFE08B9AC
:106D5000122019E0DFF84406854228BF022013D232
:106D60001022002100A8F9F7D4FF280A8DF80100AD
:106D70008DF80050280C8DF802002146280E8DF861
:106D8000030000A801F06FFE05B030BD2DE9F04111
:106D90008046DFF800060078022814BF0128122080
:106DA00082B00C4615461E462BD00DB9022028E0B5
:106DB0004046F9F797FE070008BF142021D0B86AB3
:106DC00008B1F9F714F91C212846F9F786FF0100EC
:106DD000B96208BF132014D0387B082809D146B106
:106DE000887E009001F112030A8A404601F0E0FF1C
:106DF00000E00020397941F004010CB141F00201BA
:106E00003971BDE8F6812DE9F0410D46F9F76AFECA
:106E100004001ED0656200F0C4F9C5B205B925783A
:106E2000666A94F805801020F9F790FF070010D0EB
:106E3000D0203870062200207870A11D0920B8707B
:106E400087F80380381DF9F732FFFE60394628467F
:106E500001E0BDE8F081BDE8F041F9F798BFF0B579
:106E6000040087B051D0A079DFF8245500282869A4
:106E70000CBF0826042608B9DFF824050778DFF8D8
:106E80002405006820B1416808001CBF0020884725
:106E9000E07904F10801FFF7B3FD217DE071059170
:106EA0000246618A049104F10803218A0391E18971
:106EB00002910196A18800913946E07800F056F8D9
:106EC000E07870B9172003900122E08902900196C2
:106ED00004F108000090E379A1883846F9F7BBFD7A
:106EE000E070286908B100F031F9287868B1697854
:106EF00000F09FF848B1E378312B04D0A2882978BC
:106F0000184600F061F80020287007B0F0BD70B599
:106F100005460026A888F9F7E5FD18B10678A88887
:106F2000F9F7C6FDDFF86844207838B1864205D10C
:106F3000617800F07EF840B1002020702EB1AB796E
:106F4000AA88A878314600F03FF8606908B100F0DF
:106F5000E5F8A888F9F705FE042802BFA888A189EA
:106F6000884204BF4FF6FF70A08170BD2DE9F0414B
:106F70000646884617461C461620F9F7E7FE050028
:106F800020D0D02028706E700520A870EF702CB132
:106F900006222146281DF9F78AFE04E00622002178
:106FA000281DF9F7B6FE06986881294607982873C8
:106FB0000898E881099828820A9868820B982875B1
:106FC000404648E7BDE8F081F8B504460D46164650
:106FD0001F460820F9F7BAFE48B1D021017044706D
:106FE000062181708680877101462846DCE0F1BD6C
:106FF0002DE9F04180460D4616461F460C20F9F754
:10700000A5FE040013D02846F9F76CFD08B9DFF897
:1070100090030078D021217084F801800721A170AD
:10702000A580E680278106996181214613E7BDE8A6
:10703000F08110B50C46F9F769FD28B12146BDE88D
:1070400010404088FFF76ABD122010BD2DE9F84FAF
:107050000746894692461C464846F9F743FD5FEAD3
:10706000000B1EBFCA4D6969002955D00A6A182055
:1070700002B134208A6A02B1143004B11C30496A6A
:1070800001B1163080B2F9F761FE060044D0182233
:1070900000F084F800F085F85FEA000808BF9BF86C
:1070A0000080D020307077700A20B070A6F804906D
:1070B00086F806A006F118076969086A38B1B76052
:1070C0003846096A00F11C071C22F9F7F0FD6969CE
:1070D000886A38B1F7603846896A00F114071422CB
:1070E000F9F7E5FD3CB13761384600F11C071C2279
:1070F0002146F9F7DCFD6869416A29B177611622FA
:10710000416A3846F9F7D3FD31465FFA88F0F9F75E
:107110003EFEBDE8F14F01E0BDE8F18F10B59C4C9B
:10712000606990B1006A08B1F8F761FF6069406A70
:1071300008B1F8F75CFF6069806A08B1F8F757FF9B
:107140006069F8F754FF0020606110BD10B5904CE5
:10715000206918B1F8F74BFF0020206110BDF8B589
:1071600004460D462846F9F7BDFC060015D000F090
:1071700018F8070008BF37780620F9F7E7FD060082
:107180000BD0062200F00AF8D020307074700E2068
:10719000B070B5803146F8B206E0F1BD0021F9F7D4
:1071A000B8BD2620FFF71CBBBDE8F440F9F7EFBDE2
:1071B0002DE9F84305460E46174698463046F9F73E
:1071C00091FC5FEA000921D01020F9F7BFFD04000F
:1071D0001CD01022FFF7E2FFFFF7E3FF08B999F890
:1071E0000000D021217065700F21A170A680277248
:1071F00084F80980C0B20899A1720999E1720A99CC
:10720000E1602146BDE8F443F9F7C1BDBDE8F18373
:107210002DE9F04107468846F9F764FC040022D0C6
:107220000E20F9F793FD05001DD0FFF7BAFF060009
:1072300008BF2678D0202870062200206870A11D83
:107240000B20A870E81CF9F732FD18F0010118BFF7
:10725000012129736F8118F0020118BF01216973A0
:10726000F0B22946F7E5BDE8F0812DE9F14F9046EF
:107270000D4699464046F9F735FC07000A9EDDF8B1
:107280002CA0DDF830B00D9C3ED09DF80000002809
:107290003AD1387940F010005FEA49714CBF40F0B4
:1072A000020000F0FD00002E08BFBAF1000F08D167
:1072B000BBF1000F08BF002C03D100F0FB003871B8
:1072C00022E040F0040038713CB12069786210225D
:1072D000214607F11400F9F7EAFC3EB135B9B86A66
:1072E00008B1F8F784FE1C2130460AE0BAF1000F1D
:1072F0000AD0012D08D1B86A08B1F8F778FE1C2130
:107300005046F9F7EAFCB862214D6869002839D087
:107310006EB1006A20B91C20F8F75CFE696908624A
:107320006869006A18B11C223146F9F7C0FCBBF14C
:10733000000F0ED06869406A20B91620F8F74AFE9F
:10734000696948626869406A18B116225946F9F7B6
:10735000AEFC74B16869806A20B91420F8F73AFE6F
:10736000696988626869806A18B114222146F9F750
:107370009EFC9DF8000053464A46414601B0BDE8D8
:10738000F04F63E6BDE8F18F0749086070470000E1
:10739000CC440020054500208045002040420F00DD
:1073A000044500208445002090480020DFF800F0CC
:1073B000B1AD0010DFF800F0F5D8001010B586B0C0
:1073C0001C460823ADF8003001901B23ADF80230B5
:1073D000039104922068DFF830160968029000A833
:1073E00088470299216006B010BD00B583B000F057
:1073F00019F88DF80400172105E000B583B000F0FE
:1074000011F801901E21ADF8021000A8DFF8F81560
:10741000096888470EBD00B583B000F003F80190FD
:107420001F21F0E70821ADF80010704700B583B0C8
:1074300000F0FAF9212000F00AF89DF804000EBDD2
:1074400080B500F0F1F9262000F001F802BDDFF868
:10745000B8150968ADF8020000A80847DFF8AC05C8
:1074600002F0C5BCDFF8A80540F6020101804FF428
:1074700001620021418041608160017301214173FB
:1074800000218173DFF88C150A8048600022DFF844
:107490007C054A808A608A8108614A61704710B51C
:1074A000DFF8740586B00021C160C1600160016031
:1074B000DFF85C45207E032805D11020FFF7ABFFE5
:1074C0000020FFF792FFFFF7B1FF0028FBD0FFF786
:1074D000B7FF00F060F940F60A0000F06AF9206B8F
:1074E0000490002000F05DF9607E012803D10020A7
:1074F000607600F05DFAFBF7EFFF2062207E012846
:1075000005D11020FFF787FF0020FFF76EFF002056
:10751000207606B00120A07610BD2DE9F843DFF8F3
:10752000FC44DFF8FC5420688047074600F080F9EF
:10753000032803D029683846884732E02968DFF8F5
:10754000D064307E012802D13846884758E00120B7
:107550003076384688470020DFF8C874DFF8C81452
:10756000DFF8C884DFF8C89470637861F86040F28F
:10757000FF700860FFF71AFF002038613861F8617A
:10758000F861EFF3118080060DD502203076DFF828
:107590007C0402F02CFC00F01CFE00F034F8FFF735
:1075A0007EFF00202DE000207080DFF88824DFF8C7
:1075B000880400883082DFF88404C06A8168127809
:1075C000096802EB42025118B1F80110718240685B
:1075D00070611020FFF711FF0120FFF706FF00F098
:1075E00012F8386860B920688047716B41B9DFF8DC
:1075F00050147163DFF81C14396029688847786873
:107600000120BDE8F28300224946404602F085BBD6
:1076100038B5EFF311808006DFF8F4431BD5A07E68
:1076200003282AD1207E012810D103202076606B08
:10763000010022D0DFF8E0130A689207FAD56FF054
:1076400003020A6080470020606316E00220207673
:10765000FFF763FF11E0DFF8C403006880470546C9
:10766000A07E032804D1207E012818BFFFF755FF14
:10767000DFF8AC13096828468847A07E0128FCD1B2
:10768000BDE8314081E138B5DFF89003DFF8B4534D
:10769000006880470446287820B10020FFF7A5FE47
:1076A000002028702046BDE83440DFF874130968D4
:1076B0000847DFF87403016821F0020141F400710A
:1076C00001600321DFF88003816041F230014161F4
:1076D0000121C160502141610121C1604FF4CA61A3
:1076E00041610121C16001607047F0B500F087F988
:1076F000CB4E85B08047044600206863A87E0328EF
:1077000044D0FBF7E9FE296AFFF754FEE969401807
:10771000696AE861814208D3CC480088B0F5006FFF
:107720001CBF40F20241884224D12F6B02F020FBA3
:107730000020E86100F02FF840F6090000F039F869
:1077400000F02FF80498696A286387422CBF381A22
:10775000C01B0328A7BFBE48401801F59C4020303D
:107760000028BC4948BF0020884268620ADBBA484A
:10777000686207E0B9480021C160416081608160B2
:1077800001600160FFF795FF0320A876204631686D
:10779000884705B0F0BDB248016841F002010160C0
:1077A00070478DF80C0001208DF80D0000A802F044
:1077B0002FBBADF800000020ADF802000190029050
:1077C00070473EB502F0D4FAA649012008604FF494
:1077D0004220FFF712FE00F0D8F8FFF743FEFFF754
:1077E00025FE0028FBD0A04D894CFFF729FE2D680F
:1077F0000FF26111642004F12C030022B0FBF5F0BC
:10780000FFF7DCFD00F010F81820ADF802007E490B
:107810000FF265100968019004F13800029000A889
:1078200088470320A07637BD0820ADF800007047D8
:1078300010B57A480068804775498C7E7849096898
:107840008847204610BDFEB50446714D6068002192
:10785000A962017B01F00F0102294CD18068A06070
:1078600040F61D47814800780938052832D3FBF7D8
:107870003FFE06001CBFB068002835D0FBF72CFE89
:107880000146B068FFF796FDA0F5C871784A9142AD
:1078900020D28608BE421FD3FFF7C6FF2720ADF8CF
:1078A00002004FF47A70B6FBF0F000F04DF8029849
:1078B0000FF2A101301A6F4EF668C838801B6A4E6D
:1078C000366805F12C030022B0FBF6F0FFF776FDD9
:1078D000AC6209E0642600E036B1606802F087FA25
:1078E00000F053F8BE4214D3FFF7A2FF032810D0D4
:1078F000FFF7C9FEF7BDFFF79BFF032808BFFFF79F
:1079000087FEFBF7E9FDA060606802F070FA00F006
:107910003CF8F7BD30B505464048006883B0804765
:1079200004463B48816AA94207D1FFF77BFD1C2131
:10793000ADF80210C06A00F007F800F001F837BD9A
:1079400037490968204608472F490968019000A86F
:107950000847704700B583B0FFF766FF2220FFF7A6
:1079600076FD00280CBF01980020032814BF0128D1
:1079700000F028F807BD0000052808BFFFF7CDBDBF
:10798000022808BFFFF7B1BE704738B52348244D21
:107990000068804704462B48017821B90121017015
:1079A0000120FFF722FD29682046BDE83440084742
:1079B00080B5FBF79DFD20B1BDE80240406802F0B4
:1079C00016BA01BD38B5FBF793FDB8B100F017F852
:1079D0008047044601206876FFF72AFF032808D075
:1079E00000200F496876204609688847FFF7E0FFC6
:1079F00001E0FFF7A5FFBDE83140C6E731BD07480C
:107A0000034D0068704700003048002001010E045B
:107A100058460020F8470020101004403448002049
:107A2000384800200010044000000460020000807C
:107A300000048000B94C0020944C0020A4C8010030
:107A40009F740100B6480020004104400A4F002006
:107A5000E0B1FFFF01350C0000350C0008100440B8
:107A600000200940D02108403C440020B84C0020B0
:107A7000711EA1073C46002080B54FF48030FFF70F
:107A8000BCFCBDE80140FBF747BD4FF48030C2E4C9
:107A900080B54FF480710122084602F03FFA104889
:107AA000016841F48061016000200E49086001BD59
:107AB00010B50D4CE068400558BFFFF7E9FF20689E
:107AC000C007FCD50949096849680220884705496B
:107AD0000A6890420CBF0648086010BD0000000014
:107AE000148002408048002008800240CC01001031
:107AF000EFBEADDEDFF800F06D550010DFF800F0EE
:107B000019870010DFF800F049550010DFF800F089
:107B100065B90010DFF800F029840010DFF800F0EC
:107B2000C9D80010DFF800F0F57D00102DE9F8430A
:107B3000099D002600274FF6FF7835F81740444589
:107B40001CBF761CF6B27F1C062FF6DB00270DE06B
:107B50000CF1010C5FFA8CFCE646B64505DA35F807
:107B6000179035F81EE0F145F2D1E7B2B74208DAD6
:107B700035F81740444504D0A14202D37C1CA446EA
:107B8000E8E7B7420DD176B1884202D04BB19942B5
:107B900007D308981146FFF7B1FF47F6FF718842F7
:107BA00001DB012000E00020BDE8F2832DE9F8436D
:107BB000DFF86C08DFF86C98017899F800008842CB
:107BC00000F07F8000204FF4907301E0401CC0B2B1
:107BD000884276DAD9F8042003FB002808F104066D
:107BE0003278002AF2D1DFF840180968B0703822E4
:107BF00002FB00110122327008F16107002272704D
:107C000001207871F872B280F280307388F83920E0
:107C100008F18E0072613276728302702031FA7739
:107C20000A75FF258022FA7408F1E80400227A75AB
:107C3000BA760D706276A276E2762277E2832284AB
:107C400088F80B21027108F1E30002704270226093
:107C50006260A2722273227208F5877062730280DA
:107C600042808280C2800A720A734A738A73CA731E
:107C70000A744A740421FF2208F17700FAF778FAAF
:107C80003D707D70BD70FD701F2038710020DFF8E1
:107C90009C17421800EB0803527883F8F920401C27
:107CA0000828F6DB0020207499F80000401C89F8B1
:107CB0000000C0B2012804BFB07889F80200404635
:107CC00000E00020BDE8F28310B5DFF8604708212E
:107CD000601C02F03DF9607840F00100607010BD5A
:107CE00070B504460920FFF70DFF58B300F089FB7B
:107CF0000A30C0B2E880002105F108062960297128
:107D00006971032030700822092006F8010F04F180
:107D1000F901701CF8F7CBFF94F8920028B13346B4
:107D2000092203212046FFF7F1FEFFF781FDDFF86E
:107D300000371B69DB6C0246A06E2946984700207D
:107D4000E083012070BDF8B505460E46DFF8E44635
:107D5000DFF8DC7608E0007A03281CBF481C20709E
:107D60003969A86E496D88473969A86E096E8847D8
:107D7000217810B10279032AEDD0DFF8BC06007833
:107D80001C2814DA99B1DFF8B4060078814205D2D4
:107D9000012E0CD1DFF8A806007840B1A879ADF823
:107DA0000000ADF8021000F069F800202070F1BD6D
:107DB0002DE9F8430446DFF88C06DFF878660068A2
:107DC000DFF86C76804780460020FFF7A3FDA06EA9
:107DD00000B306E0007A00F057F83969A06E496DEB
:107DE00088473969A06E096E88470028F2D1396941
:107DF000A06E496E8847054606E0287A00F044F8F0
:107E00002846F9F7CAFD2D68002DF6D13969A06E14
:107E1000096D8847206FA0B13969096E884705460A
:107E2000A946D9F8080020B1F9F7B7FD0020C9F834
:107E30000800D9F80090A945F3D13969206F096D80
:107E40008847DFF8F40500781C2808DA307840B15C
:107E5000A179ADF80010ADF8020000F00FF8002095
:107E600030702046FFF756FE2046FBF789FBDFF80F
:107E7000D815096840468847BDE8F1830DF1020234
:107E800000A90120FCF7F4BA032802D03078401C86
:107E90003070704770B50446DFF8A8050068804769
:107EA00004F17601FF234A79521E4A71D2B20AB90F
:107EB0004B7008E0002215197735521C6E782E7031
:107EC000032AF8DB0B7100220A70BDE8704011E054
:107ED00038B50446DFF86C0500680D46804700227F
:107EE00004F176010A704D704A790AB901224A718B
:107EF000BDE83440DFF85015096808472DE9F04126
:107F000000260027DFF81C45DFF8148508E03168FB
:107F1000496880688968FFF701FE00B92E467F1C1A
:107F200098F80000FFB287420CD260684FF490715D
:107F300001FB07052868697940680029EFD0002E09
:107F4000E5D1EBE7B079BDE8F081F0B54FF6FF7110
:107F50000C460023DFF8CC2403E0A64298BF344649
:107F60005B1CDFF8BC542D78DBB2AB4216D25568EF
:107F70004FF4907606FB03556E79002EF0D005F194
:107F800080068C42377804D1002F0CBF6C8E348968
:107F9000E6E7002F14BF36896E8EDEE7A04288BF69
:107FA0002046F0BD2DE9F8430446884616460027D2
:107FB0000FE02A464146F8F77AFE3846471CC3B21E
:107FC00003B101232A4649462046FBF7BDFAA844DF
:107FD000761BB6B276B11C2EACBF1B25F5B2284677
:107FE000FAF758FC5FEA0009E3D18120FBF788FA31
:107FF000072000E00020BDE8F2832DE9F04DDFF816
:108000002474DFF84864DFF848A40C461546796804
:108010004FF4907282B002FB0018307801289B4622
:1080200002D0022830D068E0B068BBF1020F04D162
:1080300000F070F80020B06029E07388B188EA1879
:10804000914205DA00F066F80020B0608B2052E023
:108050002A4621461818F8F72AFE708828187080DA
:1080600080B2B288904248D198F87400802817BF37
:1080700081287F209AF80010401A00F043F8002071
:10808000B0807080022033E0BBF1020F35D1042DA7
:10809000B8BF8C202FDB21786078091D41EA0020D1
:1080A000DFF89413B08080B20978814238BF8A200B
:1080B00021D3A84238BF8B201DD3FFF71BFDB06032
:1080C000C0B12A462146F8F7F2FDB28895420BD19D
:1080D00098F87400802817BF81287F209AF8001034
:1080E000401A00F00FF808E070882818708001200E
:1080F000307002E08120FBF703FA2046BDE8F64D20
:10810000F9F74BBC40B200905B46B168B878D2B288
:1081100001F026BF0021B180718002213170F9F792
:108120003CBC2DE9F84304462068007840284ED135
:10813000E08B00284BD0C7480078012847D1FFF7D3
:1081400067FAC048006880470546FBF7C5F9618EAD
:1081500040F6C418891C08FB0109B24A2068A179BD
:108160009278476891422CD1B8684946FFF7D6FC0F
:1081700048B3FBF7BDF9064640F20240FBF7C4F9ED
:108180003046FFF7C7FB31694846FFF713F9618EA8
:1081900008FB01F2B0FBF2F0228980B28218628102
:1081A00048432268126908FB0020B86004F13800D7
:1081B00041780170204600F0BAF8304600F0E6F948
:1081C00001E00069B8602846BDE8F44392E6BDE8E6
:1081D000F18330B587B040F60200ADF80000002012
:1081E000ADF8020001900290ADF80C0001208DF86E
:1081F0000D000020ADF80E00974C984D2088984A4D
:108200001278ADF8100002EB4202E86A8168096852
:108210005118B1F80110ADF812108549406809698C
:10822000059000A8C9698847012807BFBDF802006A
:10823000B0F5806F892000F0EBF8E868894A418842
:1082400012781143218000788149800643BF864817
:108250000068400A0020087007B030BD10B582B039
:1082600004461020ADF8000004EB44017B48C06ACE
:108270008068006808186E49B0F801000969ADF817
:10828000020000A8896988477548047013BD7348C7
:108290007349C06A80680978006801EB410108569B
:1082A000704730B50A7902F01F020A71002280F887
:1082B0003A200023545C24FA03F5EC070BD590F820
:1082C0003A502D1803EBC20485F83C4090F83A4030
:1082D000641C80F83A405B1C082BEBDB521C052A1F
:1082E000E7DB30BD10B500F138025378D47801FBDC
:1082F0000431252391FBF3F3252404FB13111170A2
:108300000023117800E05B1C9478DBB2A34206D214
:108310001C1894F83C40A142F5D1084610BD91FBD1
:10832000F4F204FB1211081890F83C0010BD70B56F
:10833000044604F1380004F18E060178417060892A
:108340002189FFF7DBFB05463078012801BF7088E3
:108350002189491C884206D104F161012046FFF7BA
:10836000A0FF0020307029462046FFF7BBFF2168A0
:108370000978402904BF3D49887370BD80B580F8F5
:10838000F120FFF7CFFB38B939480078BDE8044049
:108390004FF48041F8F7D1BD01BD70B5044602200D
:1083A000FFF7B0FB60B300F02CF8C01CC0B2E8804F
:1083B000002105F1080329602971697103201870F3
:1083C000022003F8010F94F80C01587094F8920001
:1083D00020B1022203212046FFF798FBFFF728FA7D
:1083E000134B1B69DB6C04F16806024630682946B2
:1083F000984704F10E00002101820088F0820120DC
:1084000070BDA0F1090594F8920000B104207047F6
:1084100080B5FBF775F817490020087001BD000012
:10842000BC4C0020B04C002014480020D04E00204E
:108430002C4F0020BA4C002010480020874C002010
:10844000884C002034480020384800209446002002
:10845000C04C0020BB4C0020944C0020A4C801005C
:10846000B94C00201148002080130050E04D00203E
:10847000844C0020B84C002070B50021FF224A48EF
:108480004A4B09E0182486684C43A61900257570EC
:10849000491C85686255C9B21C78A41CA142F1DB55
:1084A000002182700180416070BD10B500233E4AFA
:1084B0009168182404FB03114C78D4B90C78FF2C74
:1084C00002D05468A14214D0087000234B604B6165
:1084D00001234B7053780343537013785B1C137064
:1084E000DBB2012B1CBF8028402800D15160084618
:1084F00010BD2E4909785B1CDBB2891C8B42D7DB8F
:10850000002010BD10B5284A9268002118234B4363
:108510009C5C844202D19818407810BD00F017F896
:10852000F4DB002010BD10B51F4A9268002118230B
:108530004B439C5C844202BF9B185B78012B01D1AA
:10854000012010BD00F003F8F1DB002010BD174B37
:108550001B78491CC9B29B1C9942704710B512493F
:108560008B68002218215143CC5C844202BFC91899
:108570004C78012C01D1084610BD0C490978521CD9
:10858000D2B2891C8A42EDDB002010BD10B5044632
:10859000054844606069010018BF80472046BDE877
:1085A0001040FFF750B90000F44E0020BC4C0020F2
:1085B000DFF800F0D9890010DFF800F0EDB400100A
:1085C000DFF800F041B50010DFF800F055B50010FD
:1085D000DFF800F009B000102DE9F84F8B46D349C1
:1085E0000968804608F10604382322781BF8010B3D
:1085F00003FB021101F120090C2808F1E30708F13F
:10860000660608F2031547F6FF7AC94900F21181A0
:10861000DFE810F00D00520009016F000F010F019B
:10862000CD001601DD00EC00D000DA00F1001BF8EF
:10863000010BB0770222594608F18600FFF7B8FF18
:108640000146022208F18800FFF7B2FF014602222C
:1086500008F18A00FFF7ACFF0146022208F18C0006
:10866000FFF7A6FF0146B07F4000B0770222308CB2
:1086700040003084708C40007084F08C0001F084E5
:1086800008F18200FFF794FFB08B6188401A80B236
:10869000504525DAB08C718C401C49004843F18C60
:1086A000884228BF3B201CD20120B07600202083C6
:1086B000012089F81400C3E00522594608F1610041
:1086C000FFF776FF0146022208F19000FFF770FFE6
:1086D00008F18E0062884188891A89B2514501DB10
:1086E0002820A2E0012101700020208389F81410C5
:1086F000A6E0B87DC00708D41A20B873787B01289B
:1087000008BF0D213AD00D2195E000203070B071E6
:10871000082201207874594608F1AC00FFF748FFA1
:108720000146022208F1B400FFF742FF08F1A40459
:10873000014608222046FFF73BFF05460821204658
:10874000FFF73AFF08F19804042229462046FFF774
:108750002FFF04212046FFF72FFF08F19C00FFF7B1
:108760002FFF08F19400FFF72FFF7248018841F0B6
:1087700080010180787B012805D104214046BDE8B5
:10878000F44FFFF7A5BB307C012804BF707C0F2895
:108790000BD14046FFF77EFB04214046FAF7CCFEA2
:1087A0000F2089F80000FD2145E0042143E001206D
:1087B000F87345E000203070B07138700B21012053
:1087C00078730020787036E00120387438E000F0CB
:1087D00039F84046FFF784FA002831D1BDE8F44F5C
:1087E000554800784FF48041F8F7A7BB00F02AF80D
:1087F0000220787524E0B97F01291AD01BF8010BFB
:1088000068700222594608F58370FFF7D1FE0146D1
:10881000022208F58470FFF7CBFE0120B877287894
:1088200070B90C2107E09BF80000687201202872E3
:1088300006E0A87207214046BDE8F44FFAF77CBE77
:10884000BDE8F18F0020421810F80B3052781A4022
:1088500000EB0803401C082883F8F920F3DB70477D
:108860002DE9F0413548364F0068364C8047804648
:10887000002500260EE078684FF4907101FB060099
:108880004179012904D1806EFFF7A2FE4519EDB2AE
:10889000761CF6B220788642EDDB2B49096840460B
:1088A00088472846BDE8F0812DE9F0478146302011
:1088B000002500FB09FA254F254C4FF00C082068D5
:1088C00008FB05F650443018002101710221206890
:1088D000504430184171796920684A7850443318FF
:1088E0002132DA806A1C531002EB93739B10A2EBC7
:1088F000830208FB0202325048781F3080B2FFF733
:10890000F9F8216851447218906008B1801E906097
:108910006D1C042DD3DB0F48006800EB091000220A
:10892000016042608160C260BDE8F08714480020A9
:10893000D04E0020BE4C0020844C00203448002043
:10894000B04C0020BC4C002038480020A4C80100D6
:10895000104F00200C4F002070470000FAF79FBA1C
:10896000004805E098480020004801E094480020B5
:10897000006800B101207047010001D0172801DB19
:10898000FF2801D101207047002070472DE9F84FE2
:108990000D4693460024BBF1200F80461F462C70E5
:1089A00003DB0020BDE8F28F0419E4B25C45F8D285
:1089B000E65D641C002EF4D0E4B231198B45F0DB87
:1089C00014F807A05046FFF7D7FF641C0028E8D032
:1089D000701EC2452870E7D1E4B2E019E2E700005A
:1089E0002DE9F843DFF80457044628688946904685
:1089F0001E46002708B1112033E05EB12120FDF7AB
:108A0000EFFE317E814205D32220FDF7E9FE317E63
:108A1000884201D2022024E07820F7F7DBFA2860B0
:108A200008B913201DE078220021F8F772F92968AF
:108A30004F7028680470286880F802902868011D2B
:108A4000A1F800804E60CF6180F8247014B100F06E
:108A5000BCF907462968012048700FB100F0DCFA24
:108A60003846BDE8F28338B5DFF880562B6800241D
:108A700033B193F82420022A1CBF032A042A01D010
:108A8000122032BD9A888A4201D0022032BD0146AE
:108A9000102203F10C00F8F70AF92868102135308C
:108AA000FAF719FB286800F1250200F135010C30B6
:108AB00000F009F92868417802781AB103290DD12C
:108AC000022107E0042902D10221417006E00329B6
:108AD00004D10521417000F08EF90446204632BDD4
:108AE000DFF8081648607047DFF80026126832B1D8
:108AF0009288824203D1012908BF00F08DBA7047E5
:108B00001720AEE270B586B0044600208DF8000054
:108B1000A0680578691E0A2939D8DFE801F0060641
:108B20000D1115191D2125292D0001A901F0C7FAE4
:108B3000122824D106202BE001A901F033FB1EE00E
:108B400001A901F04BFB1AE001A901F05EFB16E060
:108B500001A901F072FB12E001A901F08BFB0EE00C
:108B600001A901F0B1FB0AE001A901F0B8FB06E0A0
:108B700001A901F0CBFB02E001A901F0E0FBD8B9AB
:108B80006088F7F7AFFF072628B9082612E007200C
:108B90008DF8000013E0027BDFF85015082A0CBFA7
:108BA0008968496831B10B68190003D001AA2946C8
:108BB000984706468DF800609DF8000020B1608857
:108BC00000A900F005F801E0FAF7C5F906B070BD9C
:108BD00038B50C46DFF818352246022101F0BDFBFE
:108BE0000546207800F03DFA284632BD70B5DFF822
:108BF000FC440546206800280E463DD08188A942E5
:108C00003AD1417806292FD1017809B381684969A1
:108C1000026ACB0704D5137BDB0748BF072113D4B7
:108C2000C1F34003002B1FBFD368C3F34003002BE5
:108C3000092109D1C1F3800100291EBFD168C1F308
:108C40008001002902D00B21417007E0A06800E0FC
:108C5000606818B14068010018BF804720684078FC
:108C6000122816D1002004E0112905D106B13226C0
:108C7000304600F0F6F90CE03EB92846F7F732FF2F
:108C800018B1017941F01001017129463046FEF713
:108C900066FA012070BD10B5DFF85044206888B135
:108CA000007800280CBF6068A06818B14068010017
:108CB00018BF804720684078122803D1BDE81040D3
:108CC0000020CEE110BD2DE9F34FDFF820643068BD
:108CD0008DB0904608B912203DE08088F7F702FF7A
:108CE000050008BF142036D009A800F0E2F930686A
:108CF000017871B1D0F82090FDF7D7FE044600202E
:108D0000FDF7D6FE95F805A009AE074605F1060B5E
:108D10000BE0066AFDF7C9FE82460020FDF7C8FE9B
:108D20006C790DF124098346AF1D07A9484601F06F
:108D30006FF905A9304601F067F9CDF81080CDF83C
:108D40000CB0CDF808A0019700940E990D9805ABD2
:108D500007AAFAF739F90FB0BDE8F08F70B5DFF860
:108D60008C530446686886B000281CBF0068002841
:108D70000E461BD030788DF8040070788DF8050011
:108D800002A8B178FAF7CAF9F0786B688DF80C0090
:108D900001AA7068049001211B682046984728B1F9
:108DA0008DF8000000A96088FFF712FF06B070BDC3
:108DB00038B5CE4CA46834B1A5682C0003D0049C0F
:108DC0000094A84732BD022032BD1FB500F031F833
:108DD00070B100A800F06DF9216888880978002931
:108DE00014BFC44BC44B00AA072101F0B6FA00E03F
:108DF000012004B010BD1FB500F01BF800F12501E3
:108E0000102200A8F7F753FF2068BC4B0AE01FB5FB
:108E100000F00FF800F13501102200A8F7F747FF26
:108E20002068B74B808800AA112101F096FA04B09F
:108E300010BDAE4C20687047F8B5AC4F044638689A
:108E4000006A0025002840F0AD801020F7F7C2F836
:108E500039680028086200F0A3808E68102221463D
:108E6000F7F725FF38680178002973D1026A12F8F4
:108E70000CCF06F114010CF0010C0B6803F0010794
:108E8000674518BF00275B0847EA43030B605F088C
:108E9000D2F800C04FEA5C0C00F087F818BF00273A
:108EA00023F0020343EA47030B609F08D2F800C097
:108EB0004FEA9C0C00F079F818BF002723F0040358
:108EC00043EA87030B60DF08D2F800C04FEADC0CEE
:108ED00000F06BF818BF002723F0080343EAC7032C
:108EE0000B601F0AD2F800C04FEA1C2C00F05DF89E
:108EF00018BF002723F4807343EA07230B605F0A3F
:108F0000D2F800C04FEA5C2C00F04FF818BF0027E1
:108F100023F4007343EA47230B609F0AD2F800C092
:108F20004FEA9C2C00F041F818BF002723F480631F
:108F300043EA87230B60DF0A1268D20A07F00107B1
:108F400002F00102974218BF002723F4006242EAB0
:108F5000C7220A60617800291EBF717800290521A7
:108F600019D16168C1F3800121B9B17C490758BFAB
:108F7000012110D50178002919BF31782278327883
:108F800021780529B8BF052A08DA0FF28C1302EB05
:108F90008202D218895C2030017104E0182502E0B9
:108FA000132500E011252846F2BD07F001070CF05B
:108FB000010C674570470A46524B15E010B586B064
:108FC0000446ADF800101046014608220DF10200DB
:108FD000F7F76DFE4C4B00AA0B21204601F0BDF9BE
:108FE00006B010BD0A46494B112101F0B6B91CB5B7
:108FF0008DF8001004461046014606220DF10100CE
:10900000F7F755FE424B00AA0821204601F0A5F9CA
:1090100013BD0A463F4BE7E710B5FFF70AFFE0B183
:10902000006A08B1F6F7E3FF2068806E08B1F6F732
:10903000DEFF2068C06E08B1F6F7D9FF2068006F28
:1090400008B1F6F7D4FF2068406F08B1F6F7CFFFFC
:109050002068F6F7CCFF00202060BDE81040F9F74B
:1090600088BF224900B5096885B081B14A6F039273
:109070000A6F0292CA6E01928A6E00920B7F8A88F2
:109080000978FEF7F2F805B05DF804EBC4E705B027
:1090900000BD16490968102000291CBF0A6A002A71
:1090A00006D0896821B1087E117A814238BF08460E
:1090B000704738B504460D48006800281CBF856815
:1090C000002D0CD02878207068786070201DA97C55
:1090D000FAF724F8287E20726869E06031BD2046E6
:1090E000BDE8384010220021F7F713BE3C480020AD
:1090F000F3A1010009A0010011A0010093A101004A
:10910000BBA1010029A2010051A2010099A2010006
:10911000ABA20100FBA20100010102010201010258
:109120000102030304010301010101010303020120
:109130000300000038B504460D46F7F7D3FC98B19C
:10914000007B042801D0122032BD3648006800B1EF
:10915000857D294600A8F9F7E1FF334B00AA0221DB
:10916000204601F0FAF832BD142032BD80B52F48F8
:109170000078400707D52E48FEF706F92D494FF62F
:10918000FF70088001BDBDE802400020FEF7FCB87A
:109190007CB5012403280E4610D042F21301884208
:1091A00004D04FF6FF7188421ED02AE0B0780C2818
:1091B00018BF112826D100F027F823E0F078B188F5
:1091C0001C4D1A2804BF2A889142F4D0728900925B
:1091D0003389F288FDF70CFFB0882988884211D1C5
:1091E0004FF6FF7028800DE070790024122809D115
:1091F000ADF800403179708800AAF8F76BFA0124C5
:1092000000E00024204676BD38B50A4C20884FF691
:10921000FF75A84205D008490A780849F8F761FAAD
:10922000258031BDE044002023A301000545002036
:109230008C450020D844002080450020D0440020E8
:10924000F8B5144600250E46AD4FAE4B40B101288F
:1092500015D0042818D006281ED0072822D02CE0CC
:10926000162928DA1622002107F10C00F7F751FD24
:109270003246214607F10C00F7F719FD1EE0022ED9
:1092800019D12088388119E0082E14D1384621469A
:10929000082201F087F811E0012E0CD1DA6903F100
:1092A000280104E0012E06D1DA6B03F14801207891
:1092B00000F02DF802E0182500E002252846F2BD56
:1092C00010B50B4600248E4920B1012808D004288F
:1092D00009D00DE015220C311846F7F7E8FC08E03C
:1092E0000889188005E01846082201F05BF800E0C4
:1092F0000224204610BD01460020C90706D50FF202
:109300001C23804810220721F5F7DCBE704710B5FA
:109310000B7884074CBF43F0020303F0FD030406FF
:109320004CBF43F0800303F07F0304074CBF43F0BE
:10933000080303F0F70384064CBF43F0200303F057
:10934000DF030B70AA21084203D0107840F00C0014
:1093500003E018B9107800F0F300107010BDF8B5F4
:1093600006980F4614461D46002608B10B20F2BD94
:109370003878022849D178680178407800F0C6F83A
:1093800008D0401E10D0401E1ED0401E14D0401EDB
:1093900020D03AE0F868F7F788FC079A80B282425A
:1093A00088BF02462A800AE0F868008802212980E6
:1093B0002070000A60702AE0062028800622F968E2
:1093C0002046F7F774FC22E001202880F868007836
:1093D00020701CE0F868B0B1082129800188217054
:1093E0000188090A61704188A1704188090AE17009
:1093F000818821718188090A6171C188A171C08841
:10940000000AE07103E0288001E02E80012630464A
:10941000F2BD2DE9FC4B0E4680463078002702282D
:1094200091461D4667D17068017840780A9CDFF844
:10943000D8B000F06BF806D0401E29D0401E4CD0AA
:10944000401E38D057E0F068F7F72FFC80B2A042FA
:1094500004D32919162903DB0D274DE007274BE01C
:10946000F3682A464946E018F7F721FC2C19F06802
:10947000A4B2C4F1160200212018F7F74AFCDBF869
:109480000000002838D00268100035D0002121E00B
:109490007CBB022DE0D199F8000099F8011000EB97
:1094A0000120F1680880DBF8000028B30268100092
:1094B00022D001210EE0E4B9062DCDD1F0680622BC
:1094C0004946F7F7F4FBDBF80000A8B1026810008A
:1094D00012D00321404690470EE054B9012DBBD174
:1094E00099F80000002813BF0128F1680870802750
:1094F00002E00B2700E001273846BDE8F68B0000AC
:10950000A8450020CC450020A448002001EB002005
:1095100080B24FF42851401A704700005F93010059
:10952000139401000000000038B50225012918BF7E
:1095300004291C460ED1FDF75CF905000AD1059AF5
:1095400004992046FDF769F900F008F9FFF70EFECF
:1095500000F06CFF284632BDDFF800F0A198001043
:10956000DFF800F0BD980010DFF800F0D998001087
:10957000DFF800F06D98001070B5DFF85066054612
:1095800030680C4608B1112070BD00F0CDF813D042
:10959000DFF83C16896800291CBF0978002901D131
:1095A000102070BDC00702D4FBF7F9F930B1207864
:1095B000032818BF022801D0122070BD0C20F6F736
:1095C00009FD306020B305700021306841700A2227
:1095D0002146801CF7F76BFB00F022F9040002D053
:1095E00000F0D8FA15E0DFF8EC050078032810D178
:1095F0001D20FDF7F5F8DFF8E015088048B1DFF829
:10960000DC0500784EF660220421F8F733FE00E016
:109610001324204670BDF8B50C46DFF8C415097850
:109620001546052211421E462AD001F005012143AC
:1096300026D0012CDFF8981502D18F6807B301E01E
:10964000CF68EFB1202D01DA15B10EB90220F2BDBD
:1096500008701F220021781CF7F75BFB2A46314671
:10966000781CF7F724FB3D70284624B1791CBDE82F
:10967000F440FFF771BF791CBDE8F440FFF770BFFD
:109680001220F2BD38B5DFF84445216809B912202F
:1096900032BD0978814201D0032032BDDFF83C554C
:1096A00028780221F8F702FEDFF83815002008803C
:1096B00004212878F8F7FAFDDFF81C15002008804F
:1096C0000320216848700020BDE83240FFF74CBFFE
:1096D00010B5044600F028F882B001D1122016BD62
:1096E0001CB12078FFF748F908B9022016BD607850
:1096F000801C202812DA207800F0ACF908B118207C
:1097000016BD00A90DF1010000F0B1F99DF80000AF
:1097100030B161780818801C202801DB0B2016BDB1
:10972000204600F064F916BDDFF8B4040078052186
:1097300008427047DFF8A81409780522114218BFC3
:1097400000F06FB900207047DFF89404007805211D
:10975000084218BF00F0A6B91220704770B5DFF8B4
:109760007044A06818B1F6F742FC0020A060E068E1
:1097700018B1F6F73CFC0020E0600521DFF86054EA
:10978000287808421CD004F11000FBF7C4F92878AF
:1097900000260521084211D000F0DDF9A06060B17B
:1097A00000F013F800F0D7F9E06010B100F00DF808
:1097B00004E0A068F6F71BFCA6601326304670BDD7
:1097C0000020FBF7A8F9002070BD20220021F7F748
:1097D000A0BA10B58188012442F20603CA1A05D046
:1097E000921E012A0DD9921E05D016E080680078DD
:1097F00000F054F803E08068007800F060F8044658
:109800000CE0806842F20802914201780CBF01220C
:109810000022104600F09EF800E00024204610BD13
:109820002DE9FF41DFF8A443206898B38578FBF762
:10983000B6F828B10A20FCF7D3FF06460B200DE04E
:1098400000F0B1F928B10620FCF7CAFF0646072050
:1098500004E00820FCF7C4FF06460920FCF7C0FF1F
:109860008046DFF87003077807B101272068011DE3
:10987000C078FDF7AFF82168CA7A03923B468A7A2E
:109880000292091D019100902A4641463046FFF799
:109890006FFE00E0012004B0BDE8F08180B5DFF884
:1098A0002C13096849B118B901204870FFF75CFE14
:1098B00008B100F053F9012002BD002002BD2DE9DE
:1098C000F041C24D80462868002841D04078C64EFD
:1098D00001282DD100F067F9C04FA0B10120FCF79D
:1098E0007FFF0446422C0AD338784EF660220221CC
:1098F000F8F7C0FCBB49A4F13C0008800CE04FF431
:109900007A70444302E0FCF76BFF044624B13878D8
:1099100022460221F8F79FFC29680220487030781F
:1099200018B9404600F01AF911E0002030700EE03E
:10993000307860B90320F7F709FA30B1D02101700F
:1099400080F80180042100F01FF900F023F90120C4
:10995000BDE8F08170B59E4E04463078FF280D4674
:109960000FD00420F7F7F2F958B1D02101704570FB
:1099700002218170C47001463078BDE87040F7F76D
:1099800006BA70BD38B501469048944D02682878F3
:10999000944C01291DD1218811B1934B1B7823B11F
:1099A00022B3BDE8324010786CE63C29A8BFA1F193
:1099B0003C000CDA0221F8F779FC20884FF47A7128
:1099C00001FB00F228780221F8F745FC00202080F6
:1099D00031BD5AB182490978490707D50221F8F704
:1099E00065FC00202080BDE83140D3E031BD38B5B2
:1099F00004460820F6F7EEFA050010D00822FFF71B
:109A0000E5FE7348416831B100E00146086800286E
:109A1000FBD10D6000E045606C60002032BD13207A
:109A200032BD10B56A4B5968002201E00A46096848
:109A300071B14C6824788442F8D14C680868002AD7
:109A400014BF106058600846F6F7D1FA204610BDE2
:109A5000002010BD5E49496800E0096829B14A68E4
:109A600012788242F9D1084670470020704770B5DD
:109A7000002202700A70564B5B6803E0AD1C2C1983
:109A800004701B686BB15C6865782AB904782E197C
:109A9000B61C202EF2DB01220C78AD1C2C190C70A8
:109AA000EFE770BDF8B54E48007800240521084264
:109AB00001D11220F2BD464DA86810B900F04BF854
:109AC000A860E86810B900F046F8E860A8680028C7
:109AD0001CBFE968002901D11320F2BDFFF775FE14
:109AE000E86820222146F7F714F96E6812E09B1C03
:109AF00088185918401C117071684978491C017008
:109B0000716809784170801C71684A784968F7F774
:109B1000CEF836689EB144B9AA6870681178437867
:109B20005F18BF1C202FE2DB01247368E9685B78B3
:109B30000A789B1C50189A18401C0A70DCE7AA6827
:109B40001078511CFFF708FDE868411C0078FFF70A
:109B500007FD0020F2BD2020F6F73CBA38B51B4DBA
:109B60000446286878B10320F7F7F0F828B1D0212F
:109B700001704470032100F007F8002C1CBFBDE801
:109B8000314000F007B831BD817001462868007887
:109B9000F7F7FDB810B50D4C206818B1F6F727FAA5
:109BA0000020206010BD80B50948806858B1027857
:109BB000431C00A90120FEF7E9FE20B10078C00790
:109BC00001D5012002BD002002BD00009848002000
:109BD00064450020064500200845002080450020FF
:109BE00005450020AC48002007450020006801071B
:109BF00001D50420704700F00300704770B514468B
:109C00001D4600F01CF8064608480068804703E03F
:109C100016F8011B04F8011B29464D1E89B20029C4
:109C2000F6D1BDE870400249096808473448002071
:109C3000384800200B460146184600F010B81D2297
:109C400090FBF2F21D2303FB120001F5E83101EB5A
:109C50000030704780B508490968496905E080B55A
:109C6000054B1B689B69984700E08847034A002121
:109C7000116002BD00000000A801001084046042D1
:109C800000B583B00821ADF8001001900D2106E069
:109C900000B583B00821ADF8001001900E21ADF899
:109CA000021068469349096888470EBD00B585B023
:109CB00008230291ADF8003028238E4909680190ED
:109CC000ADF8023003926846884705B000BD10B574
:109CD000894C20698068804700208849002241F82B
:109CE0002020401C0428FADB2069016B802212200E
:109CF000FFF7DCFF2069C16A80221920FFF7D6FF39
:109D00002069416B80221A20FFF7D0FF2069816A09
:109D1000BDE8104080221B20C8E7F8B5044678480B
:109D200000680D46164680470746734800698068FC
:109D300080477448C168A143C16045EA0402C16814
:109D40002943C1608168114381600168314301602A
:109D50001B20FFF795FF1920FFF792FF1220FFF756
:109D60008FFF1A20FFF78CFF3846BDE8F4403BE038
:109D700010B500F07FF804461920FFF789FF122084
:109D8000FFF786FF1A20FFF783FF1B20FFF780FFF6
:109D90005D480021C16041608160816001600160B7
:109DA00020465A490968BDE81040084780B500F0D0
:109DB00061F8554900228A608A607CE038B5044623
:109DC00000F058F805461A20FFF762FF4E480021C0
:109DD0004160016001604168214341601A20FFF742
:109DE0004FFF2846BDE8344048490968084738B560
:109DF000474C0546206808B1FF2032BD00F03AF814
:109E00002560E1690029FCD00021E161E1612BE0DE
:109E100038B53F4C0546206808B1FF2032BD00F040
:109E200029F86169E26800236361E3602560E36902
:109E3000002BFCD00023E361E361EB070CD42B88FB
:109E40001B0509D56368012B06D123699B07FCD547
:109E50006FF0030323612361CB4323612361D34369
:109E6000A360A3606161E26028490968884760686F
:109E7000C0B232BD22480068004780B51F48406824
:109E800001001CBFBDE802400047FFF7F3FF214976
:109E90004A688B689A430DE080B5184880680100D5
:109EA0001CBFBDE802400047FFF7E4FF19494A68BC
:109EB0008B681A40D2430A600A6014490968BDE8F9
:109EC0000440084780B50D48C06801001CBFBDE8CC
:109ED00002400047FFF7CEFF0B494A68EAE70E4809
:109EE00000210160016005480068010018BF0047BB
:109EF00070470000304800202C4F0020EC4F00201D
:109F0000344800200C100440081004403848002059
:109F100000100440101004401C10044010B40B4BFF
:109F20001C6824F480641C600902090CA4B21202AB
:109F300044EA014402F4706242EA0141C0F387102E
:109F40001C600843586010BC704700001480024039
:109F50000022F8F711B90000DFF800F0D558001022
:109F60002DE9F84304462448007801280F46154699
:109F7000994608D121480188491E018089B211B94A
:109F80000120FFF7E9FFDFF8788098F80000FF264E
:109F900078B10C20F6F7DAFE48B3902101704670D4
:109FA000022101714480C5808760014698F8000055
:109FB00019E00820F6F7CAFE010018D00120087049
:109FC0004E70781F48600222027048684470200A70
:109FD0004A6840EA091090704868C57000204A68D5
:109FE000107108480078BDE8F443F6F7D0BE384653
:109FF000BDE8F243F7F7D1BC244F0020264F0020E4
:10A000007B480020784800200A460146012002E0F3
:10A010000A460146022070B50C46150018BF002CF8
:10A0200001D1022070BD1070D61C20785070751CB4
:10A0300060789070201DF9F761F83070207A2870F0
:10A04000E068000A00F001006870E168C1F3402197
:10A0500001B1022108436870E168C1F3802101B1B8
:10A06000042108436870E168C1F3C02101B10821EF
:10A0700008436870E168090B40EA01106870207BB2
:10A0800000F00100A870E168C1F3400101B10221B4
:10A090000843A870E168C1F3800101B104210843BD
:10A0A000A870E168C1F3C00101B108210843A8709C
:10A0B000E168090940EA0110A870002070BD38B5B8
:10A0C00005000C4618BF002C01D1022032BD687873
:10A0D0002070A8786070201DE978F9F71FF82879BA
:10A0E000E168207221F48071687900F0010241EA90
:10A0F0000221420821F4007102F0010241EA4221EA
:10A10000820821F4806102F0010241EA8221C20842
:10A1100021F4784102F0010241EAC221000941EA3A
:10A120000031E1604908A87900F0010242EA4101EA
:10A13000420821F0020102F0010241EA42018208D4
:10A1400021F0040102F0010241EA8201C20821F07B
:10A15000F80102F0010241EAC201000941EA0010DF
:10A16000E0602120FCF73CFB217A814205D32220CC
:10A17000FCF736FB217A884201D2122032BD2078CA
:10A180000528BCBF6078022801DB182032BD002002
:10A1900032BD80B50B0018BF002801D1022002BDDE
:10A1A000032112E080B50B46002818BF002B01D117
:10A1B000022002BD411C10220BE080B50B0018BF2D
:10A1C000002801D1022002BD042103F8011B102246
:10A1D00001461846F6F76BFD002002BD80B50B4620
:10A1E000002818BF002B01D1022002BD411C102203
:10A1F000EFE7002918BF002801D10220704705228F
:10A200000A700078487000207047002818BF0029A5
:10A2100001D102207047407808700A2800DA08B996
:10A22000182070470020704780B50B0018BF002829
:10A2300001D1022002BD0621C7E780B50B460028E8
:10A2400018BF002B01D1022002BD411C1022C0E723
:10A2500080B50B0018BF002801D1022002BD0721E4
:10A2600019700822018859700188090A9970811CA7
:10A27000D81CAFE780B50B46002818BF002B01D1D2
:10A28000022002BD10F8011F427801EB0221198063
:10A290000822811C981C9DE780B50B0018BF002880
:10A2A00001D1022002BD08218FE780B50B0018BF45
:10A2B000002801D1022002BD09211970062201786F
:10A2C0005970411C981C85E780B50B46002818BFC3
:10A2D000002B01D1022002BD411C102279E780B57C
:10A2E0000B46002818BF002B01D1022002BD417887
:10A2F00019700622811C581C6CE780B50B0018BF32
:10A30000002801D1022002BD0A215EE780B50B467C
:10A31000002818BF002B01D1022002BD411C1022D1
:10A3200057E710B50C0018BF002801D1022010BD5E
:10A330000B212170F8F7E2FE6070002010BD80B59F
:10A340000A46002818BF002A01D1022002BD417828
:10A350001046F8F7E3FE002002BD70B5044684B055
:10A3600008460621ADF80010ADF8080015461E4657
:10A37000F8F766FD010001910DD02846B0470500B1
:10A3800004D100A92046F7F774F9054625B10198D4
:10A39000F7F703FB00E01325F8F7DDFD284604B0CE
:10A3A00070BD000062B38B0708D0521E11F8013B4C
:10A3B00000F8013B00F024808B07F6D1830740F0C2
:10A3C000208000BF103A07D330B4B1E83810103AFB
:10A3D000A0E83810F9D230BC530724BFB1E8081008
:10A3E000A0E8081044BF51F8043B40F8043BD207F2
:10A3F00024BF31F8022B20F8022B44BF0B780370E6
:10A400007047083A07D3B1E80810083A40F8043B0F
:10A4100040F804CBF7D25307E4E70000DFF800F080
:10A42000C59B0010DFF800F0E19B001080B5DFF85D
:10A430004405007840074CBFDFF83C050020FEF7DC
:10A440004FFB002002BDF0B589B004460D4616460C
:10A450001022002100A8F6F75CFCDFF820753868B0
:10A4600050B38188A14204BF0178002924D14178EA
:10A4700006290DD100F1550200F1350104AB0C3075
:10A48000F8F709FEC0B9FEF704FE024604A924E06D
:10A49000806E88B1028A112927D1964209D100F035
:10A4A00033F8012805D1FEF7F4FD02463868816EC5
:10A4B00013E03220FEF7D5FD2046F6F713FB070028
:10A4C0001CBFB86A002819D0018A8E4216D100F04C
:10A4D0001BF8012812D1B96A8A7E00A8F6F7E7FBBB
:10A4E00000A92046FFF79AFF0BE09642E4D100F066
:10A4F0000BF80128E0D13868816EEDE72046FFF7C0
:10A5000091FF012009B0F0BD00F112010822284698
:10A51000F6F7F1BBF0B5DFF864640746306885B044
:10A520001546002480B9012913D1281DF8F7E6FD4E
:10A53000E9680291297A019100906B782A787988EC
:10A540000020FCF735FECAE082887B889A4218BF5B
:10A55000082040F0C5800278012A08BF072000F0DB
:10A56000BF80491E092956D8DFE801F005550A22A7
:10A57000B63F577487A0284600F0B8F80446AEE00E
:10A58000102229464530F6F792FB306841780429BD
:10A5900008BF03215DD000F1250200F135010C3028
:10A5A000FEF791FBFEF727FC00B10824052061E0CF
:10A5B000102229465530F6F77AFB306800F1550134
:10A5C00000AA0C30FEF77FFB306800F14501102235
:10A5D00000A8F6F790FB012805D1FEF718FC00282B
:10A5E0006CD1062046E0042479E041780C2912D190
:10A5F000C06E20B91C20F5F7EDFC3168C8663068E4
:10A60000C06E40B100F06EF8FEF743FD3168C96ED0
:10A6100088760D202EE0072461E0C36E002BFAD06F
:10A6200040780D28F7D1288818820822A91C03F148
:10A630001200F6F73CFB306881684969C1F340229B
:10A64000002A1FBF026AD268C2F34022002A20D02B
:10A650000E2129E041780E29DDD1006F20B91620A6
:10A66000F5F7B8FC316808673068006F08B100F092
:10A6700039F80F203168487031E041780F29CAD18C
:10A68000006F0622691C1030F6F711FB30688168F4
:10A690004969C1F3802100291FBF016AC968C1F35C
:10A6A0008021002916D01021417018E0406F38B980
:10A6B0001420F5F78FFC3168486708B908240EE0CC
:10A6C0003068406F30B100F00DF83168496F4FF0DD
:10A6D000FF300861002000E02878FEF7C2FC204629
:10A6E00005B0F0BD10222946F6F7E1BA38B5FEF7FD
:10A6F000A3FB0024002844D1FEF767FB9F4D286888
:10A700008168897CC90709D5016A097901F00301CB
:10A71000012903D1017F41F001010177286890F8F8
:10A720002410022904D0032918BF042909D10121CA
:10A730008088FCF76DFD00F02AF804202968487035
:10A7400023E0012918BF05291FD102214170286883
:10A7500000F108010A7F012A05D1102200210C30E6
:10A76000F6F7D7FA07E009681022891C0C30F6F7D3
:10A770009EFA00F00CF8102128683530F8F7ABFC91
:10A7800003E018280CBF03240824204632BD2868A3
:10A79000017F41F00401017770472DE9F041774CCA
:10A7A00020680178002940F0E3804778D0F80880DD
:10A7B000066A062F2FD1D8F81410CA0704D5327BA9
:10A7C000D20748BF072730D4C1F34002002A1EBF7A
:10A7D000F268C2F34002002A08D00927FCF772F998
:10A7E000014620688088FEF7FDFB10E0C1F3800180
:10A7F00000291EBFF168C1F3800100290BD00B278F
:10A80000FCF73FF9014620688088FEF702FC072F1D
:10A810004ED108208EE0072F07D0F8D3092FDDD0C6
:10A820002BD30B2FECD031D3F1E7806E20B91C2055
:10A83000F5F7D0FB216888662068856E002DE6D08C
:10A84000FEF727FCA876102200212846F6F761FAC9
:10A85000A97E21B11129BCBF2846F8F73CFCF6F7C8
:10A8600062FA2882082105F11200F8F734FC20680A
:10A8700080882946FEF79FFBC9E7816ED1B101F1BF
:10A880001202098A8088FEF799FB13E0FCF70DF9A4
:10A8900001270546012D0CBF002700253846FCF78F
:10A8A00007F90246206880882946FEF7A0FB14E0DD
:10A8B000082F0CD1D8F81400C0F3400000281EBFA8
:10A8C000F068C0F34000002807D0092032E0092FCB
:10A8D00008BF0A202ED00A2F0BD1D8F81400C0F3DD
:10A8E000800000281FBFF068C0F3800000280B2004
:10A8F00020D1D8F81400C0F3002100291FBFF1684F
:10A90000C1F3002100290C2014D1C0F340210029FB
:10A910001FBFF168C1F3402100290E200AD1C0F306
:10A92000802000281EBFF068C0F38020002814BFDC
:10A93000102012202168487020684178072918BF2C
:10A94000082904D009291CBF0A290B2910D18088A5
:10A95000F6F7C8F8BDE8F04100281ABFC08900EB3F
:10A9600050024FF4FA72064800780221F7F773BCE0
:10A97000BDE8F081054500204C4600203C48002001
:10A98000B5480020DFF800F021870010DFF800F064
:10A9900041870010DFF800F031860010DFF800F08A
:10A9A000B5C10010DFF800F0F1860010DFF800F00C
:10A9B00069800010DFF800F05D920010DFF800F011
:10A9C000957B0010DFF800F0557C0010DFF800F0F8
:10A9D000F5B50010DFF800F0DD930010DFF800F0AF
:10A9E0003D930010DFF800F0A97C0010DFF800F0C4
:10A9F000557D0010DFF800F0E1910010DFF800F065
:10AA0000297F0010DFF800F0A1AF0010DFF8C006CA
:10AA10008178FF2900D170472DE9F84F40684FF445
:10AA2000907202FB010400F030FA02FB010000907A
:10AA300004F20B100178012908BF417800F08B80E7
:10AA400004F1740504F58C76287B022804BF0020ED
:10AA50002873F18811B13079F6F76FFA6089208197
:10AA6000DFF87006817A90F807C090F80C90C37AEE
:10AA7000427B01EB0C0ECE449E4402EB0E0704F524
:10AA8000877E1FFA87F8BEF804707F1CAEF804704A
:10AA9000BEF800704744AEF80070BEF80270CF19DF
:10AAA000AEF802703768DFF830666FB196F80EA026
:10AAB00037F81AB0D84427F81A8007EB4A08B8F8D4
:10AAC0004A70CF19A8F84A70BCF1000F08BF002BDC
:10AAD00004D1B9F1000F08BF002A22D02189E289F0
:10AAE0005118A18100212174217F012904BF618CAB
:10AAF000E183417859B101212177A978002904BF68
:10AB0000297B002903D1A97E09B9618CE1830099D1
:10AB100024310A7C42B3022A04BFC27A002A1FD120
:10AB200021E0E28339B100212174217F012907D17D
:10AB3000618CE18304E0BEF80610491CAEF80610F3
:10AB40002189A2898A42D4D1207C08B1052901D06B
:10AB5000082100E03E212046BDE8F44FFFF71ABF70
:10AB6000427A0AB102220A74C37BDFF87025DB0740
:10AB700007D50169183101612368D960002151614D
:10AB800006E052690A602268B168D1600021E18361
:10AB9000DFF84C154969097889074CBF807B812013
:10ABA0002870204600F076F901280BD001212046BC
:10ABB000FDF7C9F800F008F801281CBFBDE8F14F07
:10ABC000F8F7D6BCBDE8F18F2DE9F843DFF80005B2
:10ABD000416880784FF4907202FB001400F055F940
:10ABE00004F1680502FB01082868006804F18E077B
:10ABF00008B100200CE0A87B002804BF287E0028B4
:10AC000007D13878002804BF207F012801D1608C4B
:10AC1000E0832089E18B0818401C60812046FFF703
:10AC2000BDFE01281EBFDFF8BC040078012801D159
:10AC300000F025F9287E01280CD16A8B61892089D2
:10AC4000FFF7B0FE30B121896289481C82421AD0D8
:10AC50006A8B0FE03878012815D17A8861892089BC
:10AC6000FFF7A0FE00281FBF2189481C628982428D
:10AC700009D07A88824206D0501E608180B2FCF7EB
:10AC80003DFF401EE08308F1240898F8100008B149
:10AC900000F0F5F804F12E07287E012801BF688B2B
:10ACA0002189491C884237D1608104F18401204602
:10ACB000FFF768FE688CE189608400202077E083DC
:10ACC00060890818A0812189688BFCF717FFB98873
:10ACD000EA8BB5F820C001FB0026A88C8C4504BF88
:10ACE0003989884202BF698CFA88914206D00309EB
:10ACF0006A8CA0794FEA5C01F9F737FB287F38703E
:10AD0000288CB880688CF880A88C38812046FFF7A2
:10AD10003DFE0220287600E0BE88E08B2268D2F853
:10AD20000CC0401C00FB06F3DFF8BC6340F6C41007
:10AD300000FB03F18C44C2F80CC03668DFF8ACC3EA
:10AD40003678BCF800E0DFF88C23B609032E12D168
:10AD5000D67BF60748BF4FF0000E0CD40EF101066B
:10AD60001FFA86FEBEF1010F12BF668AB8F80E60A8
:10AD700006F2DC5600E0668A5E434FF4C879B6FB03
:10AD8000F9F6761C6661ACF800E0A361E38BD4F8B9
:10AD900000C084F82030D04B9E68DCF80CE0CCF882
:10ADA00010606669AEEB06069E60CCF80860DFF8BE
:10ADB0002CC31E7B06F0F00646F002061E7300262A
:10ADC0005E80DCF814E066690EEB4606CCF8146091
:10ADD0002D7E022D04D13D7800FB0565CCF8145082
:10ADE000D57BED071DD59D68A5F5A8659D60691A01
:10ADF0002668B5603161DCF8141001F5F661CCF815
:10AE00001410C8F80010B988B94D00FB0150CCF8F7
:10AE10001C00B848007801281EBFB148806A4078FD
:10AE20000FE0BD88DCF814104543A1F5E661A5F5F7
:10AE30001675A942E7D308212046FFF7ABFD012094
:10AE40001BE08CF80B00AC492068436000201070B8
:10AE500050709070D070107150719071D0711072EC
:10AE600050729072D07210735073D07310610720BB
:10AE700008702046FDF75BFA0020BDE8F283002051
:10AE8000E0832089401C608170479C48A17900685C
:10AE9000382270472DE9F04782460AF106069748A6
:10AEA000317800688B4C382282B002FB01080AF12D
:10AEB000E3090AF1E8070AF1660507E05046FFF7E3
:10AEC00075FD012835D15046FCF7E4FF687D80B35D
:10AED000687C02281BD004282ED0052842D00628E2
:10AEE00071D00728EAD0092800F0BF800B2800F0B5
:10AEF0008F800C2800F0C6800D2800F09E80FC2872
:10AF000017D0FD2800F0DD80FE28DFD111E0287C7D
:10AF1000012808D1E07800285AD016215046FFF7C2
:10AF200039FD012006E05046FDF737FA2874E88A1B
:10AF300028830020BDE8F687287C01280ED1A07860
:10AF4000002845D0FC215046FCF7C2FF30780AF1BA
:10AF5000B4020AF1AC01FFF72DFDB7E75046FFF749
:10AF60002DFDE3E7287C01280FD1A07828B101202E
:10AF70008AF89200002038607860B87A01286BD196
:10AF800006215046FCF7A4FFA0E799F8000001282D
:10AF900009D15046FFF716FD0128CAD10020B8722A
:10AFA00001202874C5E799F801000028C1D00AF1F2
:10AFB000C3020AF19C010AF1D300FFF707FD01204B
:10AFC00089F8000082E7287C01281DD1A07800289C
:10AFD00042D0B08B30835046FCF75CFF00F09CF809
:10AFE0000120A871397A3078012903D10021FFF7B7
:10AFF000F1FC03E001220021FFF7F0FC0020387291
:10B000003873F872B87261E75046FFF7EBFC8DE7D2
:10B01000287C012805D1F87A012808BFFC21B0D08E
:10B020001AE05046FFF7E2FC0128BBD10020F8727D
:10B030008AF892000120287448E7287C012810D162
:10B04000A07830B100208AF8920000F065F8012065
:10B05000A871E078002810D100F058F8A2D1222180
:10B060005CE75046FCF75EFD60E7287C012805D1CF
:10B07000A0780028F0D0B08B308324E75046FCF74E
:10B080002FFE53E7287C012815D1787E012808D1AE
:10B09000B87E012804D100F033F80020FFF7AAFCA5
:10B0A00011E700F033F87FF444AF00F029F82220D4
:10B0B000FFF7A0FCD3E70120F8765046FFF79EFC8F
:10B0C00034E798F820105046FCF702FFB2E7000082
:10B0D000B04C0020704E0020E04D0020384D002084
:10B0E000A4C80100894C00201C480020B048002062
:10B0F000F0DDFFFF864C0020B84C002014480020F3
:10B10000388C0090FB8B3A7F31787047288B401E3B
:10B11000288380B200287047012028705046FFF72E
:10B1200071BC000080B500F067FB02E080B500F064
:10B130005FFB00B10120C0B202BD81B001208DF8DB
:10B1400000009DF800000028FBD101B0704780B5D9
:10B150000948804709490A4809680160094909689E
:10B1600041600949096881600FF22001C1600FF256
:10B17000B801016101BD00000150001030480020FD
:10B18000E84800203448002038480020D5FF00005F
:10B19000EFFF00002F2401004D0D01008F0D010075
:10B1A0003B0F0100AF0C0100130D01006D190100F0
:10B1B0009B190100E519010057220100AD22010091
:10B1C000D90F0100F121010025B101002DB10100CD
:10B1D000A5C7010007C80100F5C90100917A010067
:10B1E000B17A0100C377010031780100477801008E
:10B1F000C5790100537901005D740100797A01007D
:10B200008B7A010011760100877601001579010023
:10B21000784800207B4800207A4800207C480020A5
:10B2200079480020A4C80100DD8A0010A18B00101D
:10B230002D8A001025950010F1A0001009A1001022
:10B24000799D001063200100AD9D0010D19D00107C
:10B250003F20010011A00010699F0010ED9E00101A
:10B2600095A00010D1A00010F19F0010AD9E00101D
:10B27000CD9E00108D9E0010B5A10010459D0010C0
:10B2800095A1001075A0001031A000101120010040
:10B29000B19F00100D9F00104D9E0010819F001067
:10B2A0002D9E0010D19F0010D59C0010499F0010CA
:10B2B0006D9E0010099D0010F58B00103196001056
:10B2C0005D960010159A0010F999001001200100F8
:10B2D0003BB101003BB10100F59A0010E19B001069
:10B2E000C59B0010519B0010F59800105D1F0100D8
:10B2F000A19A0010299800108B1F0100159C0010C6
:10B30000C9990010C71F0100319A0010A1980010C0
:10B31000D99800106D980010672001003BB1010022
:10B32000499800103BB101003BB10100BD980010ED
:10B330003BB101008D9C0010B51F0100714401005C
:10B3400065970010C71E01003D9700109D20010069
:10B35000419500108D970010D1950010A51E010099
:10B36000CDD70010818C0010598C0010318D001049
:10B37000E9940010F595001071950010691E010008
:10B380004F450100A194001039570010818D001025
:10B390003BB10100195700108D6700103BB101004F
:10B3A0003BB10100AD8E00103BB101003BB101008B
:10B3B000D5580010973F010071940010CD3E010058
:10B3C000DB3D0100395A00100590001039B600101D
:10B3D000F5B50010DDB9001051B8001065B90010C6
:10B3E00021B7001055B5001041B5001069B5001027
:10B3F0000DB500101DB50010C9B400108DB50010BA
:10B40000EDB40010257000105F4201007D6B00104C
:10B4100041420100816B0010856B0010A17000108B
:10B420004D6F0010D16D00101D700010ADA2001006
:10B4300021700010496F00100D400100593D0100BE
:10B44000016C00100D710010596B00100971001093
:10B45000ED6F0010996F001059A20010D570001008
:10B46000FD6E0010016E0010C56B0010F96E00102B
:10B47000D33B01003B3C0100D96A001001A200103F
:10B48000856E0010DD6B0010033C010011A200105E
:10B490003D930010DD9300104B3B0100053B010084
:10B4A0005D920010D557001089350100B957001082
:10B4B00039380100015800106D550010F557001083
:10B4C000D5A1001005610010C9560010A159001047
:10B4D000795800109D580010853B0100F943010088
:10B4E000E9580010E1910010D559001011420100F7
:10B4F000573C0100A1570010655700104139010069
:10B50000619F0100D5400100895F0010695E001055
:10B51000E95600103BB101003BB101002D61001064
:10B520003BB1010049550010953C0100D9D20010F3
:10B53000ADD10010F5D1001025D400106DD200104F
:10B540003DD2001029D2001089D100106DD3001017
:10B55000DDD300102785010051CD001025C3010067
:10B5600071CC0010AD7B0100AB8401003BB1010048
:10B570004DD90010B5C10010A5730010E97200107C
:10B58000B17D010031860010418700102187001035
:10B590008589001065890010957E010021890010C1
:10B5A0007DC80010E5720010ED720010BD80001023
:10B5B00089880010B58800103BB101003BB1010043
:10B5C0003BB1010019870010F186001039A9001065
:10B5D00095A80010EDAB00103BB101003BB101009C
:10B5E000A9AC00103BB101003DAC0010C1D8001067
:10B5F0004B7F0100FD7E0100E5820100E1AC0010FF
:10B6000009B000105D850100058501008F820100F1
:10B610003BB101003BB101000D720010C97C01007B
:10B62000B5D800103BB101003BB101003BB10100B6
:10B630003BB10100F1890010D9890010A1AF0010C1
:10B640003BB10100B1AD001065860010A38201007E
:10B650003BB101003BB10100477D0100F1720010D8
:10B660003BB10100D985010095AE01005989010067
:10B6700041AE001045AE001049AE001061840010CC
:10B6800029840010D17E010001720010D3810100D5
:10B69000697200103BB101008D85010035A30010D7
:10B6A00079840100E17200102F8301005D820100A6
:10B6B000E5730010B1AE00103BB10100A988010094
:10B6C0003BB10100957B00103BB10100E17C010022
:10B6D0003BB101003BB1010021AD00103BB10100C5
:10B6E000C9AB01003BB10100557D0010C9AD001090
:10B6F000F57D00106DAD00103BB101003BB10100C4
:10B70000557C0010A97C00109B830100698000100B
:10B710003BB101003BB10100297F00100DAA0100DF
:10B72000C9D80010F5D800103BB10100C98700103E
:10B73000E1D9001011840100ADBE0100ADC00100CF
:10B7400061C20100DB1E01003BB101003BB1010001
:10B750003BB101003BB10100593A01003BB101008E
:10B760003BB101003BB101003BB101003BB1010025
:10B770003BB101003BB101003BB101003BB1010015
:10B780003BB10100A57F0100FB7F01003BB101003F
:10B790002D7B01003BB10100238101006188010084
:10B7A0002D430100D91F01003BB101003BB1010055
:10B7B0002D4201003BB101003BB101003BB1010052
:10B7C0003BB101003BB101003BB101003BB10100C5
:10B7D0003BB101003BB101003BB101003BB10100B5
:10B7E0003BB101003BB101003BB101007D83010091
:10B7F000EFF3108072B67047EFF3108062B67047B7
:10B800002DE9F0410FF2B0102449272250F8043BF3
:10B8100050F8044B50F8045B50F8046B50F8047B6C
:10B8200050F804CB50F804EB50F8048B41F8043B7B
:10B8300041F8044B41F8045B41F8046B41F8047B88
:10B8400041F804CB41F804EB521E41F8048BDDD1E2
:10B8500042688368006808604A608B60BDE8F081D8
:10B8600010B50F4C0F4800F029F814D1EC220FF25C
:10B870005C010D48FEF7A6FD0C48002101700C4943
:10B88000C0F80D100B49C0F82D10FFF7B9FF0A489A
:10B8900000F014F800D0002010BD000000C000210E
:10B8A000001004404100070604040021A303002106
:10B8B0000904002149040021010007062060606896
:10B8C0000028FCD060680128704700007104002146
:10B8D000F0B5174C40216118C878022805D00948F6
:10B8E0000021016008498847F0BD256E074E35608C
:10B8F000600728432066276824600E488047276039
:10B900003560F0BD2C110440A565000028400440BE
:10B9100010B5074CA17D002905D10121A175480270
:10B9200004493E3988472068002800D0804710BD70
:10B93000540200218B390000F8B51A4E0546316BD0
:10B940001948CC09E401002D11D0184909780229C1
:10B950000FD0007B044372B60120154F4002B84758
:10B96000114820380088C109C90704D016E0C07A00
:10B97000F0E7407BEEE70F493463CC61400AC00733
:10B980000CD001208003F16A002D01D0014300E0BA
:10B9900081430846F1620749403948630020B847AF
:10B9A00062B6F8BD800200218800002196020021C5
:10B9B000DF3C000040400440546100007F1402005E
:10B9C000060005000F0008004800520080FF3F00FD
:10B9D0000000000000000000000000000000000067
:10B9E000304000400140034007400F404F40CF40EF
:10B9F000CF41CF43CF47CF4FCF3FCF2FCF1FCF0F19
:10BA0000000000000000000000000F00080000001F
:10BA10003F00000040003F000000040068000E00EE
:10BA2000DC00060043001A000500000000000200D0
:10BA300000000000000000000400C000000004003E
:10BA4000C00000000700000000000000000000002F
:10BA5000000000000000000050C00091007070C0A5
:10BA60000091007082312100319110B1007001818C
:10BA700001B100A18231329110B1019111104181C7
:10BA800041226340F106007051C001913018103915
:10BA9000833108D01831416F3100319110B18314D6
:10BAA00014166F680070251050C00091F4C340C197
:10BAB0002014036F311041045082F022844051263B
:10BAC00022C082312100319110B16339311041041B
:10BAD00082C082312100319110B163393110A2C08E
:10BAE00082312100319110B15010153105140592A9
:10BAF0000070536452C0311031066131C102566486
:10BB000012C13110213971065131E10256640070C1
:10BB100051C0019101CCE2C05664536411C1C2C04E
:10BB2000566454B0007154A064B0F0800022B54057
:10BB300011C122C1566451C00191E2C082316082BC
:10BB40000200329110B100C3C86853644012B09033
:10BB500032B000C3CE6840C2D0688012B09032B01C
:10BB60000070536401C122C1566401C1C2C0566451
:10BB700053829D64C012B09032B00070536472C2A0
:10BB800081C0566422C111C1566402C011C15664FD
:10BB900062C031C3566462C311C1566402C311C18D
:10BBA0005664538253399D64E2C35B641122F840AA
:10BBB00042C281C8566452C211C1566472C2E1CEFB
:10BBC000566402C281C8566402C201C85664B0C03D
:10BBD0000C690070536442C201C8566452C211C05D
:10BBE000566472C2E1C0566402C001C1566462C0AC
:10BBF00001C3566422C101C1566462C301C15664C7
:10BC000002C301C1566453829D64007002C1623157
:10BC100001C0A080001E3241101A34612010101A99
:10BC2000136F236E1116121634690070E092D082E1
:10BC300000223B45C0B20070000000000000000080
:10BC400000000000000000000000000000000000F4
:10BC500000000000000000000000000000000000E4
:10BC6000067305720B720E7250B00071818060B065
:10BC700050A09280F0EFF19202933A65412278450C
:10BC80008080F1C11004301601110114016C8B6128
:10BC90008C618D618E618F6190619161936195611D
:10BCA00097619961706273629180F2C021042131C1
:10BCB0008280422A1214321601112114016CA661ED
:10BCC000C761AC617362A661C761AC6173629B615D
:10BCD0009B619B619B619B619B61AC649B61D56433
:10BCE0009B61E2649B610E659B612A659B6182801A
:10BCF000E0DFF2923A65B0B0A261B1B006730572AE
:10BD000030B05861D0CF3A6584C203C0C0C3686404
:10BD100090785091607810316178101400925078CA
:10BD20004031617810004031717810001092B07885
:10BD300060928178219230784031417810003092C1
:10BD400010C0F0919B6154A0F0805022CF454080FC
:10BD500000226646C76100C86091598150B0918049
:10BD600041222E46C0CF3A65128282318239423951
:10BD7000281077641282F11212042F101F312F1431
:10BD800040C120140D6F6D39DE10F4C34E0482C023
:10BD900082312E006D39A2C082312D001A828A397B
:10BDA0002082803180390BC00B18AC78308240394A
:10BDB000021011C0013010C0011802188231210098
:10BDC000C126919103B013B063B053B0038239140C
:10BDD000418001226646B481C491D5819518B51C75
:10BDE0001C4EC51C544A6591F08010220C422C62F6
:10BDF0003D9110B13E9110B165910F925981F914A6
:10BE0000AB18BC10F0805022C74110222C460C62A7
:10BE1000B0CF3A6563B030820010F2C02004021047
:10BE200011C0013010C00118021882312100C12652
:10BE30009191919113B003B063B053B064B054B01A
:10BE4000007141800122664663B064B0F0805022E8
:10BE5000C741B181C191D1819118619131B04462E2
:10BE600012828231823942392810776459810582E1
:10BE7000591420820BC00B18AC7880C0007163B0DD
:10BE8000626A0C62018262818231823DA0EFF1928E
:10BE900002933A6503A09B61A28077649B6150B0D6
:10BEA00000719B61DFF800F0DDB90010F8B500F01B
:10BEB000D4F9DFF8F813DFF8F8230C6802EA04037A
:10BEC000DB430B600B6823401342F7D100F0C2F94B
:10BED000002C04D58220FCF79BFAF7F7F1FADFF883
:10BEE000D40301680A0006D0A20704D5002202602C
:10BEF000BDE8F140084714F0030F74D0DFF8B81321
:10BF0000DFF8B8030B784488DFF8B413DFF8B453D4
:10BF1000DFF8B4231E0066D05E1E032E0DD9B61FB7
:10BF20005FD0B61E012E40F28C80B61E012E40F26C
:10BF30009B80B61E00F09B80B2E0DFF890030D609E
:10BF400041F204454488AC421FBF468BAE42468E48
:10BF5000AE4204D11580DFF8780308606AE0022C55
:10BF6000DFF8705314804FF4A05641F2024736D9DF
:10BF70004FF4806CB4EB0C041BD0241F012C1ED991
:10BF80004FF47F7CB4EB0C041BD04FF44060241AB8
:10BF90000FD0A41E012C0CD9241F0AD0641E012C22
:10BFA0000DD940F2F930241A012C18D9241F14D0CD
:10BFB00076E0022B14BF1680C74D0D603AE0C74DE6
:10BFC000FBE7C74A927C012A03D147804783478613
:10BFD000F3E7468046834686EFE7872061E08320CB
:10BFE0005FE000F033F960D0BE480D6040F20444D9
:10BFF000438813801B1B012BBB4A56D94FF47F7417
:10C000001B1B0FD04FF440641B1B032B84BF5B1F13
:10C01000012B0AD99B1E012B47D940F2FD341B1B73
:10C0200005D102E041F2014343800A6002E085202D
:10C03000FCF7EEF9BDE8F440AC4800780121F4F7D4
:10C040007CBF40F204418C421CBF41F208418C424B
:10C0500014802AD041F604018C4206D1A449096912
:10C060008969BDE8F44008471480852019E01480F0
:10C0700040F20441641A18D040F6FC71641A05D0ED
:10C08000083C12D04FF47F71641AEED1817B891C79
:10C09000C9B2B529A8BF6621817300214180F1BDD5
:10C0A0008420BDE8F240FCF7B3B9F1BD2DE9F047BB
:10C0B0007E4C82B0606820F0C040606000F0CDF837
:10C0C00025688C4A02EA0501C9432160216829409C
:10C0D0001142F7D100F0BEF87748007805281CBF60
:10C0E000082807284BD168050BD500F0AFF834D0ED
:10C0F000814A52684FF49073002103FB0020FBF744
:10C1000022FE280240F19B806B480078C01F012866
:10C1100000F2928000F09AF81FD0774949684FF4F6
:10C12000907202FB001A72490969096E0AF16C05E6
:10C13000686888470646D6F8088018F8010B18F892
:10C14000017B10F0030914D0B9F1030F06D00FB131
:10C15000287870B169480078012875D09AF8920063
:10C1600090B13F1F4346FAB249465046FFF79AFE48
:10C1700030B90AF20B103D2141700121017063E0DA
:10C1800000F06BF800F066F8B9F1030F46D05C4898
:10C19000D0F814A09AF801001F3080B2FBF7AAFC77
:10C1A000B06038B9F0804FF4807150480078F4F7EF
:10C1B000C4FE05E0801EB0609AF801002130F080D6
:10C1C0009AF80000810708D5C0074CBF0320002063
:10C1D000FFB2C01910F8080000E081202872494819
:10C1E00000781C2812DA287A802818BF81280FBF0F
:10C1F0007F2045490978401A40B200904B463E489E
:10C200008078FAB24146FDF7ABFE0FE03A488078FD
:10C210004B46FAB24146FBF7F0FE07E026480078AD
:10C22000082803D041465046FCF7D6F93049096941
:10C230006868896E884702E08620FCF7E9F8206884
:10C240002C4908427FF43AAFBDE8F3872A4880784A
:10C25000FF2870472D49096808472D4800680047A6
:10C2600070B5FFF7FAFF04462A480168426802EAFF
:10C270000105E94315F47F2F016010D00026264800
:10C2800000EBC600417839B901780C3125FA01F28A
:10C29000D10744BF40688047761C042EEFDB204660
:10C2A000BDE87040194909680847000010100440B3
:10C2B000030000808C460020B84C0020284E00204F
:10C2C000C44C0020E1D900100A4F0020244C00206B
:10C2D00025C3010071CC00107DC8001051CD0010A5
:10C2E000EC490020E04D00200DAA0100844C002004
:10C2F0002C4F002000048000B04C00208A4C00200D
:10C30000A4C8010010480020C04C0020384800207C
:10C310003448002008100440AC4F0020DFF800F043
:10C320004DD900102DE9F84F0120FCF7EBF801285A
:10C3300040F07181BA4CBB4EDFF8EC92DFF8ECB202
:10C340000020A0732046F7F71BF9FBF72FFC0546EA
:10C350000120687105F12C07B5484178491C4170EE
:10C360004020FCF7A2F8B34928600968AA7938236D
:10C3700003FB0213B049CA681832CA6002F5B06103
:10C38000C16003F128083068006800F1080A06223D
:10C390009AF80000C0F3801088F800000AF102014A
:10C3A00003F12C00F4F783FC04220AF10E0109F1D9
:10C3B0000C00F4F77CFC03220AF1120109F11000D1
:10C3C000F4F775FC9AF81500B87002220AF116010C
:10C3D00005F13000F4F76BFC02220AF1180105F1B7
:10C3E0003200F4F764FC02220AF11A0105F122007E
:10C3F000F4F75DFC0020388102220AF11C0105F1EE
:10C400003600F4F754FCB8784000B870B8884000A3
:10C41000B880F8884000F88080B279890901798174
:10C4200043006A8C521C5A4389B28A4200D230B906
:10C430009BF800008021F4F780FD3B216FE005F1BF
:10C440002E012846FEF79EFA0520A8812846FEF711
:10C450009DFA05220AF11E0105F16100F4F727FC9F
:10C460009AF8230040093870FFF758FF6882E18A84
:10C47000724C401AA8F80A0005F161019AF82300ED
:10C4800000F01F00F8732846FBF70BFF31686C4E75
:10C49000096800200871012141F601002080002078
:10C4A000608060602846FBF71DFFA073C4F8109001
:10C4B0000020E0736661634841690A78D1074CBF88
:10C4C0001021002193074CBF202300235FEA427A0A
:10C4D0004CBF4FF0400A4FF0000A12074CBF8022B9
:10C4E000002219434AEA0101114341F00F0189F882
:10C4F00008100B2189F80910042189F80A10524903
:10C50000097801290EBF0120806A407889F80B0064
:10C51000A879FCF7C9F9C9F8000020B90721284615
:10C52000FEF738FA77E0DFF824A1A979DAF80000FD
:10C5300000EB011046490969096D8847DAF80000E7
:10C54000A97900EB0110C9F80400F8630421D9F8B7
:10C5500000007864002030707070B070F07030713E
:10C560007071B071F07130727072B072F0723073BD
:10C5700070738020B0730020F07330619BF800006E
:10C58000F4F7DBFCB8884FF4C872811C688AA96193
:10C590004843B0FBF2F0421C6A6140F6C4102B68BD
:10C5A000DE6800FB0161891AA1F5A861A1609960AC
:10C5B000217B01F0600141F002012173617B01F0F8
:10C5C000F00141F0010161732A68A1681161696994
:10C5D000BA78490000FB021101F5F661C9F81410A0
:10C5E0001C4A99F8131001F0F00141F0040189F898
:10C5F0001310F98800FB0120C9F81C00164999F8AE
:10C600001B0000F0F00040F0040089F81B002868CF
:10C61000446007200870BDE8F14FF6F7A9BF00BFDE
:10C62000EC490020584D0020384D0020844C00205B
:10C63000B04C002014480020984E0020E04D00200F
:10C64000704E0020A4C80100864C00201C4F002022
:10C650002C4F0020F0DDFFFFB84C002080B50948CA
:10C66000804709490948096801600949096841602A
:10C670000849096881600FF22001C1600FF23001A2
:10C68000016101BD014C0110304800202C4F0020F9
:10C690003448002038480020D5FF0000EFFF00009C
:10C6A0009B190100AF0C0100130D0100F5C9010039
:10C6B000CF9C01001B9D0100719D0100AD9D0100FB
:10C6C000BD9D010035890110EF9D0100119E010003
:10C6D0003D89011045890110DF9E01007B9E01000C
:10C6E000999E0100C59E0100AD82011015830110C5
:10C6F0003D8301106983011091830110158401109D
:10C70000B983011085840110A9840110C58401102A
:10C71000CD840110D1840110D5840110F984011059
:10C720004985011051850110E185011069860110CC
:10C73000756901107969011085690110996A011004
:10C74000F56A0110796B0110296C0110456C01101C
:10C75000796C0110056D0110296D0110A16D01109A
:10C76000C96D01108D6E0110A16E0110D56E011002
:10C7700065730110FD7401107D7601103978011088
:10C7800095780110F578011071770110ED750110A1
:10C79000098B0110998A0110C58A0110198A0110AC
:10C7A000358A0110042804D12F48016841F48031F2
:10C7B00013E0052804D12C48016841F400310CE055
:10C7C000062804D12848016841F4802105E00F289B
:10C7D00005D12648016841F0020101607047A0F1CF
:10C7E0001001202906D20121103801FA00F0204959
:10C7F00008607047302805D30121303801FA00F075
:10C800001B4948607047042804D11748016821F487
:10C81000803113E0052804D11348016821F4003168
:10C820000CE0062804D11048016821F4802105E0BD
:10C830000F2805D10D48016821F002010160704701
:10C84000A0F11001202906D20121103801FA00F0D0
:10C85000084908607047302805D30121303801FAB3
:10C8600000F004494860704724ED00E010E000E06B
:10C8700000E100E080E100E00061310078C80100E3
:10C88000010000000000D0020A05000000000000C6
:10C890000201000000000000100000000000000085
:10C8A000EC0000210000000061B80100A0C80100F8
:10C8B00084C801000000000088C801008CC8010085
:10C8C00090C8010094C8010098C801009CC80100EC
:10C8D0003C46002019E050F8041BCB0744BFA9F1E7
:10C8E00001035918121F0023042A41F8043BF9D20E
:10C8F0005FEA827C0B4604D54FF0000CA1F800C023
:10C900009B1CD10744BF0021197050F8042B002A4A
:10C91000E1D1704730B5016842688468014401EB99
:10C920005203D20748BF4C44994201D10C3030BD6C
:10C9300011F9012B11F8015B002A04F8015B02D503
:10C94000521CF9D1F0E7521EF4D5EDE73938010059
:10C95000EB4501000F2701009B460100D94801006B
:10C96000594B01009713010087F000003556010074
:10C97000E55901000A00000010B507497944183153
:10C98000064C7C44163404E00A68081D11448847AC
:10C990000146A142F8D110BD2C0000004800000063
:10C9A0000018000001180000002800000128000005
:10C9B0000328000002290000002A0000012A0000CC
:10C9C000042A000011FFFFFF10020000A84600200B
:10C9D0000000000041FFFFFF1E0000009002000069
:10C9E000E843002002000000A4C90100020000008A
:10C9F000A0C901007047010001FB00050577100088
:10CA0000000AF10001E803DE0000FFD90000FF8109
:10CA100000F800FEFFD60000FFEF0031B400002850
:10CA2000002800283075A000A000A000A000000889
:10CA30000008E001F00010001000100010001000CD
:10CA4000100050005000500010001000D007FA00F5
:10CA50000F0F000100050030750700100001008174
:10CA6000FFFA0000FFF1000DD39701008599010046
:10CA70002198010000FFF600049191010002FD00E1
:10CA800004A8C9010001FD0004E4C9010001F90086
:10CA9000025000A0FD0001E803E4000002FD0004D4
:10CAA000A8C9010001FD0004ECC9010002FD000459
:10CAB000B0C9010001FD0004A546002002FD0004EC
:10CAC000B8C9010001FD0004B445002002FD0004C6
:10CAD000B0C9010001FD0004A646002002FD0004CB
:10CAE000BCC9010001FD0004B045002002FD0004A6
:10CAF000B0C9010001FD0004A746002002FD0004AA
:10CB0000C0C9010001FD0006A845002003081BFB69
:10CB100000127CC801003408000015A501009BA785
:10CB2000010047A401E3000201350CFB0002801A5A
:0ECB300006EB000002F500011700FDFFFD02FC
:10D000000000000000000000000000000000000020
:10D010000000000000000000000000000000000010
:10D020000000000000000000000000000000000000
:10D0300000000000000000000000000000000000F0
:040000050000F00106
:00000001FF
